:020000040800F2
:1040000000500020A1E400083DBC000841BC0008AD
:1040100045BC000849BC00084DBC00080000000079
:1040200000000000000000000000000055BC000877
:1040300051BC00080000000059BC0008CD8B0008EE
:104040005DBC000861BC000865BC000869BC0008D4
:104050006DBC000871BC000875BC000879BC000884
:104060007DBC000881BC000885BC00080000000081
:104070000000000000000000000000000000000040
:104080000000000000000000A5BC0008A9BC00085A
:10409000B9BC0008C9BC0008D9BC0008E9BC0008CC
:1040A000EDBC0008F1BC0008F5BC0008F9BC000834
:1040B000FDBC000801BD000805BD000809BD0008E1
:1040C0000DBD000811BD000815BD000819BD000890
:1040D0001DBD0008418800087D87000829BD000833
:1040E0002DBD000831BD000835BD000800000000EE
:1040F00000000000000000000000000000000000C0
:0C41000000000000000000005FF800005C
:1041100030BF704720BF704740BF7047BFF36F8FFD
:104120007047BFF34F8F7047BFF35F8F704701DF5A
:104130007047EFF31480704780F31488BFF36F8FDC
:104140007047EFF30980704780F309887047EFF3F9
:104150000880704780F30888704772B6704762B66F
:10416000704771B6704761B6704780F31188704729
:10417000EFF31280704740BA704700BA70470000F2
:1041800037B508F05FFE524B00254FF480301D70AC
:1041900008F078FE08F0DCFF0128044626D1102044
:1041A00008F03AF9284608F0BDFE284608F0CEFE91
:1041B000284608F0C1FE4FF480304FF4802108F00B
:1041C0008DFE204608F096FE392008F0ABFF00284F
:1041D000FAD0012008F008F9012008F091FE08F05B
:1041E00099FE0428FBD13A4B01221A7004200121C8
:1041F00008F04EFF03238DF80630153301A935482A
:104200008DF807304FF48073ADF8043008F038FBB8
:10421000062008F081FF0120014608F039FF4FF425
:1042200080414FF0006008F02FFD4FF4407008F01F
:104230008DFC00F005FB00F01FFC2749274A284BA6
:104240001160284A284D136001222A70274A284C01
:10425000136000F0C7F804F09DFD04F0FFFC04F0CB
:1042600067F900F049F8207804F0FCFBE07804F0EE
:10427000EDF9207804F03CFBE07804F00FFA2B789D
:104280000BB105F0C9F805F04FFE00F07DF907F01D
:10429000A7FA01F0C5FC05F0D9F805F08BFE154B27
:1042A0004FF480625A6104F0D3FC03F0BBFA05F0CE
:1042B0008FFE05F005F900F0EBF800F0DDF80028BE
:1042C000F3D005F031FE01F0ABFC05F073FEECE736
:1042D0004C0C002000080140B99200085C0C002042
:1042E000C98B0008EC0B00206C0B00208C0B00200D
:1042F00008000020000C0140144B82B01B7813B35F
:10430000134B4FF400725A614FF480721A6100230C
:1043100001E0019B01330193019A4AF69B539A42B3
:10432000F7D90B4B4FF400721A614FF480725A6147
:10433000002301E0019B01330193019A4AF69B534C
:104340009A42DDD8F6E702B0704700BF980B002014
:10435000000C014010B1012805D101E0082200E065
:104360000422014B5A617047000C014010B1012832
:1043700005D101E0082200E00422014B1A617047D8
:10438000000C014038B50546002455FA04F2E3B2AA
:1043900012F0010F184602D0FFF7E8FF01E0FFF727
:1043A000D9FF0134082CF0D138BD00BF18B1012865
:1043B00006D0002008E0054BD868C0F3C00003E039
:1043C000024BD868C0F38000704700BF000C01406A
:1043D00008B1002003E0024B9868C0F3C03070477A
:1043E0000008014062B6704772B6704718B9024BB8
:1043F0004FF480625A617047000C014018B9024BBB
:104400004FF480621A617047000C014020B1054BE7
:104410004FF400521A6103E0024B4FF400525A610C
:10442000704700BF0010014020B1054B4FF480429F
:104430001A6103E0024B4FF480425A61704700BF9B
:104440000010014010B9024B09011960704700BF0C
:104450000400002008B9014B197070473002002099
:10446000044B58780138C0B201288CBF00200120CD
:10447000704700BF30020020044B5878012801D05B
:10448000002001E002225A70704700BF3002002075
:10449000082008B504F0F8FB592804D9064B5A78CF
:1044A0004AB9013206E0082004F0EEFB542802D895
:1044B000014B00225A7008BD3002002008B50328C5
:1044C00003D8DFE800F0040D1217002016E00020EA
:1044D00004F0DAFBB0F5006F94BF002001200DE07E
:1044E000074B9868C0F3801008E0054B9868C0F34C
:1044F000C01003E0024B9868C0F3401008BD00BF35
:10450000000C014038B500242546E0B2FFF7D6FF85
:1045100020B10123A34043EA0505EDB20134082C84
:10452000F3D1284638BD00BF10B5FF21002203207B
:1045300000F026FAFF210122032000F021FAFF21DA
:104540000022032000F01CFAFF2104460122032070
:1045500000F016FA034B40EA04205B6803EA90007F
:10456000181A10BD3002002008B5FFF7DDFF05283E
:1045700001D8012007E0FFF7D7FF40F2F933984256
:1045800094BF0020012008BD38B51E4C00202169D1
:104590004909FFF757FF2169002001F01F01FFF7CC
:1045A00059FFFE210022032000F0EAF940210122F8
:1045B000032000F0E5F900210A46032000F0E0F9AD
:1045C000002104460122032000F0DAF9082C0E4BEA
:1045D00005D14FF400629A6040F6FF7204E04FF498
:1045E00000729A6040F2FF325A60FFF79DFF064B5F
:1045F000040224464FEAE475C3E90645C3E90445CD
:10460000D86038BDF00B0020300200202DE9F843BF
:1046100004F01EFB624C2062FFF786FFE3686062D5
:1046200098423EDDA268C11A91420BDA5D4BA56A41
:104630001A684D195143D4E90667721847EBE173C4
:10464000A5622BE094F800C0564A1CF0040F12D06B
:1046500063681668C31A5E432CF0040C36464FEAB2
:10466000E677A36200220023C4E9066784F800C04D
:10467000C4E904234EE0656816685A190132121A1B
:104680007243D4E90667A36AED43ED18B6EB02085E
:1046900067EBE27942464B466918A162C4E90623FA
:1046A00038E037DAA1681A1A8A420EDA3D4DA16A5B
:1046B0002D68C91A6A43D4E90667B6EB020867EBAE
:1046C000E27942464B460918E7E72178354A11F06E
:1046D000040F0FD0126821F00401424312464FEA42
:1046E000E273C4E90623002200232170C4E90423F5
:1046F000A0620FE0616812680131CB1A1B185A439F
:10470000D4E90667B61847EBE277A26AC4E9066700
:104710009B18A362224B9D6ADA6A196BAA1A82EA75
:10472000E27CACEBE27C8C452CD942F210714A431E
:104730001E6A5C6B3C21341B92FBF4F251434FF434
:10474000807C91FBFCF181EAE172A2EBE172D9631A
:1047500040F6B8318A425E63DD629C6301DDC822A7
:1047600019E0B2F57A7F01DD642214E0322A01DD1E
:104770000A2210E00A2A01DD05220CE0012A0BDDE5
:10478000012208E0196A5A6B8A1AB2F5FA6F03D946
:104790000022DA6301321A63014BD860BDE8F88366
:1047A000300200200400002038B50D4618BB124C22
:1047B000FFF72CFFD4E90601002901DB626803E062
:1047C0006268404261EB4101120212464FEAE27315
:1047D0000CF086FCC4E9042328464FEAE071064C3D
:1047E0000B02020243EA1063D4E90401801841EB92
:1047F0000301C4E9060138BD3002002008B508B144
:1048000000200CE0FFF702FF054BD3E90401D3E9D8
:104810000623121A63EB0103100A40EA036008BD85
:104820003002002008B510B108F038FA01E008F0B5
:104830003DFA08BD08B5C90804F0E0FF08BD00BF97
:104840002DE9F745DFF830814848012108F0A8F844
:1048500001AE0420012108F01BFC03251024404672
:1048600042F212233146ADF804308DF806508DF82F
:10487000074008F005F802233D4F4046C8F81040B5
:104880004FF0040AC8F8143031464CF20043ADF83A
:1048900004308DF806508DF807A007F0F1FF0820CE
:1048A000012108F0F5FB41F61C7338463146ADF89E
:1048B00004308DF806508DF8074007F0E1FF4FF403
:1048C000F8533B610C23384631467B614FF0E003DF
:1048D00008F50068ADF804308DF807A08DF8065093
:1048E00007F0CEFF2046012108F0D2FB4EF2000374
:1048F00031464046ADF804308DF806508DF807403B
:1049000007F0BEFF4FF42043C8F81030A3F5C043B2
:104910000121C8F81430174808F042F800231A465D
:104920001946154C4FF4005565612046A4680133C3
:1049300014F4804F4FF400540461806808BF0131C3
:1049400010F4804F18BF01320A2BEAD10A2903D193
:104950000A2A01D1012200E00022084B03481A7004
:10496000012108F01DF8BDE8FE8500BF00023000FF
:10497000000C01400004300000080140980B0020AA
:1049800070B504460D461646032868D8DFE800F0E7
:1049900002070A0E334B4FF480525A6112E0102284
:1049A000314B0DE04FF400622E4B09E02F4A138883
:1049B00023F002031B041B0C13802D4B4FF4004209
:1049C0005A6110E02B48022108F0C4FC0028F9D0FD
:1049D0002946284808F062FC2648012108F0BAFC64
:1049E0000028F9D00FE02148022108F0B3FC00288C
:1049F000F9D029461D4808F051FC1C48012108F057
:104A0000A9FC0028F9D0EEB1032C28D8DFE804F087
:104A100002070A0F134B4FF480521A6118E010225C
:104A2000114B02E00F4B4FF400621A6112E0104A82
:104A30000E4B4FF4004111611A8892B242F002020B
:104A40001A8007E0032C0AD8DFE804F0020404040B
:104A5000084800E0054808F023FCC0B200E0002050
:104A600070BD00BF000C0140000801400030014053
:104A700000100140003800402DE9F04F01218BB0BB
:104A80004FF4804008F012FB494C012009AF014669
:104A900008F0FEFA03264FF0180B204639464AF27A
:104AA0000003DFF81491ADF824304FF0040A8DF8BC
:104AB00026608DF827B007F0E3FE204639464FF414
:104AC00080430DF11008ADF824308DF826608DF884
:104AD00027A007F0D5FE4FF48273002402224FF482
:104AE000007C012548464146ADF812304FF00803DE
:104AF000ADF81620ADF81AC00392CDF808C0ADF895
:104B00001C30ADF81040ADF81440ADF81850ADF8B9
:104B10001E40ADF8204008F04DFB4846294608F0FD
:104B200085FB29464FF4805008F0B2FA09F5504948
:104B30002846214607F034FF484639464FF0A00387
:104B4000ADF824308DF827B08DF8266007F098FE78
:104B5000484639464FF04003ADF824308DF82660C2
:104B60008DF827A007F08CFE039ADDF808C04FF4FB
:104B700082734146ADF812300E484FF01003ADF885
:104B80001620ADF81AC0ADF82040ADF81040ADF8D1
:104B90001440ADF81850ADF81C30ADF81E4008F0C8
:104BA00009FB0448294608F041FB0BB0BDE8F08F33
:104BB000000C01400030014000380040014B1878E3
:104BC000704700BF700200202DE9F84505461446E5
:104BD0000E4600294BD0002849D0814247D04FEAE9
:104BE00042185FFA88F848F006073946002006F0B8
:104BF000F3FA48F00C018246002006F0EDFA8046F8
:104C000028460CF02FF8054630460CF02BF80146EC
:104C100028460CF033F9064650460CF023F831468E
:104C20000CF02CF90CF03CFA054640460CF01AF852
:104C300031460CF023F90CF033FA0E49002814BF6A
:104C400080464FF001083046002D08BF01250CF0CA
:104C5000FFF918B14146204606F038FD39462A468C
:104C6000002006F06BFB044BE41801232371BDE820
:104C7000F88500BF0000A0417002002070B50D4D06
:104C8000044645192B799BB1C6B20B4B710141F01B
:104C9000060153F8202001F0E601002006F0E2FBB7
:104CA000064B304653F8241006F010FD00232B71FC
:104CB00070BD00BF70020020680B00206407002058
:104CC00073B5A54CA578002D40F00C836378A42B18
:104CD00000F044825AD8842B00F0C68026D8062BD8
:104CE00000F00D8110D8022B00F0BE8006D8002BFA
:104CF00000F0AA80012B40F0F382ABE0042B00F01F
:104D0000D78000F2E780CDE0802B00F09D8007D8AF
:104D10000C2B00F00F810D2B00F02C81072B70E085
:104D2000822B00F0398100F2C38093E0942B00F0D5
:104D3000018116D88A2B00F03F8108D8862B00F01D
:104D4000C980C0F0AF80872B40F0CA822EE18D2B46
:104D500000F05181932B00F00D818C2B40F0C0822C
:104D60003EE1A02B00F0E58109D8992B00F0668187
:104D70009A2B00F07881952B40F0B28241E1A22B72
:104D800000F0E181744B00F2E481D7E1B62B00F032
:104D90006A8228D8AC2B00F0318210D8A82B00F002
:104DA0000F8205D8A62B00F0F68100F20382E3E122
:104DB000AA2B00F00F82684B00F2128205E2B02BA2
:104DC00000F0388206D8AE2B00F02882624B00F249
:104DD0002C821EE2B22B00F03882C0F03082B52B5C
:104DE00040F07E8237E2C82B00F06A8115D8C12BD3
:104DF00000F0528108D8B82B00F04E82C0F04782F4
:104E0000C02B40F06D8288E0C32B00F05181C0F0D0
:104E10004781C72B40F0648271E0D42B00F065819C
:104E200009D8D12B00F03E82D22B00F04482CC2B4B
:104E300040F0568251E1D62B00F06381C0F05C81D6
:104E4000FE2B40F04D8264E1434B00205A6801463E
:104E5000DB7804E0404B00205A68DB78022143EA0B
:104E6000022206F06BFA40E23B4C0020E3786268D5
:104E7000082143EA022206F0F5FAE378A178626895
:104E8000490143EA0222002A41F00601B8BF52421A
:104E900001F0E601002006F0E5FA304AA378D318C5
:104EA0000122F7E12C4B00205A680A21DB7878E0D8
:104EB000294C0020E3786268062143EA022206F0CA
:104EC000D1FAE2786068A37842EA0020234A2449B4
:104ED0009A180FE0204C0020E378616843EA012132
:104EE00006F0F4FBE2786068A37842EA00201B4AEF
:104EF0001C499A1841F8230000231371F5E1164B61
:104F0000194AD978194B01201B781070184A022BC6
:104F1000517240F0EA810138B6E10F4B0122D97895
:104F2000124B1878104B1A70114B9972002840F0F0
:104F3000DC81A9E11421002001AA06F09FF9064AAC
:104F40009DF805305168D27852EA012114BF43F030
:104F5000020323F0020365E0E00600207002002057
:104F6000680B002064070020540C0020580C00201F
:104F7000F00B00201421002001AA06F07FF99B4AC3
:104F80009DF805305168D27852EA012114BF43F0F0
:104F9000010323F0010345E0944B00205A68DB78BD
:104FA000042143EA022206F05DFA9EE18F4B0020C5
:104FB0005A680E21DB78F4E701AE32461421284608
:104FC00006F05CF9A178E378490141F01401284624
:104FD00001F0F40132468DF8063006F0EBFA84E178
:104FE000824B834ADB780020C3F10801C9B2D37237
:104FF00004F01EFF79E17D4B00205A681A21DB780E
:10500000CFE71421002001AA06F038F9774A9DF86D
:1050100005305168D27852EA012114BF43F00403ED
:1050200023F004038DF80530704B0020997801AA15
:10503000490141F0140101F0F401CEE701AC224630
:105040001821002006F01AF9684A9DF80530917879
:10505000D278490102F00F0223F00F0341F018014A
:1050600042EA030311E001AC22461821002006F0B9
:1050700005F95E4A9DF805309178D278490103F030
:105080000F0341F0180143EA021301F0F801224630
:1050900000208DF80530A0E7E278554B1A7224E124
:1050A000524B5A68DB7843EA0222514B1A601CE1EA
:1050B0004E4B5A68DB7843EA02224D4B5A6014E1AA
:1050C0004C4B4D4A1B780120E1781070484A032B65
:1050D000D17740F00A812846D6E0444B5A68DB7805
:1050E00043EA0222424BDA81FFE0E378626843EA56
:1050F00002223F4B5A61F8E03C4BDA783C4B9A77FE
:10510000F3E03A4B5A68DB7843EA0222384B9A8341
:10511000EBE0364B364A5968DB7843EA0121052932
:1051200004D818461373FFF77FF9DEE000231373EA
:10513000DBE02846E17804F06DFED6E0D978002067
:1051400004F05EFED1E0294B0020D97804F038FD50
:10515000CBE0D978002004F027FDC6E0284604F013
:10516000E5F9E178A37818B9184604F005FDBCE02C
:10517000184604F0D1FCB8E0002004F0D7F91B4B2E
:1051800020B9D978987804F0EBFCAEE0D97898781B
:1051900004F0AAFCA9E0002004F0C8F9134B20B9E0
:1051A000D978987804F0D0FC9FE0D978987804F00A
:1051B000A7FC9AE00D4B0020D97804F0B9FC94E0EC
:1051C0002846E17804F0BEFB8FE0D978002004F097
:1051D000ADFB8AE0054B0020D97804F09BFB84E00E
:1051E000D978002004F08AFB7FE000BFE0060020B1
:1051F000F00B0020580C0020540C0020E1782846C9
:1052000004F070FBA178394BE27803EBC1035A71CB
:105210006BE0D978002004F009FB66E0344B0020F5
:1052200093F9031004F0F6FA5FE0D978002004F057
:105230008BFD5AE02846E17804F07AFD55E02C4BCE
:105240000020D97804F068FD4FE0294B0020D97880
:1052500004F056FD49E0264B5A68DB7843EA022207
:10526000244B9A6141E06068E278204B42EA0020DA
:10527000186010B9597904F035FB1D4B1E4A987817
:10528000125C012A31D1D978FFF7D4FA2DE0184BFE
:10529000DA78164B1A7128E0154B0020D97804F003
:1052A00077FC22E0124B00205968DB7843EA0121A9
:1052B000FFF77AFA19E00E4C0020E378626803F0F9
:1052C0001F0143EA02220B4B1A61FFF7C3F8E37890
:1052D0006168A07843EA01214911FFF7B3F804E0BF
:1052E000032200E00422054B1A707CBD7C0B0020D9
:1052F000E0060020F00B0020580C0020580700208A
:1053000013B5A84CA078002840F05B826378A52BE9
:1053100000F0EE81A44C79D8842B00F0FB8036D8C5
:10532000082B00F00A8113D8032B00F0F68005D873
:10533000012B00F0E98000F2ED80E2E0052B00F0A7
:10534000F380C0F0EF80062B00F0F180072BA4E083
:105350000D2B00F005810BD80A2B00F02F81C0F037
:1053600009810B2B00F00B810C2B40F02782EDE024
:10537000812B00F0C98003D8802B40F01F82C0E051
:10538000822B00F02881832B40F01882CAE0992BF1
:1053900000F043811ED88C2B00F02D810BD8862B7A
:1053A00000F0C280C0F0B980872B00F019818A2BF1
:1053B00040F0048217E1932B00F0D28003D88D2BAC
:1053C00040F0FC811CE1942B00F0C080952B40F054
:1053D000F58118E1A02B00F06C810BD89B2B00F01D
:1053E000CE80C0F023819C2B00F0E8809D2B40F004
:1053F000E581A2E0A22B00F06381C0F05D81A32BC8
:1054000000F06281A42B40F0D98163E1B82B00F059
:10541000C68135D8AE2B00F0A08115D8A92B00F09D
:105420008A8105D8A72B00F07E8100F280816CE193
:10543000AB2B00F08781C0F08181AC2B00F086811E
:10544000AD2B40F0BB8184E1B32B00F09A810BD8E7
:10545000B02B00F08A81C0F08481B12B00F08981EB
:10546000B22B40F0AB8188E1B52B00F09081C0F009
:105470008B81B62B00F08E81B72B40F09F818BE1A2
:10548000CE2B00F0EF8020D8C42B00F0E0800ED8A7
:10549000C12B00F0D48003D8C02B40F08F8149E0AD
:1054A000C22B00F0CF80C32B40F08881CCE0C72B0B
:1054B0003DD003D8C52B40F08181CAE0C82B00F055
:1054C000CB80CC2B40F07A81C9E0D42B00F0E48073
:1054D0000BD8D02B00F0DE80C0F0C680D12B00F0BE
:1054E0006181D22B40F06A8160E1D62B00F0DB8035
:1054F000C0F0D680D72B00F05E81FE2B40F05E819D
:10550000D4E00020014601E00020022105F064FE05
:10551000606059E1002008215FE000200A2105F0C9
:1055200095FEF5E7214B00E0214B1B68B6E0214BCF
:105530005B7AB3E01F4B9B7AB0E0002005F062FD80
:10554000184B9B785B0050FA03F310E00020142105
:1055500001AA05F093FE9DF80530C3F340039DE0DA
:105560000020142101AA05F089FE9DF8053003F002
:10557000010393E0104B9A68C2F3401218E17C21BA
:10558000002001AA05F07AFE064B02219A789DF8C8
:105590000630520011FA02F21A420CBF0023012316
:1055A0007CE000BFE006002058070020680B0020C8
:1055B00064070020F00B0020000C014001AA00202D
:1055C0007C2105F05BFE894B9DF806209B785B00F3
:1055D00052FA03F3CBE70020042105F037FE76E012
:1055E00000200E21F9E701AA0020142105F046FE53
:1055F0009DF80620DCE003F079FFC0F1080087E7A2
:1056000000201A21E9E701AA0020142105F036FE46
:105610009DF80520C2F38002CAE0182101AA05F016
:105620002DFE9DF8053003F00F0337E001AA00209E
:10563000182105F023FE9DF805201209B8E06C4BF7
:105640001A7AB5E06A4B05E0694B5A68B0E0694BDD
:105650006BE7694B1A68ABE0654BDA7FA8E0644BF7
:10566000DA89A5E0654B60E7654A664B1278002150
:1056700059600AB101225A60634B614A1B780021CC
:10568000117023B15F4B5A6842F002025A60002247
:105690005D4B98E05D4B78E0554B5B69636093E050
:1056A000534B9A7F84E0524B9A8B81E0504B1A7B8C
:1056B0007EE003F023FF2BE7002003F027FF06E046
:1056C000002003F02BFF02E0002003F02FFF4D4BE2
:1056D000586079E0002003F029FF4A4C434B18B989
:1056E000987803F033FF13E7987803F04FFF0FE744
:1056F00003F01CFFA378434C18B9184603F02EFFA3
:1057000006E7184603F052FF02E7002003F00EFF01
:105710003C4C364B18B9987803F028FFF8E6987897
:1057200003F03CFFF4E6002003F028FFCFE7002061
:1057300003F044FFCBE703F049FFE9E6002003F064
:105740004DFFC4E7002003F051FFC0E7304B5A790A
:105750002EE0002003F05AFFB9E703F05FFF40B2EC
:10576000D6E6002003F06CFFB1E7002003F070FFE5
:10577000ADE7002003F074FFA9E7002003F078FFF5
:10578000A5E703F085FFC3E6224B1A7810E0184B1B
:105790009A690DE01E4B5DE71D4B1A7908E003F096
:1057A000CDFEB5E60020FFF729F890E7104B1A6907
:1057B000144B5A6008E0FEF7B7FE88E70323237016
:1057C00002E0104B04221A70134B1B786BB10D4B87
:1057D00012495A68124B0A601AB91A6842F0080254
:1057E00002E01A6822F008021A601CBDE0060020E0
:1057F000F00B0020700B0020140C0020940B0020F4
:10580000E40B002058070020880B0020E80B002044
:105810007C0B0020780B002052070020400700205E
:10582000E806002010B51B4A5378142B2DD8917828
:1058300071B95468D078184A1849927E40EA042019
:1058400041F8230022B31BB303F5C270013013E00B
:10585000FF2918D163B94FF4C364114920460919CF
:105860000422043402F09CFCB4F5CD6FF5D10FE0B6
:1058700003F5C2700949013001EB83018000042265
:1058800002F08EFC04E0042200E00322054B1A70B3
:1058900010BD00BFE006002008000020EC0600203C
:1058A000D80000205807002038B51F4C6578142D0B
:1058B00036D8A07810F0800F18D010F0010F06D065
:1058C0000020022105F088FC184B43F82500184BF6
:1058D0009B7E43B3144B5B782BB303F5C270134923
:1058E000013001EB83018000042214E0B0B90221F1
:1058F00005F072FC0E4A0D4B927E43F8250092B1E2
:10590000617881B1A0780422091801F5C2700130D4
:1059100003EB8101800002F043FC04E0042200E07C
:105920000322044B1A7038BDE0060020EC0600206C
:10593000080000205807002038B56E4CA07808B148
:105940000422D3E063789A2B22D8992B80F09B8095
:10595000822B00F081800BD8062B6ED003D8042B4D
:1059600038D0052B0AE0072B6DD00C3B012B0CE047
:105970008C2B75D005D8832B2CD0862B40F0B5808E
:105980003FE08D2B7DD0933B022B00F2AE8060E098
:10599000C72B52D00ED8C12B7AD005D8B52B74D0D6
:1059A000C02B40F0A2804EE0C22B77D0C32B40F03A
:1059B0009C8076E0D42B7DD005D8C82B74D0CC2B1E
:1059C00040F0938073E0D62B7CD077D3FE2B40F051
:1059D0008C807DE0474D0020062105F055FEAC7817
:1059E0000020610141F0060101F0E60105F02EFC06
:1059F000414AAB78D318414A42F8240000221A7178
:105A000076E03C4D00200C2105F03EFEAC780020F5
:105A1000610141F00C0101F0EC0105F017FCAB78DD
:105A2000374A354942F8240018465B1852F82010CE
:105A300000221A7105F04AFE5AE0492002F098FB54
:105A4000304B587254E04A2002F092FB2D4B987272
:105A50004EE00020142100E0042105F015FE47E08F
:105A60004B200122284902F05FFBA378254A184603
:105A700002EB4313D97AC1F10801C9B204F0D8F995
:105A800036E01A21E9E71821E7E758201F4913E01B
:105A9000482002F06DFB1B4B187229E04020194989
:105AA0000AE044201A4907E05F201A4908E04E2026
:105AB000194909E019495420042206E018495E20DA
:105AC000012202E017495C20022202F02DFB0FE0C8
:105AD0004C200122144902F027FBA278094B03EB6A
:105AE0004213187BFEF7A0FC02E003220F4B1A7052
:105AF00038BD00BFE006002070020020680B0020C7
:105B000064070020F00B0020FB0B0020080C002095
:105B1000F40B00200F0C0020FE0B0020040C0020D2
:105B20000E0C00200C0C0020FC0B0020580700205D
:105B300010B51E4A5378142B34D89278AAB91C4A4F
:105B40001C4952F823201C4B4A601B78002B2CD098
:105B50001A491B4B0A601AB91A6842F0080202E09F
:105B60001A6822F008021A601FE0FF2A18D163B9F0
:105B70004FF4C3641349204609190422043402F087
:105B8000D3FAB4F5CD6FF5D10FE003F5C270084933
:105B9000013001EB83018000042202F0C5FA04E029
:105BA000042200E00322034B1A7010BDE00600201F
:105BB000EC06002058070020520700204007002074
:105BC000E8060020D800002037B5134C657815B1E1
:105BD000012D1DD112E0042240F2FB7001A902F058
:105BE000A3FAE378626843EA0222019B9A420B4BD4
:105BF00002D101225A600EE05D600CE0A3782A2BEE
:105C000006D1E11C40F2FB70042202F0C9FA02E066
:105C1000024B03221A703EBDE00600205807002008
:105C2000374938B500230B603649374A0B6037498E
:105C300093740B609360D36013745374344A4FF0C1
:105C4000FF3142F82310334A0024D45401332F2B60
:105C5000F4D10731204605F0BFFA2F4B0C21186014
:105C6000204605F0B9FA2D4D2D4BE97A1860C1F1A7
:105C700008012046C9B204F0DBF8287BFEF7D4FB0C
:105C8000284B0022E2500434B4F5806FF8D1264B43
:105C90009B7E5BB104F50674244920460919042251
:105CA000043402F041FAB4F5CD6FF5D11E4BDB7E22
:105CB0005BB94FF4A7641E49204609190422043435
:105CC00002F032FAB4F5C36FF5D1174B1B79012BF3
:105CD00003D0112B01D0212B01D1012200E00022A1
:105CE000094B83F8D020104B5B7D23B1FEF7B8FB46
:105CF00008B1012200E00022034B83F8D12038BD17
:105D0000400700206007002070020020E806002005
:105D100084020020680C0020680B0020F00B00209B
:105D2000640700206807002008000020D800002039
:105D30003002002008B50B4B5A7892B9997881B996
:105D40005A68DB7843EA022240F2D2439A4208D1F1
:105D500040F2FF7002F0A2FA02F064FB0120FEF7AD
:105D600061FD08BDE006002010B5994B9A78022A23
:105D700000F05181032A00F05781002A40F0E781AA
:105D80005A784D2A00F0BC8023D8452A70D00ED80E
:105D9000422A56D005D8402A45D0412A40F0D58124
:105DA00046E0432A53D0442A40F0CF8156E0482AA7
:105DB0007BD005D8462A61D0472A40F0C6816AE0E8
:105DC0004B2A00F0848000F29480492A40F0BD8183
:105DD00071E0542A00F0DA8011D8512A00F0B08026
:105DE00006D84F2A00F09280502A40F0AE81A0E001
:105DF000522A00F0B780532A40F0A781BCE0832AE2
:105E000000F0EC8006D8552A00F0CD80572A40F0EB
:105E10009C81D5E0852A00F0F180C0F0E780FF2A60
:105E200040F09381F3E06A4B40F2FF70D97805E0CF
:105E3000674B684ADB7800201946137002F02EFA8F
:105E400088E1DB78634A194601205370F6E7604B1E
:105E5000604ADB78042019461371EFE75C4B5D491B
:105E60005A68DB781C2043EA022341F81C3F0EE00D
:105E7000DB78584A194605205371DFE7544B5549E2
:105E80005A68DB780C2043EA022341F80C3F0422D5
:105E900002F086F95EE14E4B4E495A68DB780820E5
:105EA00043EA022341F8083FF1E7DB78494926201D
:105EB00001F8263F75E0464A464BD27812B1464972
:105EC00001224A60DA75434B1720D97DB6E7404B73
:105ED000404CDB7803201946E37002F0DFF9E078EC
:105EE00002F0B4FBE07802F0B1FBE07802F0D6FB00
:105EF00030E1374B374ADB780220194693709DE733
:105F0000DB78344A19461520537597E7304B314CEE
:105F1000DB7819201946637602F0C0F9607E10F034
:105F2000010002D00020012100E0014605F088FABE
:105F300010E1274B274ADB781620194693757DE739
:105F4000244A127D12F0010F05D0DB7813F0010F07
:105F500001D102F067FA1E4B1E4ADB781420194665
:105F600013756BE71A4B1B495A68DB78202043EA0C
:105F7000022341F8203F8AE7154B16495A68DB781F
:105F8000102043EA022341F8103F80E75A68DB788B
:105F900043EA0222012A00F2DA800E491A2001F8AF
:105FA0001A3F012274E70A4B5A68DB7843EA02225F
:105FB000012A00F2CC8007491B2001F81B3FF0E7C3
:105FC000034B0449DB78272001F8273FE9E700BFAE
:105FD000E006002008000020580700205A68DB78FF
:105FE00043EA02225C4BC3F8D420B3E05B4B5A680F
:105FF000DB7843EA02225A4B1A60ABE0574B5A68EF
:10600000DB7843EA0222544BC3F8D820A2E0534B7A
:10601000DA78544B9DE05868D9785A78524B41EA67
:10602000002143F8221095E05A78272A59D00ED83B
:10603000022A33D004D8CAB1012A40F0868021E078
:106040001B2A3ED01C2A44D0092A7ED132E02B2ABA
:106050005FD005D8292A50D0D978444A54D847E08F
:106060002D2A64D05CD32E2A6FD167E05A68DB7882
:1060700043EA02223D4B1A6002F0EAFD364BC3F8B8
:10608000DC0067E05A68DB7843EA0222374B5A604B
:1060900002F0DEFD304BC3F8E0005BE05A68DB78CD
:1060A00043EA0222314B9A6002F0D2FD2A4BC3F838
:1060B000E4004FE05A68DB7843EA02222B4BDA60B7
:1060C00048E05968DB78002043EA012105F0B2FA84
:1060D00040E05968DB78002043EA012105F07EFAB0
:1060E00038E05A68DB7843EA0222204B1A6131E03B
:1060F0005B6841EA032151612CE05A68DB7843EA8E
:1061000002221A4B9A6125E05B6841EA0321D161C2
:1061100020E05A68DB7843EA0222144B1A6219E045
:106120005A68DB7843EA0222104B5A6212E05A683E
:10613000DB7843EA02220D4B9A620BE05A68DB7867
:1061400043EA0222094BDA6204E0032200E004225F
:10615000074B1A7010BD00BF70020020E00600203F
:10616000540700205107002068070020180C002069
:106170005807002008B5824B9A78022A00F0B980AF
:10618000032A00F0BB80002A40F01E815B78502B70
:106190006ED022D8462B54D00ED8422B47D005D8EB
:1061A000402B3DD0412B40F00D813EE0442B43D0AD
:1061B000744B754A43D83DE04B2B4DD006D8482B45
:1061C00043D040D3492B40F0FD8042E04D2B49D0D5
:1061D00045D34F2B40F0F68047E0812B5FD010D89D
:1061E000542B4ED005D8522B47D0664B664A46D822
:1061F00041E0572B4BD0802B4DD0552B40F0E28007
:1062000042E0852B5DD004D8832B53D05D4B55D80D
:106210004DE0FE2B64D066D8F02B40F0D3805FE0D9
:1062200040F2FF7001F0A4FF9CE0574B59E0564B41
:106230005A78C4E01279C3E0534BDA69BFE052796F
:10624000BEE0514B85E0504B80E04F4B93F8262049
:10625000B5E04D4BDA7D48E04B4BDA78AFE04A4B86
:106260009A78ACE0484B5A7DA9E0474B5A7EA6E0AD
:10627000454B9A7DA3E0127DA2E0434B95E0126965
:106280009EE0414B9A7E9AE03F4BDA7E97E03E4B90
:1062900093F8272093E03D4B93F8D1208FE03B4BC0
:1062A00093F8D120042A14BF0022012287E0374A44
:1062B000926885E0354BD3F8D42080E0344A1268E8
:1062C0007EE0324A334BD2F8D8104B4303F54053AB
:1062D00039332C4923F000404860C2F8D83076E0CA
:1062E0002D4B1A786BE02D4B1A78003A18BF01221B
:1062F00065E05A782A4B53F8222060E05B78272B20
:1063000033D00DD8022B20D003D8C3B1012B59D1E3
:1063100018E01B2B1FD01C2B21D0092B52D117E0CA
:106320002B2B41D005D8292B24D0164B1D4A24D81D
:106330001EE02D2B3ED03AD32E2B43D13DE0194BFE
:106340001A683CE0174B5A6839E0164B9A6836E0F9
:10635000144BDA6833E0002004F0BAFF02E00020BA
:1063600004F0A2FF074B586031E00E4B1A6926E09B
:10637000526925E00B4B9A6921E0D26920E000BF09
:10638000E0060020580700200800002070020020CE
:10639000540700206D4EC6414C0C002051070020D0
:1063A00068070020180C0020124B1A6A07E0114BF6
:1063B0005A6A04E00F4B9A6A01E00E4BDA6A0E4B00
:1063C0005A6004E0032200E004220B4B1A700B4BCE
:1063D0001B786BB1084B0A495A680A4B0A601AB914
:1063E0001A6842F0080202E01A6822F008021A60F5
:1063F00008BD00BF180C00205807002052070020DD
:1064000040070020E806002010B5154CA07818BB06
:106410006378012B16D003D3022B124C19D114E050
:1064200004F098FAA17839B10F4A937FBBB102EB1F
:106430004112927F9A4212D10C4B01221A71013AF9
:106440000B4B0BE004F08EFA09E004F093FA606065
:1064500005E00323237002E0024B04221A7010BDF2
:10646000E006002058070020F00B002070020020FA
:10647000880B002037B5504B1A7CA2B94F494868A9
:10648000CA7842EA0022B2F1FF3F04BF4C4A1268C8
:106490000A214A43C3F8E82002F0DAFB464B012206
:1064A0001A74C3F8EC00454B5B78042B00F2828031
:1064B000DFE803F003353F4F130002F0C9FB3E4B0A
:1064C000D3F8EC10D3F8E820411A0029B8BF4942AC
:1064D00091426CD900221A746CE0384B364C987893
:1064E00004F048FA30B9374A2074136823F01003D7
:1064F00013605FE0D4F8E830002B57D002F0A8FB1F
:10650000D4F8EC20D4F8E830821A002AB8BF5242FE
:106510009A424BD92B4B00211A68217442E000208B
:1065200004F070FD254B244C9D786D0050FA05F564
:106530001CE000207C2101AA04F0A0FE1F4B0222D7
:106540009D789DF806306D0012FA05F51A4C1D4035
:106550000EE001AA00207C2104F090FE174A9DF86D
:1065600006309578144C6D0053FA05F515F00105C9
:1065700006D0144B00211A68217422F0100213E097
:10658000D4F8E83093B102F063FBD4F8EC20D4F8EF
:10659000E830821A002AB8BF52429A4206D9094B03
:1065A00025741A6842F010021A6003E0024B9A68E0
:1065B000013A9A603EBD00BF70020020E006002054
:1065C00040070020E806002008B5184B9A7812B161
:1065D000022A26D106E05868DB7843EA0020FDF75E
:1065E00015FF21E0587807280AD85A68DB7853EA63
:1065F000022202D1FDF7AEFE16E0FDF7B7FE13E072
:10660000FF280CD15868DB7843EA0020B0F1FF3F47
:106610000ABF074BC0B21878FDF7B4FE04E00322AE
:1066200000E00422034B1A7008BD00BFE006002002
:10663000400700205807002010B5224B9A78012A05
:1066400023D003D3022A204C28D122E058780828EE
:1066500002D8FDF733FF15E00A2801D100220AE035
:106660000B2802D1FDF780FF0CE00C2806D1174B58
:106670009A68C2F34012144B5A6011E0FF280FD100
:10668000FDF740FF104B58600AE0587802F0FCFA22
:10669000F8E75878FDF78AFE606001E00423237074
:1066A0000B4B1B786BB1084B0A495A680A4B0A60BE
:1066B0001AB91A6842F0080202E01A6822F00802C9
:1066C0001A6010BDE006002058070020000C0140B1
:1066D0005207002040070020E806002010B5204B9C
:1066E0005A78812A3AD19A78922A37D19A79A32A6C
:1066F00034D15A79B42A31D11A79C52A2ED1DB780E
:10670000D62B2BD1174B4FF480621A6102F044FE56
:1067100002F09EFA044602F09BFA001B0028B8BF64
:106720004042B0F57A7FF6DBFDF75EFE06F0DCF95D
:10673000002006F009FF00210B4805F08BFD0A48F8
:1067400005F0E8FC094805F0BBFC05F0D3FD4FF06F
:10675000804007F07DFC0020FEF764F810BD00BF0C
:10676000E0060020000C0140080002400024014027
:106770002DE9F3479D4A9E4DD0785168137840EA41
:1067800001204FF0640C222B85F800C06B7068600C
:1067900000F0838554D80F2B00F03E8324D8072BBC
:1067A00000F00A8210D8032B00F0F88006D8012BE5
:1067B00000F0A680022B40F0B187C8E0052B00F066
:1067C000F38100F2F58101E10B2B00F0E88205D89E
:1067D000092B00F0DC8200F2DE82D4E20D2B00F007
:1067E000138300F21583F3E2192B00F0BD8412D855
:1067F000152B00F0C98306D8132B00F01183142B3E
:1068000040F08C8774E3172B00F08E84794B00F2F4
:106810009E8400F082BC1E2B00F0D08409D81B2B74
:1068200000F0C484C0F0B0841C2B40F0778700F0E7
:10683000C0BC202B00F0C88400F2C98400F0C1BCA9
:10684000812B00F0D8852ED8412B00F0BA8515D8C1
:10685000252B00F0688507D8232B00F02A85242BF0
:1068600040F05C8700F031BD272B00F09385C0F02D
:106870006585402B40F0528700F0A0BD452B00F00D
:10688000AC8506D8432B00F0A28500F2A38500F06A
:106890009BBD472B00F0A785C0F0A285802B40F060
:1068A0003D8700F0A3BD882B00F0478612D8842BCB
:1068B00000F0EC8507D8822B00F0B585832B40F0E3
:1068C0002D8700F0B5BD862B00F0FA8500F25586C5
:1068D00000F0F1BD8C2B00F09A8606D88A2B00F0D0
:1068E0007D8600F28F8600F076BEF22B00F0E78600
:1068F000FF2B00F005878D2B40F0108700F08ABE3B
:106900009378FBB93B4B4FF0010C83F804C03A4B32
:1069100000241C70394B21461C702046022204F0D2
:1069200035FC2046062140F2FF7204F09BFD2F4B00
:1069300020465A68DB78082143EA022204F092FDDF
:1069400000F0EFBE2A4B04221A7000F0EABE274D79
:10695000AC78F4B9274B4FF0010C83F804C0264BF8
:1069600021461C70254B20461C70022204F00EFCB0
:106970002046062140F2FF7204F074FD6A68EB784D
:10698000204643EA02225242082104F06BFD00F047
:10699000C8BE174B04221A7000F0C3BE94788CB99D
:1069A000154B20461C70154B1C7003F0DBFF204676
:1069B0002146022204F0EAFB2046082104F066FD8D
:1069C00000F0AFBE04232B7000F0ABBE074B9A78EB
:1069D000002A40F0E4805B78032B00F2DB80DFE8E4
:1069E00013F00F0049009400BA0000BFE006002039
:1069F0005807002070020020E40B0020880B0020C4
:106A0000A64D0020FEF73AF9A54EAB780024686841
:106A1000EA78F454A34E590142EA0022F45401F0FA
:106A2000E001204604F08AFCA9782246204604F0C2
:106A3000ADFBA9789C4A02EB41139B7F002B00F031
:106A40007086002900F06D86927F9A4240F0698638
:106A50002046FEF713F96A68EB78204643EA0222E3
:106A6000214604F06BFC20462146224604F08EFBB2
:106A700000F057BE894D0020FEF700F9AB78884A38
:106A800000245901D454874A41F00201D45401F042
:106A9000E201204604F0A0FBEB786E68A97843EA97
:106AA00006268619490101F0E0013246204604F02D
:106AB00045FC2046A978224604F068FBA8787A4A6B
:106AC0007A4902EB40139B7F4E60002B00F0298631
:106AD000002800F02686927F9A4240F02286FEF738
:106AE000CDF80221204604F077FB6A68EB78214656
:106AF00043EA02228218204604F020FC2046214668
:106B0000224604F043FB00F00CBE644CE37862685C
:106B100043EA0223142B19DC654A002052F8236053
:106B2000FEF7ACF8A37832465D4E0025F5545D4E75
:106B30005901284601F0E001F55404F0FFFB284616
:106B4000A1782A4604F022FB00F0EBBD574B04224B
:106B50001A7000F0E6BD514C0020E3786268002511
:106B600043EA0222524B53F82260FEF787F8A378DB
:106B700032464B4E5901F5544A4E284601F0E00189
:106B8000F55404F0DBFB2846A1782A4604F0FEFA0F
:106B900000F0C7BD454B03221A7000F0C2BD434B45
:106BA00004221A7000F0BDBDFEF78AF800F0B9BDEE
:106BB000FEF7A6FB00F0B5BD907818B104232B704A
:106BC00000F0AFBD53789A2B21D8992B80F08480A8
:106BD000822B6FD00BD8062B4BD003D8042B3CD084
:106BE000052B0AE0072B4BD00C3B012B0CE08C2B28
:106BF00065D005D8832B30D0862B40F0BF8032E0A3
:106C00008D2B63D0933B022B00F2B8803FE0C82B62
:106C100000F083800FD8C12B6AD005D8B52B60D087
:106C2000C02B40F0AB802BE0C32B6FD067D3C72BBA
:106C300040F0A4801DE0D42B00F0848005D8CC2B3C
:106C400072D0D22B40F09A8075E0D62B00F088806D
:106C50007FD3FE2B40F0928089E00020062104F0D3
:106C60004BFB00F05EBD00200C2104F045FB00F062
:106C700058BD0D4B4920597A01F010FB00F051BD71
:106C8000094B4A20997A01F009FB00F04ABD002027
:106C9000142104F031FB00F044BD00BFE0060020E9
:106CA000880B0020E40B0020F00B00205807002088
:106CB000EC060020042104F01FFB00F032BD4B2045
:106CC000A149012201F06CFA00F02BBD00201A212D
:106CD00004F012FB00F025BD182104F00DFB00F0BC
:106CE00020BD58209949042201F05AFA00F019BD3C
:106CF000974B4820197A01F0D1FA00F012BD4020DC
:106D00009349042201F04CFA00F00BBD4420914954
:106D1000042201F045FA00F004BD5F208E490122F3
:106D200001F03EFA00F0FDBC4E208C49022201F039
:106D300037FA00F0F6BC50208949042201F030FAFD
:106D400000F0EFBC54208749042201F029FA00F03A
:106D5000E8BC5E208449012201F022FA00F0E1BC87
:106D60005C208249022201F01BFA00F0DABC4C20C0
:106D70007F49012201F014FA00F0D3BC7D4B0322BD
:106D80001A7000F0CEBCFEF7D7FD00F0CABCFEF7CB
:106D9000EBFF00F0C6BCFFF7EDF900F0C2BC937842
:106DA000022B11D15378372B0AD8734903F5A770FA
:106DB00001EB83018000042201F0F2F900F0B1BC84
:106DC00003232B7000F0ADBC04232B7000F0A9BC92
:106DD0006A4B9A78022A12D15B78372B0AD8664917
:106DE00003F5A77001EB83018000023201F09CF9EA
:106DF00000F097BC5F4B03221A7000F092BC5D4B11
:106E000004221A7000F08DBCFFF7FEFA00F089BC76
:106E1000FFF7DAFB00F085BCFFF70EFC00F081BC49
:106E20005278574B092A53D8DFE802F0050D151D9B
:106E300026313941494C514A19685068D27842EAA2
:106E40000022521843E04D4A19685068D27842EA4D
:106E500000228A1A3BE0494A19685068D27842EA0F
:106E600000224A4333E0454A19685068D27842EA22
:106E7000002291FBF2F22AE0404819684468C27887
:106E800042EA042291FBF2F002FB10121FE03B4A9F
:106E900019685068D27842EA00220A4017E0374A5F
:106EA00019685068D27842EA00220A430FE0334A58
:106EB00019685068D27842EA00224A4007E01A680E
:106EC000D24304E02D4A5168D27842EA01221A6086
:106ED0002B4A2C4B12682AB91A6842F008021A6031
:106EE00000F01FBC1A6822F008021A6000F019BCFA
:106EF000224B234A5968DB78126843EA01239A42FD
:106F000006DD204B1A6842F0040222F003020CE076
:106F10001C4B05D11A6822F0060242F0010204E07F
:106F20001A6822F0070242F002021A60144A154B56
:106F3000126822B91A6842F008021A60F1E31A686E
:106F400022F008021A60ECE3FB0B0020080C002082
:106F5000F00B0020F40B00200F0C0020FE0B002093
:106F6000000C0020040C00200E0C00200C0C002053
:106F7000FC0B00205807002068070020E0060020D6
:106F800040070020E806002053780C2B00F2C9834C
:106F9000DFE813F00D001B00290037004500530007
:106FA00061006F007D008B009900A700B500944B35
:106FB0001B6813F0080F00F0B483924B5A68DB781B
:106FC00043EA0222904B9A60ABE38D4B1B6813F0AF
:106FD000080F40F0A6838B4B5A68DB7843EA022205
:106FE000894B9A609DE3864B1B6813F0010F00F0FC
:106FF0009883844B5A68DB7843EA0222824B9A607A
:107000008FE37F4B1B6813F0010F40F08A837D4BA9
:107010005A68DB7843EA02227B4B9A6081E3784B23
:107020001B6813F0040F00F07C83764B5A68DB7802
:1070300043EA0222744B9A6073E3714B1B6813F0AE
:10704000050F00F06E836F4B5A68DB7843EA02222B
:107050006D4B9A6065E36A4B1B6813F0020F00F0FA
:107060006083684B5A68DB7843EA0222664B9A6079
:1070700057E3634B1B6813F0030F00F05283614B1F
:107080005A68DB7843EA02225F4B9A6049E35C4B23
:107090001B6813F0100F00F044835A4B5A68DB78DA
:1070A00043EA0222584B9A603BE3554B1B6813F0AE
:1070B000200F00F03683534B5A68DB7843EA0222F4
:1070C000514B9A602DE34E4B1B6813F0400F00F0BC
:1070D00028834C4B5A68DB7843EA02224A4B9A6079
:1070E0001FE3474B1B6813F0800F00F01A83454BDA
:1070F0005A68DB7843EA0222434B9A6011E3404B23
:107100001B6813F4807F00F00C833E4B5A68DB78D9
:1071100043EA02223C4B9A6003E33A4A5168D27830
:1071200042EA01229A60FCE2374BDA68072A00F251
:10713000F88234499C684868C97841EA0020511CAB
:1071400003EB8202C2F8F0409860D960E9E2DA68A5
:107150002D4B002A00F0E582013A03EB8201D1F8C1
:10716000F010DA609960DCE253782E2B03D8274ABE
:107170000121D154D5E2FF2B03D1234B01225A74B4
:10718000CFE203232B70CCE21E4B5B782E2B03D86F
:107190001E4A0021D154C4E2FF2B03D11A4B002216
:1071A0005A74BEE21A4B03221A70BAE2FFF762F970
:1071B000B7E2154B002283F8D120B2E2FEF732FB92
:1071C000AFE2FEF7B5FCACE2FEF76EFBA9E20D4ABA
:1071D000104B52780A2A52D8DFE802F0060B20251D
:1071E0002B33393F45494C000B491A6809688A1806
:1071F00003E0094A196812688A1A1A603FE000BF62
:10720000E8060020E006002070020020680C002044
:10721000580700204007002060070020934A1968A3
:1072200012684A43E9E7914A1968126891FBF2F241
:10723000E3E78E4A1968126891FBF2F002FB101224
:10724000DBE78A491A68096801EA0202D5E787493B
:107250001A68096841EA0202CFE784491A68096896
:1072600081EA0202C9E7814B1A68D243C5E71A686E
:107270007E4BC2E77D4A18681168106019607C4A2D
:107280007C4B126822B91A6842F008021A6048E280
:107290001A6822F008021A6043E2754B01F07F4140
:1072A00018681B7841EA10215160D370FDF708FD82
:1072B00037E26F4B01F07F4118681B7841EA1021DB
:1072C0005160D370FEF750FD2BE26B4B5B78052BC2
:1072D00000F22782DFE803F003090F151B21654B3D
:1072E0001A6802F00F021A601BE2624B1A6822F061
:1072F00010021A6015E25F4B1A6822F020021A6031
:107300000FE25C4B1A6822F040021A6009E2594B06
:107310001A6822F080021A6003E2564B1A6822F4BF
:1073200080721A60FDE153782E2B04D8534A02EB89
:1073300083035861F5E103232B70F2E14F4BDFF833
:1073400030C1D3F810914E4993F82C21D3F814A1F1
:10735000CCF80090DFF814C1D3F81871D3F81C8171
:10736000D3F82061D3F82451D3F82841CCF800A0F9
:10737000885CDFF800C19F60CCF800801E74C3F801
:10738000EC50C3F8E84008B101238B543B4B00227A
:107390009A74C6E193786BB9374B5B78142B05D898
:1073A000334A1168374A42F82310BAE1364B0322B8
:1073B0001A70B6E1344B04221A70B2E102F048F8B8
:1073C000AFE102F047F8ACE102F046F8A9E102F0C3
:1073D00045F8A6E102F044F8A3E102F043F8A0E189
:1073E00002F042F89DE102F041F89AE1234B0022BD
:1073F00083F8D12095E1537813B1012B10D104E02B
:107400001E4B012283F8D1208BE1B0F5006F04D22E
:107410001A4A906082F8D13083E104232B7080E116
:1074200003232B707DE1154B022283F8D12078E1F4
:10743000124B002199745974104A4FF0FF3402F135
:10744000140040F821400E480023435401312F29F5
:10745000F2D1084913740B60054982F8D1300B60F2
:10746000024993600B60D3605BE100BF60070020BE
:1074700040070020E8060020E006002070020020FF
:10748000680C0020EC060020580700208D4B1B7D67
:1074900013F0020F0CD1B0F5006F06D28A4B042214
:1074A000C3F8300183F8D1203BE104232B7038E18D
:1074B00008232B7035E1844B002283F8D12030E182
:1074C000804B01219A78814BB0F5006F1970804B89
:1074D0001A7028D27B4B1C7D0C4024D1694600F0E9
:1074E000E5FF7B4B9DF800709DF801609DF8025010
:1074F0009DF806C09DF805009DF804109DF8032036
:107500001C725F709E70DD7083F804C058719971B1
:10751000DA7101236E4A985C117A01334118082B05
:107520001172F7D1FDE00123694A0021995401331A
:10753000082BF9D113781372F3E053788BB9614AB1
:1075400001209178634A1468604A1070604A117093
:107550000133E21812F8011C5D4A082B9954F7D147
:10756000DFE0012B40F0DD8015222A710422EA7150
:107570006FF07602AA716B71D3E0574B5B78032BE7
:1075800000F2CF80DFE803F002101D224E4A534B79
:10759000D2F8301192F8D1C0107C0A0A197183F820
:1075A00007C098715A71BCE0474A4C4B916892F8F9
:1075B000D1C0107C0A0A197183F807C098715A71FA
:1075C000AFE0474B1A68454B5A60AAE0454B1A6832
:1075D000424B5A60A5E0FEF7ADFBA2E05278424B69
:1075E00002B101221A703C4B404AD878364B1070D9
:1075F00093F834113E4A002311703E4A13703E4AFC
:1076000013708EE0304B012283F8352189E0FEF7BC
:10761000DBFA86E0304B5B78032B4CD8DFE803F0D5
:107620000C023C472C4B28495A68DB78D1F83811BA
:1076300043EA022C00232BE0234BD3F83821092AFC
:107640000CD82549501C4C68C97803EB820241EAEA
:107650000421C2F83C11C3F8380162E01F4B092233
:107660001A705EE052F82340581C64450FD102EBBB
:107670008002013904E052F8040C013342F8080C8E
:1076800004328B42F7D3104BC3F8381149E003465C
:107690008B421A4AE6D344E00B4A0023C2F8383141
:1076A000164A0021D1500433282BF9D139E00B4B75
:1076B0000A225A6035E0094B03221A7031E0FFF7C5
:1076C0000DF82EE008000020700200204407002082
:1076D0004807002000000020E00600205807002096
:1076E0004007002060070020740B0020900B002052
:1076F000560C0020970C0020890B0020AC030020C2
:10770000094B5A68DB7843EA022240F2D2439A429C
:1077100007D1064B012283F8642102E0044B0222C8
:107720001A70BDE8FC8700BFE00600207002002050
:107730005807002073B5204B024640781F4D187043
:10774000907800265870D078EC46987010790C46E6
:1077500098715079587192F806E095E8030083F823
:1077600004E0D2798CE80300DA70154B1E70FEF746
:10777000FFFF144B1B7873B9637023702B78A370D1
:107780006B78E370EB792371AB7963716B79A371DB
:107790002B79E37108E0012B06D10B4B9B195B7829
:1077A000A3550136082EF8D1044B6A4692E803002F
:1077B00083E803007CBD00BFE006002058070020DE
:1077C000520700204407002048070020F7B5114D5C
:1077D000114C6F684FF0000C07F07F4747EA132702
:1077E0006F600E4F6E4687F800C028706970AA70EF
:1077F00094E80300EB7086E80300FEF7B9FF96E813
:1078000003006368227884E80300054918460A707B
:10781000FEBD00BFE00600205807002052070020F0
:10782000700200202DE9F04F7E4B93B01B781BB9FE
:107830007D4B93F865316BB17C4B1B78062B09D0DF
:107840000A2B07D00F2B05D01F2B03D0764B00221D
:1078500083F83421744A92F83431032B25D192F8FD
:10786000D040002C40F0D980714B1B7893B9714DFA
:10787000714CA8786E78227863788619B618E27908
:10788000F618A379B6186279F6182379B618F6189F
:10789000F6B219E0012B40F0FE80684BE05C013449
:1078A00000F040FF092CF8D1F5E0042B27D1614D01
:1078B000614CAB786E7818469E1901360023012280
:1078C00022706360F6B2637000F02CFF687800F0FD
:1078D00029FF207800F026FF607800F023FFE07990
:1078E00000F020FFA07900F01DFF607900F01AFF82
:1078F000207900F017FF304600F014FFCBE0052B95
:1079000025D192F8D040002C40F08780484B1B785E
:1079100093B9484D484CA8786E78227863788619D8
:10792000B618E279F618A379B6186279F6182379B1
:10793000B618F618F6B219E0012B40F0AC803F4BB8
:10794000E05C013400F0D2FE092CF8D1A3E0062B54
:1079500027D1384D384CAB786E7818469E190136D1
:107960000023012222706360F6B2637000F0BEFE55
:10797000687800F0BBFE207800F0B8FE607800F078
:10798000B5FEE07900F0B2FEA07900F0AFFE6079BC
:1079900000F0ACFE207900F0A9FE304600F0A6FE13
:1079A00079E0072B4ED192F8D030002B35D1204A08
:1079B000127822BB1F4A204B557896781C7893F892
:1079C00001C0AF19D879E719997967445A79C7196D
:1079D0001B79CF19D719DF198DF838708DF8306001
:1079E0008DF831508DF832408DF833C08DF8340069
:1079F0008DF835108DF836208DF8373008E0012AE3
:107A000006D10E4A995C0CAAD1540133092BF8D146
:107A10000B4B1B78002B3ED039E0074803F070FF7A
:107A200039E000BF5107002070020020E00600206E
:107A300044070020080000205807002048070020C5
:107A40006C0B0020082B26D1954B00225978987892
:107A5000944B45181C78944B4FF0010C01355A603B
:107A60008DF832C08DF8332016468DF834208DF80D
:107A700035208DF836208DF837208DF838505A7023
:107A800083F800C08DF830008DF831101CB10CA8BF
:107A9000092101F04FFB854B1B78002B56D0844BFE
:107AA0001B78032B02D0072B4BD123E07C4C814D5C
:107AB000A07866782B7886190A36F61800F032FE20
:107AC000607800F02FFE802000F02CFE8A2000F06D
:107AD00029FE002000F026FE002000F023FE0020FA
:107AE00000F020FEF6B2287800F01CFE304600F0D0
:107AF00019FE26E06A4B6FF07F05597898786D4B38
:107B000000EB010C1A78674B0CF10A0C1C789444BA
:107B100000238DF826500A358DF827508DF82A302D
:107B20008DF82CC08DF824008DF825108DF82830A4
:107B30008DF829308DF82B201CB109A8092101F0FE
:107B4000F9FA5A4A002313705A4A13705A4B5B4889
:107B500093F864110022027083F8652183F83421C0
:107B600011B10120FCF75EFE534B93F8352152B161
:107B700093F8D0200021D2F1010238BF002283F80F
:107B8000351183F8D0204C4C94F8D050002D72D190
:107B90000DF1470000F044FD00286CD000F05CFDC2
:107BA00008B184F86651444B9DF8470093F866117C
:107BB0004A1CD2B2C918092A81F8680183F86621E3
:107BC00040F07681364993F8682148784FF0000CF0
:107BD000904283F866C107D091F82730002B00F05F
:107BE00067819A4240F064812D4B93F8273093428D
:107BF00003D1314B012283F8652100231A462E4C14
:107C000004F5B471C95C01335218082BD2B2F6D115
:107C100094F8703193422CD1294B94F86D1194F85B
:107C20006E2194F86F5194F8696194F86AE194F8C0
:107C30006BC194F86C01DD7059711A711E7083F874
:107C400001E083F802C0987101F002F81D4D94F82C
:107C5000D1302860591E1C480022C9B2027003208E
:107C6000012984F8340184F8662140F2EE80052B66
:107C7000A0E00423EDE0104C94F8D03033B310486A
:107C800003F084FE10B300F0E3FF0E4994F8D13006
:107C900008600D495A1E00200870D2B20321CEE0C0
:107CA000080000206C0B002058070020970C0020D3
:107CB000560C0020890B0020700200204407002091
:107CC000E0060020500C0020550C00206F4C94F86A
:107CD000D050002D73D10DF1470000F0C7FC0028F3
:107CE0006DD000F0E1FC08B184F86651674B9DF857
:107CF000470093F866114A1CD2B2C918092A81F8C4
:107D0000680183F8662140F0D380614993F86821C7
:107D100048784FF0000C904283F866C107D091F884
:107D20002730002B00F0C4809A4240F0C180584BAD
:107D300093F82730934203D1544B012283F86521F5
:107D400000231A46514C04F5B471C95C0133521832
:107D5000082BD2B2F6D194F8703193422DD14D4B0D
:107D600094F86D1194F86E2194F86F5194F869614C
:107D700094F86AE194F86BC194F86C01DD70597164
:107D80001A711E7083F801E083F802C0987100F048
:107D90005FFF414D94F8D1302860591E3F480022C2
:107DA000C9B202700520012984F8340184F86621E3
:107DB0004BD9834249D0013248E0062349E0334B96
:107DC00093F8D040002C47D1354B1B78002B43D083
:107DD0000FA801F099F900283ED0234622460FA9AA
:107DE000C95C01335218082BD2B2F8D19DF8441067
:107DF000264C91422DD1274B9DF841109DF84220F1
:107E00009DF83D609DF83EE09DF83FC09DF8400024
:107E10009DF8435059711A711E70DD7083F801E0AE
:107E200083F802C0987100F013FF1B4994F8D13019
:107E300008601A495A1E00200870D2B20721012A90
:107E400084F8341101D9052B1ED10022154B1A706C
:107E50002EE084F834312BE00C4C94F8D130013B07
:107E6000DBB2012B24D8A368B3F5006F1CD2FCF75A
:107E7000F7FAC8B1A368074918460133A36000F0B8
:107E800015FB092384F834310122DFE7700200205A
:107E900008000020E0060020500C0020550C0020B7
:107EA0006C0B002052070020964B002283F8D12053
:107EB000944C94F8D130042B05D1934E327812F0C3
:107EC000800F00F0EF808F4B93F834313BB1042BDF
:107ED00005D0082B03D0062B01D0FEF749FC894CB6
:107EE00094F83431092B40F0B28000F0B1FED4F8A0
:107EF000DC30864AC31A002B1268B8BF5B4293423B
:107F00000AD9834B1A78012A01D101321A7000F084
:107F10009FFE7C4BC3F8DC0000F09AFE794BD3F84F
:107F2000E0207A4B821A002A5B68B8BF52429A421C
:107F30000AD9774B5A78012A01D101325A7000F0E0
:107F400087FE704BC3F8E00000F082FE6D4BD3F863
:107F5000E4206E4B821A002A9B68B8BF52429A42B4
:107F60000AD96B4B9A78012A01D101329A7000F03C
:107F70006FFE644BC3F8E400624A537C002B66D06A
:107F8000937C002B63D19C46624B92F82C011B68BA
:107F900002900793604BD2F8E8001B6803900693A9
:107FA0005E4BD2F810811B68D2F814710593D2F899
:107FB000EC30D2F818410493D2F81C619368107C1D
:107FC000D2F82051D2F824B1D2F828210192624689
:107FD000DFF83C91194619F802A0BAF1020F18D146
:107FE0004F4951F82210B1F1FF3F0ED00546D0B2F3
:107FF00002900398DDF810B00190059E069FDDF811
:108000001C804FF0010C002004E0002109F8021050
:108010001946234601322F2A02D01C460B46D7E7C9
:10802000384AC2F818311074019B029882F812C0C5
:10803000C2F81081C2F814719160C2F81C61C2F8D4
:108040002051C2F824B1C2F8283182F82C012D4BFE
:1080500093F83421092A06D193F8D120022A02D1BB
:10806000033283F8D120274BD3F83811002946D0AA
:1080700093F83421092A42D193F8D120012A3ED124
:108080009868002308E054F823400133A04203D14C
:10809000052382F8D13032E01A4A8B4202F59E74F1
:1080A000F1D32CE094F834314BB3042B27D0082BB8
:1080B00025D0062B23D0F3787168D4F83001194D00
:1080C00043EA0123B0F5006F6A706B6012D231464B
:1080D00000F01CF93146D4F8300100F03FF930B11E
:1080E000D4F830310133C4F83031652300E0072380
:1080F0002B7004E007232B70002384F8D13013B0D9
:10810000BDE8F08F70020020E0060020180C00206F
:10811000680C00204007002060070020E8060020CF
:10812000840200205807002070B5044600200E4647
:10813000154603210246FCF723FC0020C4F3072167
:108140000246FCF71DFC0020E1B20246FCF718FCD9
:10815000002407E0944214BF00220122FCF710FC27
:108160003055013400206A1EAC420146F2D370BD86
:1081700010B50446002003210246FCF701FC002054
:10818000C4F307210246FCF7FBFB0020E1B20246E4
:10819000FCF7F6FB002001460122FCF7F1FB10BDC5
:1081A0002DE9F04104460F46164600200621012223
:1081B000FCF7E6FB002005210246FCF7E1FB00206E
:1081C00001220146FCF7DCFB10F0020FF2D0002088
:1081D00002210246FCF7D4FB0020C4F3072102462B
:1081E000FCF7CEFB0020E1B20246FCF7C9FB0025FC
:1081F00043E0013414F03F08795D01D1012204E02D
:10820000721E954214BF002201220020FCF7B8FB29
:10821000B8F1000F30D1731E9D422DD200200521F0
:108220000246FCF7ADFB002001220146FCF7A8FB4B
:1082300010F00100F2D106210122FCF7A1FB002081
:1082400005210246FCF79CFB002001220146FCF7B9
:1082500097FB10F0020FF2D0002002210246FCF73B
:108260008FFB0020C4F307210246FCF789FB0020A6
:10827000E1B20246FCF784FB0135B542B9D30020D8
:1082800005210246FCF77CFB002001220146FCF799
:1082900077FB10F0010FF2D1BDE8F08138B5012273
:1082A00004460D4600200621FCF76AFB002005214C
:1082B0000246FCF765FB002001220146FCF760FB4B
:1082C00010F0020FF2D0002002210246FCF758FB0A
:1082D0000020C4F307210246FCF752FB0020E1B264
:1082E0000246FCF74DFB294600200122FCF748FB23
:1082F000002005210246FCF743FB00200122014635
:10830000FCF73EFB10F0010FF2D138BD38B5072560
:10831000454305F500650C46284609780135FFF709
:10832000BDFF284661780135FFF7B8FF2846A178E0
:108330000135FFF7B3FF2846E1780135FFF7AEFFBF
:10834000284621790135FFF7A9FF28466179FFF713
:10835000A5FF681CA179FFF7A1FF38BD2DE9F34700
:108360000725454300200C4602460321FCF708FB85
:1083700005F500650020C5F307210246FCF700FB68
:108380000020E9B20246FCF7FBFA00200146024653
:10839000FCF7F6FA8246002001460246FCF7F0FAA6
:1083A0008046002001460246FCF7EAFA0746002014
:1083B00001460246FCF7E4FA8146002001460246E7
:1083C000FCF7DEFA0646002001460246FCF7D8FA22
:1083D0000546002001220146FCF7D2FA23785345D6
:1083E0001DD1637843451AD1A378BB4217D1E378F6
:1083F00021798DF804608DF805508DF806006279BA
:1084000043EA012343EA0243A079019A43EA006068
:1084100049EA0229814514BF0020012000E0002024
:10842000BDE8FC8738B54FF4006400200621012226
:10843000FCF7A6FA002005210246FCF7A1FA00206D
:1084400001220146FCF79CFA10F0020FF2D0002046
:1084500002210246FCF794FA0020C4F307210246E9
:10846000FCF78EFA0020E1B20246FCF789FA0025FB
:1084700000203F2D14BF0022012201460135FCF7E8
:108480007FFA402DF4D1002005210246FCF778FA4E
:10849000002001220146FCF773FA10F0010FF2D11F
:1084A0004034B4F5804FC0D138BD00BF38B5072582
:1084B000454300200C4602460321FCF761FA05F50E
:1084C00000650020C5F307210246FCF759FA002099
:1084D000E9B20246FCF754FA002001460246FCF7D6
:1084E0004FFA2070002001460246FCF749FA6070FE
:1084F000002001460246FCF743FAA0700020014626
:108500000246FCF73DFAE070002001460246FCF707
:1085100037FA2071002001460246FCF731FA6071FB
:10852000002001460122FCF72BFAA07138BD00BFE4
:1085300037B5002005210246FCF722FA002001226F
:108540000146FCF71DFA10F07104F2D100F080FB37
:10855000054605E0FFF70CFE422814BF0024012465
:1085600000F076FB431B002BB8BF5B42B3F5FA6FFC
:1085700040F2FF7002DA002CECD000E01CB1234B7B
:108580001B78002B36D040F2FF700021FFF786FEEB
:10859000FFF748FF00201E494022FFF701FE4FF47D
:1085A00080701C49B422FFF7FBFD40201A492022AD
:1085B000FFF7F6FD002301934FF4C36401AD20469D
:1085C000042204342946FFF7EBFDB4F5FF6FF5D123
:1085D00000230193A4F53074204604220434294674
:1085E000FFF7DEFDB4F5C36FF6D140F2FF70422114
:1085F000FFF754FE002040220549FFF795FD40207B
:1086000006492022FFF790FD3EBD00BF980B0020D9
:1086100008000020D017010800180108F00B002006
:10862000094B19685A68914201D100200BE01A6881
:10863000D118097A013201701A601A68202A01D112
:1086400000221A6001207047E4030020014B986269
:10865000704700BFE4030020034B1A78104612B1A4
:1086600000221A7001207047A80C00200A4BD96A1A
:108670001A6B914201D100200CE0DA6AD11891F80E
:10868000341001320170DA62DA6A202A01D1002244
:10869000DA620120704700BFE4030020014B5865F7
:1086A000704700BFE4030020034B1A78104612B154
:1086B00000221A7001207047A90C002008B5FBF7B2
:1086C00093FE034B0022DA621A63FBF78BFE08BDB0
:1086D000E403002008B5FBF787FE034B00221A6075
:1086E0005A60FBF77FFE08BDE403002038B50B4B52
:1086F00084469C6DDA6D0134202C08BF002494421E
:108700000AD09D6D0648ED1885F860C040F22771CB
:1087100001229C6505F034FD38BD00BFE403002054
:108720000044004038B50D4B8446D3F88040D3F860
:1087300084200134202C08BF002494420CD0D3F8AC
:1087400080500748ED1885F888C040F22771012253
:10875000C3F8804005F014FD38BD00BFE4030020DD
:108760000038014038B50546002401E0FFF7DAFF84
:108770002B5D01341846002BF8D138BD2B4910B5BC
:108780000B8813F0200F1DD0294BDB6813F0020F6C
:1087900001D08B8816E0274B1A6BD86A0132202A49
:1087A00008BF0022824206D01C6B8888E118C0B244
:1087B00081F834001A63204B0A221A601D4B5A6D4F
:1087C0001E4B1A601948038813F0800F1BD01B4BF7
:1087D0001A68C2B9174B9C6DD96D8C420FD01449E1
:1087E00002240C61D96DCC1894F860C00131A0F856
:1087F00004C0D965D96D202905D1DA6503E040F2BE
:10880000277105F0BDFC0948038813F0400F0BD019
:1088100040F2266105F0ACFD064BDA6D9B6D9A4285
:1088200002D1034B02225A6110BD00BF0044004038
:1088300000080140E4030020980C0020A00C002058
:10884000274910B50B8813F0200F15D0254B5A6817
:1088500018680132202A08BF0022824205D05C68D5
:108860008888E118C0B208725A601F4B0A221A6049
:108870001C4B9A6A1D4B1A601948038813F0800F2D
:108880001ED01A4B1A68DAB9164BD3F88040D3F8C9
:1088900084108C4210D0D3F88410CC1894F888C07F
:1088A0000131A0F804C0C3F88410D3F88410202943
:1088B00006D1C3F8842003E040F2277105F060FC84
:1088C0000748038813F0400F08D040F2266105F0F6
:1088D0004FFD044BD3F88420D3F8803010BD00BF87
:1088E00000380140E4030020A40C00209C0C002070
:1088F00030B5054687B0564805F08AFD4FF4003084
:10890000012104F0D3FB0420012104F0C1FB042069
:10891000002104F0D9FB0820002104F041F806AC46
:108920004FF0040324F8083D03234A4821468DF8FC
:10893000123015338DF8133003F0A2FF4823454859
:108940008DF8133021464FF00803ADF8103003F0D6
:1089500097FF684605F0DEFB0B2D25D8DFE805F014
:108960002406090C0F1215181B1E20224FF4615308
:108970001CE04FF4964319E04FF4E14316E04FF446
:10898000164313E04FF4614310E04FF496330DE0CB
:108990004FF4E1330AE04FF4613307E02E4B05E07A
:1089A0002E4B03E02E4B01E04FF416530093009B37
:1089B00006A95B0841F8183D2548694605F0E0FC2A
:1089C00026230024012505A88DF8143007238DF8EF
:1089D00015308DF816408DF8175004F0C1F81C487A
:1089E00040F2FF3105F0A0FC28212246184805F08E
:1089F000C7FB2A46164840F2277105F0C1FB2A46FC
:108A0000134840F2266105F0BBFB2A46104840F2AD
:108A1000255105F0B5FB22460D4840F2244105F0F2
:108A2000AFFB22460A4840F6460105F0A9FB224664
:108A3000074840F66A1105F0A3FB6021224604486E
:108A400005F09EFB2946024805F08CFB07B030BDBF
:108A5000004400400008014090D0030020A107001E
:108A600040420F0030B5054687B0524805F0D0FCB3
:108A70004FF48040012104F00BFB0420002103F09F
:108A80008FFF06AC4FF4007324F8083D03234A48D7
:108A900021468DF8123015338DF8133003F0F0FEB7
:108AA000482345488DF8133021464FF48063ADF8D4
:108AB000103003F0E5FE684605F02CFB0B2D25D8A1
:108AC000DFE805F02406090C0F1215181B1E2022E2
:108AD0004FF461531CE04FF4964319E04FF4E14327
:108AE00016E04FF4164313E04FF4614310E04FF4E7
:108AF00096330DE04FF4E1330AE04FF4613307E0C1
:108B00002E4B05E02E4B03E02E4B01E04FF41653A5
:108B10000093009B06A95B0841F8183D254869466B
:108B200005F02EFC25230024012505A88DF814301E
:108B300007238DF815308DF816408DF8175004F086
:108B40000FF81C4840F2FF3105F0EEFB28212246C9
:108B5000184805F015FB2A46164840F2277105F023
:108B60000FFB2A46134840F2266105F009FB2A460E
:108B7000104840F2255105F003FB22460D4840F213
:108B8000244105F0FDFA22460A4840F6460105F068
:108B9000F7FA2246074840F66A1105F0F1FA60211B
:108BA0002246044805F0ECFA2946024805F0DAFAB4
:108BB00007B030BD003801400008014090D00300EC
:108BC00020A1070040420F00704700BF184B1A78E1
:108BD000AAB15968174A013159601168164B013121
:108BE00011601A6812B11A68013A1A60134B1A68B8
:108BF00012B11A68013A1A6000220D4B00E00122FE
:108C00001A700F4B1A683AB11A68013A1A601B6859
:108C100013B90C4B01221A700B4B1A683AB11A683F
:108C2000013A1A601B6813B9084B01221A70704789
:108C30008C040020540700209C0C0020A00C002075
:108C4000A40C0020A80C0020980C0020A90C0020E7
:108C5000014B5868704700BF8C04002008B5042001
:108C600004F046FC4FF4FA5004F052FC012004F0EA
:108C700055FC04480321002204F040F8012004F0D0
:108C800063FC08BD9AC302000828F8B508D009287B
:108C90000ED008B100205AE03B4B188880B256E055
:108CA000394B588840F26B1380B2584300134EE0A2
:108CB000354B988880B207F0D5FF07F0B7FB00224C
:108CC000324B07F007FC22A3D3E9002306460F46E8
:108CD00007F000FC20A3D3E9002307F049FA1EA304
:108CE000D3E9002304460D463046394607F0F2FB2F
:108CF0001BA3D3E9002307F017FD02460B462046CD
:108D0000294607F011FD07F0A7FE07F08FFB0022B0
:108D10001F4B07F009FD06F031FE13A3D3E9002332
:108D200007F0D8FB12A3D3E9002307F021FA02468B
:108D30000B4611A1D1E9000107F0F6FC10A3D3E91D
:108D4000002307F013FA07F087FE08F0A9F9F8BD31
:108D50006666666666660AC06666666666660A4037
:108D60009A99999999990140C3F5285C8FA272400C
:108D70000000000000FEAA409A999999FD6F2F41CA
:108D8000C3F5285C8F127140940400200000303F2E
:108D900000002440F0B593B011AF01240025032654
:108DA00040483946ADF844408DF846608DF847504C
:108DB00003F066FD39463C48ADF844608DF84660E6
:108DC0008DF8475003F05CFD2046214604F052F92F
:108DD00021464FF4007004F05BF9344803F09AF92F
:108DE000334B32480193334B01A9029380230693FE
:108DF000DB18079303F540730893A3F57873099381
:108E000003F5FF530A930395049605950B9503F01C
:108E1000F1F92648214603F01DFA4FF46023264855
:108E20000CA90E938DF834400C958DF835400F95B4
:108E30008DF8406002F0A2FF1F4808212246334609
:108E400003F01EF81C4829460222334603F018F8A6
:108E5000334632461848092103F012F82A461648CC
:108E60004FF4FC6102F0CEFF1348214602F0C0FF30
:108E70001148214602F0B2FF0F4802F0CDFF0E4824
:108E800002F0D0FF0028FAD10B4802F0CFFF0A48C9
:108E900002F0D2FF0028FAD10748012102F0D0FFEA
:108EA00013B0F0BD00080140000C01400800024072
:108EB0004C2401409404002000240140AFF30080C2
:108EC000014B03221A6070479C040020044A054BA2
:108ED000927A0AB1052200E001221A60704700BFB1
:108EE000B80C00209C040020704700BF014B0022FA
:108EF0005A6070479C04002008B5074B1A6892B26C
:108F000042F008021A601A6892B242F004021A6033
:108F1000FFF7D6FF08BD00BF405C004010B5064C0F
:108F20004FF6FB73226802EA03032360FFF7CEFFCC
:108F30004FF40643236010BD405C0040072818BF73
:108F40001F4B10B51E4C18BF18702378052B33D853
:108F5000DFE803F003060A0E1621FFF7DFFF2BE020
:108F6000FFF7DCFF042328E002236370013324E0D1
:108F70006378013BDBB263706378FBB9042218E0CD
:108F8000104B1A6892B242F010021A600523237047
:108F9000DB18637012E06378013BDBB263706378C7
:108FA00063B9084A4FF6EF73116801EA03031360CF
:108FB0000622034B1A7001E00623237010BD00BF88
:108FC0001C0D0020405C0040034B9B7A13B1034B07
:108FD00005221A60704700BFB80C00209C040020D6
:108FE000014B04221A6070479C040020034B1A7A3C
:108FF000202A01D100221A72704700BF9C04002071
:10900000704700BF212808B508D1124B1B681B7898
:1090100003F07F03212B1AD10F4B0EE0202816D12D
:109020000C4B0E4A1B681B7810720D4A03F07F032D
:10903000212B0CBF134600234BB1064A4FF0000111
:1090400012680020518293619847002000E00220BE
:1090500008BD00BF180D0020999000089C04002056
:10906000B5900008074B1B681B7803F07F03212B8A
:1090700005D1022801D0222801D1002000E00220E1
:10908000704700BF180D002019B9012801D8084603
:1090900000E00220704700BF28B9044B4FF00802DF
:1090A0001B681A8200E00248704700BF180D0020BC
:1090B0004800002028B9044B4FF008021B681A82B0
:1090C00000E00248704700BF180D00204800002053
:1090D0000B4B10B5DA6882B11B68052B01D000225A
:1090E0000BE0002303E00749595CC15401330449F4
:1090F000CC68A342F7D30023CB60104610BD00BF5D
:109100009C040020200D0020084BDB68082B01D8B0
:1091100000200AE00023064A9A5CC2540133092B5E
:10912000F9D1024B0022DA60012070479C04002034
:10913000200D002010B5074C0B468AB2C021636099
:1091400005F042FF0120A18806F04CF9012006F04D
:1091500017F810BD9C04002007B5142200238DF8D9
:10916000042001A801228DF806308DF807208DF823
:10917000053003F0F5FC0EBD07B5142200238DF871
:10918000042001A801228DF806308DF807208DF803
:10919000053003F0E5FC0EBD08B5064B1B68DB7817
:1091A000042B01D9002004E0034901EBC30105F0C1
:1091B000B3FA08BD180D00205000002008B5024980
:1091C00005F0AAFA08BD00BF7000002008B50249EA
:1091D00005F0A2FA08BD00BF78000020334B10B59F
:1091E0001B686FF03F0200245A72DC729C722046AA
:1091F00005F03EFF20464FF4007105F057FF1021A7
:10920000204605F069FF4021204606F0BFF8802186
:10921000204606F0ABF8204605F0E8FF244B204638
:1092200093F8641006F000F9204605F0B7FF01201E
:10923000214605F03BFF0120C02106F097F80120F0
:10924000202105F049FF0120214605F05DFF0220A5
:109250004FF4C06105F02AFF02204FF4807106F040
:1092600085F80220214605F04FFF0220202105F05D
:1092700033FF0320214605F019FF03204FF48871C6
:1092800006F084F80320402106F0CEF803204FF4C6
:10929000405105F039FF2146032005F01DFF20460F
:1092A00005F048FA034B01221A6010BD180D00208A
:1092B000480000209C04002008B5174B174A196885
:1092C00089B2118016491288098801EA020212F453
:1092D000806F05D04FF6FF321A60124BDB6B984758
:1092E0000E4B1A880E4B1B8803EA020212F4007F11
:1092F00008D009490C4A4FF6FF500860117C013133
:10930000C9B21174054A1288134013F4004F01D0FA
:1093100005F096FD08BD00BF445C0040AE0C002087
:10932000600D0020480000209C04002010B50320A0
:1093300006F0AAF8064C034602464FF48871054829
:10934000E36005F059FE032005F028FF10BD00BFC3
:109350009C040020200D002008B520B104481021F5
:1093600003F0F4FA03E00248102103F0F1FA08BD1B
:10937000000C014038B5064D01232B60054B00243D
:1093800020461C60FFF7E8FF03232B60204638BD12
:10939000405C0040445C004008B5FFF7EBFF08BDAF
:1093A00008B50120FFF7D8FF064B012119600649D7
:1093B0004FF4E0520A8005490020186008601A60E6
:1093C00008BD00BF405C0040600D0020445C0040D0
:1093D000084B10B51B6800249C72FFF7E1FF064A9A
:1093E0004FF406431460043A1360044A1460044ABC
:1093F000138010BD180D0020445C00409C04002028
:10940000600D0020012008B503F0B8FD4FF4000006
:10941000012103F04BFE08BD07B5FFF7F3FFFFF78F
:10942000ABFE05F0AFFC0820012103F031FE102354
:109430000322054801A98DF806208DF80730ADF804
:10944000043003F01DFA0EBD000C0140704700BF50
:10945000704700BF704700BF704700BF704700BF34
:10946000704700BF704700BF704700BF08B5FBF7EB
:109470005BF8052805D9FBF757F840F2F933984215
:1094800001D9012200E00022094B5A60094B1B78E8
:109490006BB1074B08495A68084B0A601AB91A6839
:1094A00042F0080202E01A6822F008021A6008BDC1
:1094B000580700205207002040070020E80600203F
:1094C00010B5FFF7C5FB074C2368C31AB3F5FA7F45
:1094D00007D9054BDA6882F40072DA60FFF7B8FB4F
:1094E000206010BD640D0020000C0140024B03EB16
:1094F000C003D879704700BFB0040020024B03EBD3
:10950000C0035879704700BFB0040020024B03EB42
:10951000C0039879704700BFB0040020024B0B22B3
:1095200002FB0033187A7047B0040020024B0B2274
:1095300002FB0033587A7047B0040020024B0B2224
:1095400002FB0033D87A7047B0040020024B0B2294
:1095500002FB0033987A7047B0040020024B0B22C4
:1095600002FB0033187B7047B0040020024B0B2233
:1095700002FB0033587B7047B0040020024B0B22E3
:1095800002FB0033987B7047B0040020024B0B2293
:1095900002FB0033187C7047B0040020024B0B2202
:1095A00002FB0033587C7047B0040020024B0B22B2
:1095B00002FB0033987C7047B0040020024B052268
:1095C00002FB0033187D7047B0040020024B0522D7
:1095D00002FB0033587D7047B0040020024B052287
:1095E00002FB0033987D7047B0040020024B052237
:1095F00002FB0033D87D7047B0040020024B0522E7
:1096000002FB0033187E7047B0040020024B032297
:1096100002FB0033187F7047B0040020034B032285
:1096200002FB003393F91D00704700BFB004002017
:10963000024B032202FB0033987F7047B0040020E6
:10964000024B03EBC00393F820007047B0040020E6
:10965000024B03EBC00393F821007047B0040020D5
:10966000024B03EBC00393F822007047B0040020C4
:10967000024B03EBC00393F823007047B0040020B3
:10968000024B03EBC00393F824007047B0040020A2
:10969000024B03EBC00393F825007047B004002091
:1096A000024B03EBC00393F826007047B004002080
:1096B000024B03EBC00393F827007047B00400206F
:1096C00006281AD8DFE800F004070A0D1013160068
:1096D0000A4B9B6A10E0094BDB6A0DE0074B1B6BE2
:1096E0000AE0064B5B6B07E0044B9B6B04E0034B0B
:1096F000DB6B01E0014BDB7B0B607047B0040020AB
:1097000070B5C0F30741054600220120FBF738F988
:109710000A4C0602C5F3072100220120A662FBF7CE
:109720002FF9064301203602E9B20246A662FBF792
:1097300027F906433609A66270BD00BFB0040020B9
:109740002D4B032202FB003310B51C3393F901208B
:109750003F2A01DD3F225A70274B032202FB0033D0
:109760001C3393F9012012F13F0FBCBF6FF03E0292
:109770005A70214B032202FB00331C339A781F2AB4
:1097800001D91F229A701C4B032202FB00324FF4B6
:1097900040211964127F012A04BF4FF450221A6439
:1097A000154B03EBC00292F827203AB9033202FBB3
:1097B0000032527F196C02F07F020BE0032101FBA3
:1097C000003191F81DC002F003020CF07C0C196C02
:1097D0004CEA0202084C41EA02221A64032303FB0A
:1097E0000040236C827F42EA030318462364FFF79C
:1097F00087FF236CA36310BDB004002008B5044BA1
:10980000032202FB00339977FFF79AFF08BD00BFE0
:10981000B004002008B5044B032202FB0033597743
:10982000FFF78EFF08BD00BFB004002008B5044B51
:10983000032202FB00331977FFF782FF08BD00BF48
:10984000B0040020264B052210B502FB00331A7D20
:10985000012A01D901221A75214B052202FB00338E
:1098600014335A78032A01D903225A701C4B05225B
:1098700002FB003314339A780F2A01D90F229A7011
:10988000174B052202FB00331433DA78032A01D97F
:109890000322DA70124B052202FB003314331A79CB
:1098A0000F2A01D90F221A710D4C052303FB00402A
:1098B00000F114021379017D43F42023507843EA28
:1098C000C133917843EA4033D27843EA012343EA33
:1098D000421318462364FFF713FF236C636310BD24
:1098E000B004002008B5044B052202FB00331976B2
:1098F000FFF7A8FF08BD00BFB004002008B5044B67
:10990000052202FB0033D975FFF79CFF08BD00BF9D
:10991000B004002008B5044B052202FB0033997502
:10992000FFF790FF08BD00BFB004002008B5044B4E
:10993000052202FB00335975FFF784FF08BD00BF05
:10994000B004002008B5044B052202FB0033197552
:10995000FFF778FF08BD00BFB0040020514B0B2279
:1099600010B502FB00331A7A032A01D903221A72B6
:109970004C4B0B2202FB003308339A78032A01D99F
:1099800003229A70474B0B2202FB003308331A79EB
:109990000F2A01D90F221A71424B0B2202FB00330E
:1099A00008335A79072A01D907225A713D4B0B22F5
:1099B00002FB003308339A790F2A01D90F229A71DA
:1099C000384B0B2202FB003310335A780F2A01D98F
:1099D0000F225A70334B0B2202FB003310339A785C
:1099E0000F2A01D90F229A702E4B0B2202FB003254
:1099F000117AC90341F400241C64527A12B141F473
:109A000004211964274B0B2101FB0031C97A19B1DC
:109A1000196C41F400511964224B8AB90B3202FBD4
:109A20000032083292F804C091784FEACC1C1C6CCA
:109A30004CEAC12C51794CEA040242EA01121DE0C1
:109A40000B2202FB0032127C1AB11A6C42F48052D3
:109A50001A64144B0B2101FB0031103191F801E025
:109A60001A6C897842EACE1201F0070C42EA0C1215
:109A700011F0080F1A6402D042F400621A64094B14
:109A80000B2202FB00300830C27922B981791A6CAE
:109A900041EA02021A64034C206CFFF731FE236C8A
:109AA000236310BDB004002008B5064B0B2202FB57
:109AB00000330833DA791AB10022DA71FFF74EFF6A
:109AC00008BD00BFB004002008B5064B0B2202FB06
:109AD00000330833DA791AB90132DA71FFF73EFF41
:109AE00008BD00BFB004002008B5044B0B2202FBE8
:109AF00000339974FFF732FF08BD00BFB0040020A7
:109B000008B5044B0B2202FB00335974FFF726FF04
:109B100008BD00BFB004002008B5044B0B2202FBB7
:109B200000331974FFF71AFF08BD00BFB00400200E
:109B300008B5044B0B2202FB00339973FFF70EFFAD
:109B400008BD00BFB004002008B5044B0B2202FB87
:109B500000335973FFF702FF08BD00BFB0040020B7
:109B600008B5044B0B2202FB00331973FFF7F6FE16
:109B700008BD00BFB004002008B5044B0B2202FB57
:109B800000339972FFF7EAFE08BD00BFB004002061
:109B900008B5044B0B2202FB0033D972FFF7DEFE3F
:109BA00008BD00BFB004002008B5044B0B2202FB27
:109BB00000335972FFF7D2FE08BD00BFB004002089
:109BC00008B5044B0B2202FB00331972FFF7C6FEE7
:109BD00008BD00BFB004002010B5254B4FF4602233
:109BE0001A6403EBC00292F8272012B14FF47022DE
:109BF0001A641F4B03EBC00292F8211092F820C0A8
:109C00001C6C090341EA8C312143196492F822202B
:109C1000012A04BF41F480611964154B03EBC001B4
:109C200091F823C01A6C42EA0C221A6491F82410AD
:109C3000012904BF42F080021A640D4B03EBC002FD
:109C400092F82520012A03D11A6C42F040021A64CE
:109C5000074C04EBC00090F82620236C43EA021363
:109C600018462364FFF74CFD236CE36310BD00BF6F
:109C7000B004002008B5044B03EBC00383F82610A2
:109C8000FFF7AAFF08BD00BFB004002070B50F4B5E
:109C9000064603EBC00393F82650032D02D00321A0
:109CA000FFF7E8FF3046FFF797FF084B9C6A14F474
:109CB000002F1CBF6FEA04346FEA1434032D03D065
:109CC00030462946FFF7D6FF204670BDB00400207D
:109CD00008B5044B03EBC00383F82510FFF77CFFA6
:109CE00008BD00BFB004002008B5044B03EBC0035F
:109CF00083F82410FFF770FF08BD00BFB0040020F8
:109D000008B5044B03EBC00383F82310FFF764FF8F
:109D100008BD00BFB004002008B5044B03EBC0032E
:109D200083F82210FFF758FF08BD00BFB0040020E1
:109D300008B5044B03EBC00383F82110FFF74CFF79
:109D400008BD00BFB004002008B5044B03EBC003FE
:109D500083F82010FFF740FF08BD00BFB0040020CB
:109D6000064B10B503EBC003044683F82710FFF73A
:109D700033FF2046FFF7E4FC10BD00BFB004002015
:109D800010B5144B00221A6403EBC002527912B1D1
:109D90004FF400721A640F4B03EBC00292791AB1B0
:109DA0001A6C42F480721A640A4B03EBC003DA792E
:109DB0000F2A01D90F22DA71064C04EBC000C279D8
:109DC000236C42EA030318462364FFF799FC236CD3
:109DD000E36210BDB004002070B5084D9DF810E09E
:109DE0009DF8146005EBC00426716270A37084F8BE
:109DF00003E005F83010FFF7C3FF70BDB00400208A
:109E000008B5034B03EBC0039971FFF7B9FF08BD19
:109E1000B004002008B5054B03EBC003597109B12C
:109E20000422DA71FFF7ACFF08BD00BFB0040020C8
:109E300008B5054B042903EBC003D97101D00022FA
:109E40005A71FFF79DFF08BDB00400202DE9F047CF
:109E5000344D0446401990F844000E461746984683
:109E6000DDF82090DDF824A004281FD8DFE800F0FA
:109E700003090F151B002046FFF770FD651901232C
:109E800016E02046FFF7A8FE6519022310E02046E1
:109E9000FFF7D8FC651903230AE02046FFF750FCC2
:109EA0006519042304E02046FFF76AFF65190023C3
:109EB00085F844301B4B03EBC40494F82620012A98
:109EC0000DD002D3022A23D111E016B19B6A9B0C5C
:109ED0003370EFB1134B9B6A9B0A3B7018E0B8F1EB
:109EE000000F15D09B6A9B0AC8F8003010E0B8F14B
:109EF000000F04D09B6ADB0B5B01C8F80030B9F19E
:109F0000000F05D0074B9B6AC3F3842389F8003008
:109F1000BAF1000F03D0034B9B6A8AF80030BDE80A
:109F2000F08700BFB0040020214B10B503220024AD
:109F30004FF0050C02214FF0010E83F825E0197354
:109F400083F80EC09A745C7483F81CE083F81DC01B
:109F500083F81EC083F8202083F8212083F8224054
:109F600083F8234083F8244083F8261083F82740A1
:109F70001C755C759C75DC751C765C719C71DC7164
:109F800019725C72DC729C725A73DC731C7420460A
:109F9000FFF758FC2046FFF7D3FB2046FFF71CFED7
:109FA0002046FFF7EDFE2046FFF7D8FC10BD00BFAE
:109FB000B004002008B5044A0023917A034A1846E9
:109FC0001370FAF737FC08BDF00B0020580C002086
:109FD0002DE9FF417F4B1A7822B901321A706FF0D8
:109FE00000425A607B4B1C7A5CB9E0B2FAF766FA21
:109FF000784B03F10C0210550134082CF5D10122E5
:10A000001A7227240025E8B2FAF758FA724A535D0B
:10A01000834219D0714B291D53F821305055022B22
:10A0200005D0032B0AD0012B0ED168B106E058B938
:10A030006B4A115D012907D1135505E0684B1A5D84
:10A04000012A01D101321A5501350134082DDAD126
:10A05000644EF36993B1644C25787DB9FEF7F8FD41
:10A06000624AF3691268821A002AB8BF52429A42C1
:10A0700004D9284601F028FA01232370594E336A87
:10A0800093B15B4C25787DB9FEF7E2FD594A336AFE
:10A090001268821A002AB8BF52429A4204D928464E
:10A0A00001F012FA012323704A4D534C2A7D93008C
:10A0B00004EBC3010E7B002E00F028814F48504F67
:10A0C000504E0021C318BF18B61810460A46009714
:10A0D0000196FFF7BBFE2B7D04EB4314227B013A74
:10A0E000042A00F20281DFE812F005004E00D300DE
:10A0F0004E00D300444A374D926812F0200F1BD017
:10A100005D192A7E022A04D1404AD25C002A00F05E
:10A11000EC80394A2F4C02EB43121846517AFAF779
:10A1200089FB207DFFF7C0FC237D384A0021E4181D
:10A13000D15402232376D8E05D192A7E012A04D166
:10A14000324AD25C002A00F0D0802B4C184604EB37
:10A150004313997AFAF76EFB1E4B187D04EB4014FB
:10A16000A37A13B9FFF7B0FC04E0284B1B5C0BB1DA
:10A17000FFF79AFC174A2549137D0020D218C854CE
:10A1800001231376B1E01F4A124DD256002A3FDB5D
:10A190005D192A7E022A02D11C4AD25C8AB1164A73
:10A1A0000C4C02EB43121846517AFAF743FB207D20
:10A1B000FFF77AFC237D154A0021E418D1540223CD
:10A1C0002376044C257DFEF743FD04EB8504606097
:10A1D00056E000BFF804002004050020180C002001
:10A1E000680C002008000020550C0020500C0020B6
:10A1F0006D0B0020480C0020F00B0020940B002079
:10A20000780B0020E80B0020000C0140540C0020CB
:10A210005B191B7E012B11D0FEF71AFD2B7D894A9D
:10A2200005EB830502EB43139B8B0A2253436A68B9
:10A23000821A002AB8BF52429A4204DC824B834AF7
:10A240001B7DD35CE3B1804D7E4C287D04EB401335
:10A25000997AFAF7EFFA287D04EB4014A37A13B940
:10A26000FFF732FC04E0794B1B5C0BB1FFF71CFCE1
:10A27000754A7649137D0020D218C85401231376FD
:10A28000714B1A7D6F4B03EB42131B7B042B20E0B9
:10A290006D4A9A18127E022A02D16C4AD25C8AB1A7
:10A2A000684A694C02EB43121846517AFAF7C2FA2F
:10A2B000207DFFF7F9FB237D644A0021E418D15487
:10A2C00002232376604B1A7D5E4B03EB42131B7B0C
:10A2D000052B0AD15E4B9A6812F0200F15BF4FF480
:10A2E00080624FF480625A611A61FEF7B1FC564CED
:10A2F000E369C31A002BB8BF5B420A2B40F31A83F1
:10A30000FAF784F9FEF7A4FCE06113E3FEF7A0FC82
:10A31000EB69C31A002BB8BF5B420A2B40F30A83D8
:10A32000FAF774F9297D3046490141F00A0101F03C
:10A33000EA0100F08BFF0446287D01F0E9F82B7D4F
:10A340000C20584343494218157A0DB1455800E096
:10A350005568414AD25C032A00F2E480DFE802F04B
:10A3600002801C4B002C00F0DD80364A364D02EB9B
:10A370004311C97F384E29B11846FAF75BFA2B7D95
:10A38000032207E002EB43121846517AFAF752FA19
:10A390002B7D0222F254C5E04CB95B0143F0080169
:10A3A00001F0E801204600F051FF002862D0264E5F
:10A3B000244B307D03EB4013D97F002900F0AB80A4
:10A3C000002D84EAE472B8BF6D42A2EBE472AA42A7
:10A3D00002D0002C40F09980204B53F830108A4274
:10A3E00080F0998003EBC0031979FAF723FA164B32
:10A3F00001211B7D8DE0002D84EAE471B8BF6D4220
:10A40000A1EBE471A94202D0002C40F08480134AF1
:10A410000D4D52F83300104E814208D202EBC302B8
:10A4200018461179FAF706FA2B7D012208E0054A51
:10A43000184602EB4313597AFAF7FCF92B7D0222F6
:10A44000F25468E0F00B0020F8040020540C0020C7
:10A45000000C01409C0B0020580C00207C0B0020BD
:10A4600044BB5B0143F0080101F0E801204600F025
:10A47000EDFEF8B9FEF7ECFB1F4D204A2B7D4FF0A7
:10A480000A0E02EB4311B1F81CC099004E19766810
:10A490000EFB0CFC861B002EB8BF7642664541DDE4
:10A4A00002EBC1021846917AFAF7C4F92B7D144ADF
:10A4B000D45437E0104E114A337D02EB4312D17F62
:10A4C00049B3002D84EAE472B8BF6D42A2EBE47296
:10A4D000AA4200D0C4B90B4951F833108A421AD3AA
:10A4E000064A184602EB4313597AFAF7A3F9024BCE
:10A4F00002211B7D0DE000BFF8040020F00B0020BE
:10A50000580C00207C0B00201846FAF793F9337D95
:10A510000321A34AD154A34D2E7DFEF799FB05EBF1
:10A52000860568609F4DA04F2B7DA04E1846F618FB
:10A53000FF189F4B002103EB80030A46019600970A
:10A540009C4EFFF783FC287D06EB40139B6943B3C9
:10A55000F9F73EFF28B3287D84EAE47206EB401346
:10A560009B69A2EBE4729A421BD900F0ADFF2A7DF1
:10A57000914906EB42139B7F0120885443B1B27F7F
:10A580009A4205D1013800F09FFF002000F0EAF95F
:10A59000844B8A4A1B7D0F33D15C012901D10131E3
:10A5A000D154804D2B7D022B25D8002000F02AFDB0
:10A5B00095F8203010F0010F03F0F80385F82030F3
:10A5C0001CBF43F0010385F8203010F0040F8DF814
:10A5D0000C0006D0734B93F8202042F0020283F85F
:10A5E000202010F0100F06D06E4B93F8202042F080
:10A5F000040283F82020724A137853B1694991F814
:10A6000020100B4205D16F496F480978037001B9DA
:10A6100011706D4B1B784BB1624A92F8202003EA0F
:10A6200002029A4202D1694B01221A705D4B93F8E3
:10A63000202012F0010F0AD093F8213013F0010FFF
:10A6400005D15E4BDA78012A01D10132DA70554B1F
:10A6500093F8202012F0020F0AD093F8213013F063
:10A66000020F05D1554B1A79012A01D101321A7115
:10A670004C4B93F8202012F0040F0AD093F82130AD
:10A6800013F0040F05D14D4B5A79012A01D1013243
:10A690005A71444D03222B7D04A8B3FBF2F28218B9
:10A6A00012F9042C95F82010002A85F821104ADAB6
:10A6B0005B0143F01601002001F0F60102AA00F050
:10A6C000DDFD9DF80A3013F0400F08D02A7D3B498C
:10A6D00052001B32885C012801D10130885413F0EC
:10A6E000800F0AD02F49354A097D0E3112F811002A
:10A6F000012802D1013002F8110013F0100F09D027
:10A70000284A2E49127D52001B32885C012801D153
:10A710000130885413F0200F0AD0224A274B127DB3
:10A720000E3213F81210012902D1013103F8121070
:10A730001C4B0020197D02AA490141F0160101F0CD
:10A74000F60100F037FF174F1A4E3B7D06EB431220
:10A750005269002A00F082801D4AD55C002D7DD10F
:10A76000002C7CD05B0143F0020101F0E20128469D
:10A7700000F032FD8046387DFAF740F8397DC0EBB5
:10A78000080806EB41135B69B8F1000F83EAE37236
:10A79000B8BFC8F10008A2EBE372904568DD19E08C
:10A7A000580C0020F8040020780B0020E80B002053
:10A7B000940B0020F00B0020E40B0020680C00201C
:10A7C000900B0020740B0020890B0020970C0020B8
:10A7D000880B0020002B0EDD084600F075FE3B7D47
:10A7E00006EB43139B7F3BB3B27F9A4224D12846AA
:10A7F00000F06AFE1DE02846022200F0C7FC397D09
:10A800002846490141F0080101F0E80100F03EFE50
:10A810003B7D06EB43139B7F73B1B27F9A420BD112
:10A8200029462846022200F0B1FC2846082100F003
:10A830002DFE284600F096F83F4B404A1B7D15330D
:10A84000D15C012901D10131D1543B4B3C4A1B7DE4
:10A8500001211846D15400F085F809E044B95B01A4
:10A8600043F0080101F0E801002000F0EFFC20B106
:10A87000314D344B2E7D9B5D43B32F4B324A1B7DB4
:10A8800002EB4312D28912B92E4AD35C1BB3FEF7F6
:10A89000DFF9294D2C492B7D4FF00A0C9A0001EB72
:10A8A000C201C9895219526A0CFB01F1821A002AAD
:10A8B000B8BF52428A420EDD244EF25C5AB91846A5
:10A8C000FFF702F92B7D0122F25404E0FEF7C0F9F4
:10A8D00005EB86056862184E1D4D307D002C55F83D
:10A8E0003030B8BF64429C420AD2FEF787FE337D07
:10A8F00005EBC3056A7982420DD11846002108E0B4
:10A90000FEF77CFE337D05EBC3056979884202D0F2
:10A910001846FEF7E7FF084C207D00F031F8237D54
:10A920000133DBB223750BB100232375FEF790F9D9
:10A93000014BD861BDE8FF81F8040020680C0020BD
:10A94000880B0020600C0020F00B0020640C00201D
:10A950007C0B0020024B1A5C0AB901321A54704772
:10A9600020050020024B1A5C0AB10F221A547047CE
:10A9700020050020014B185C704700BF2005002017
:10A980002DE9F3474501EDB2044645F07C01002076
:10A9900001AA00F073FC4FEA440A0227012307FAD8
:10A9A0000AF703FA0AF3A94A9DF8061002EB4412CB
:10A9B000127A0B400F4012F0800F02F07F0804D093
:10A9C000A34A966886F0200601E0A14A966808F13D
:10A9D000FF32C6F34016072A00F2E182DFE812F0E8
:10A9E000080008000800080079017901790179015F
:10A9F000984A125D013A0E2A00F2D182DFE812F085
:10AA00000F003D00550064007D0085009400A90002
:10AA1000D90020013001CF024F015901B60201AA2D
:10AA200045F0140100208B4E00F028FC9DF8053005
:10AA300045F0060506EB84077B602946002000F000
:10AA400005FC0222B8602146002000F09FFBA8F11F
:10AA500002080020294640F2FF7200F003FD5FFA71
:10AA600088F800200322214600F06AFBB8F1010FAC
:10AA700040F2CB810423335591E2764E002006EB61
:10AA800084035A68214602F00402824214BF052260
:10AA9000012200F055FB6D4B6201D25845F00801D0
:10AAA000002000F0DFFC0323E5E7002B00F07782B5
:10AAB00045F00201002000F08FFB664B04221A557E
:10AAC000654B43F824006AE2624E002006EB8403E3
:10AAD0005A68214602F00402824214BF0622022272
:10AAE00000F02EFB594B6201D25845F0080152424A
:10AAF000002000F0B7FC0523BDE7002F00F04F82D7
:10AB0000204600F0E1FC06223CE200202146032220
:10AB100000F016FB4D4B45F0080103EB44135A6857
:10AB2000002000F09FFC77E1002F40F0388245F0D4
:10AB30000805384629463A4600F094FC434B38460F
:10AB400003EB44135A682946524200F08BFC08225A
:10AB500018E2002F00F0238245F00201002000F0EF
:10AB60003BFB06460020024645F0080100F07AFC57
:10AB7000394B002053F824702146BF1B43F8247042
:10AB8000032200F0DDFA314B6701FB185A6845F0EB
:10AB90000601002000F066FC07F0E00132460020CC
:10ABA00000F0CCFB00200246214600F0EFFA09221B
:10ABB000E8E1002000F026FA40FA0AF010F0010F58
:10ABC00000F0ED8145F002063146002000F004FB64
:10ABD000224B45F0080543F8240000200246294690
:10ABE00000F040FC00200222214600F0CFFA0020B5
:10ABF0003146024600F0A2FB67010020024607F042
:10AC0000E001A8F1030800F099FB5FFA88F8002141
:10AC10002046F9F7C9FDB8F1010F0E4E0ED80020FD
:10AC20002146022200F0B2FA084B2946FF187A6842
:10AC30000020524200F016FC0A231CE70E231AE7FC
:10AC4000002F00F0AC810B229CE100BFF00B002034
:10AC5000000C014020050020700B0020140C002087
:10AC6000002F40F09C8145F00201384600F0B4FA14
:10AC700045F0080106463A46384600F0F3FB61010C
:10AC8000022296FBF2F201F0E001384600F056FB9A
:10AC90003A463846214600F079FA0D2272E100204A
:10ACA00000F0B0F940FA0AF010F0010F00F07781DF
:10ACB00067E1AB4E45F0060106EB84050020AA686B
:10ACC00000F0D0FB2A790020214600F039FA002359
:10ACD000D1E6A34A125D013A0E2A00F26081DFE854
:10ACE00012F00F003500570067008A005E019D00DA
:10ACF0005E015E01D300E200B6000F015401450180
:10AD000045F0140101AA0020954E00F0B7FA9DF815
:10AD1000057006EB8403002002225F60214600F0EC
:10AD200035FA002045F0060140F2FF7200F09AFB70
:10AD300000200322214600F003FAB8F1060F03D0E9
:10AD4000B8F1080F7FF496AE02221BE1B8F1060FAE
:10AD50000CD1834B002003EB84035A68214602F098
:10AD60000402824214BF0522012205E0B8F1080F57
:10AD700004D100202146032200F0E2F9794B620160
:10AD8000D25845F00801002000F06CFB0322F9E0E6
:10AD9000A8F10502D2B2012A05D823B1B8F1060FF5
:10ADA0006F4E34D166E6002E00F0F9800C22E9E007
:10ADB000B8F1050F0CD16A4B002003EB84035A68ED
:10ADC000214602F00402824214BF0622022205E05C
:10ADD000B8F1070F04D100202146032200F0B0F99A
:10ADE000604B6201D25845F008015242002000F049
:10ADF00039FB0522C6E0A8F10503DBB2012B08D818
:10AE00003FB1B8F1050F564E01D1022333E60F23AF
:10AE100031E6002E00F0C3800722B3E0002E40F0A0
:10AE2000BE804F4F304607EB84035A68214602F03C
:10AE30000402002A14BF0522012200F081F9494BC7
:10AE4000304603EB441345F008015A6818E0002E21
:10AE500040F0A580424F304607EB84035A682146F4
:10AE600002F00402002A14BF0622022200F068F950
:10AE70003C4B304603EB44135A6845F008015242FC
:10AE800000F0F0FA0A2339E0002E00F0888045F047
:10AE90000201002000F0A0F9314B0B2103EB8402EA
:10AEA0001955D0607BE0002E79D145F00201304683
:10AEB00000F092F92B4B4FEA44184FEA840A08EB52
:10AEC0000302274F03EBCA03814645F0060152688F
:10AED00030465E7300F032FA0AEB0703DB6808F0D5
:10AEE000E0019944022399FBF3F2304600F026FA80
:10AEF00030462146324600F049F90D233B554EE0DD
:10AF0000002000F07FF840FA0AF010F0010F46D060
:10AF1000134B0E2245F002061A553146002000F070
:10AF20005BF9114B45F0080143F82400002002466C
:10AF300000F098FA21460020022200F027F90020B4
:10AF40003146024600F0FAF900206101024601F0A4
:10AF5000E00100F0F3F920460021F9F725FC1EE09E
:10AF600020050020F00B0020140C002000202146BA
:10AF7000022200F00BF9002045F00801024600F023
:10AF800071FA0E22074B1A5509E0064D002005EB19
:10AF900084031A79214600F0D3F800232B55BDE82D
:10AFA000FC8700BF20050020154B10B503EB0012F5
:10AFB000926891420EDD8A1AC2F18074A2424FEA71
:10AFC000001C03DC63445C6812190EE063445A6899
:10AFD000141B0FE00FDA521AC2F18074A2424FEA3A
:10AFE000001C04DC63445C68A21A5A6003E06344FA
:10AFF0005A68A4185C60024B03EB0010816010BD1E
:10B00000680D0020012108B502200A46F9F7B8FCB6
:10B0100008BD00BFF8B51378144613F0600F06465C
:10B020000D4627D1414A127B22BB13F0010F21D1DB
:10B030005F2B1FD83E4A1278E2B913F09F0301D06C
:10B04000082B17D13B4F387860B9384BD97F19B1ED
:10B05000F9F7F0FB032304E00846597AF9F7EAFB15
:10B0600002233B70344F3B7823B10020FEF71CFDD8
:10B0700000233B70002221780220F9F781FC287020
:10B08000002261780220F9F77BFC68700022A17829
:10B090000220F9F775FCA87001220220E178F9F787
:10B0A0006FFCE870237813F0010F3ED15F2B3CD882
:10B0B00003F01E02082A04D0142A2CD0062A34D108
:10B0C0001BE0242171435B090C2000FB0313A578CE
:10B0D00094F803C0194A4CEA05259D50A37813F053
:10B0E000080F22D02678760900FB0616B3586FEABF
:10B0F00003536FEA1353B35017E0242256435B09FE
:10B100000C22A17802FB0363E27842EA01220B4998
:10B110005B185A6009E0242256435B090C2202FBAB
:10B1200003630649E2785B181A72F8BDF00B002041
:10B13000600C0020580C0020640C00209C0B0020A8
:10B140002DE9F3414901CEB201AC46F01503174693
:10B15000694622468DF804308046FFF75BFF9DF874
:10B1600001C09DF8033046F0140640466946224669
:10B170006D468DF804608DF805C08DF806708DF869
:10B180000730FFF747FFBDE8FC8100BF2DE9F34121
:10B190004901CEB201AC46F0150317466946224676
:10B1A0008DF804308046FFF735FF9DF801C09DF80B
:10B1B000023046F014064046694622466D468DF838
:10B1C00004608DF805C08DF806308DF80770FFF724
:10B1D00021FFBDE8FC8100BF37B541F001030C46FB
:10B1E0006A4601A98DF800300546FFF713FF9DF868
:10B1F00006009DF8052000029DF8073040EA024055
:10B20000184310F4000F18BF40F07F405F2C1AD88D
:10B21000C4F3411314F01E0402D0022C13D106E033
:10B22000032202FB0535084A2D01A8580BE0032232
:10B2300002FB053520F07F41E8B2FFF7B5FE024B77
:10B2400003EB051568683EBD680D002007B541F0A9
:10B2500001036A4601A98DF80030FFF7DBFE9DF877
:10B2600006009DF8073043EA002010F4006F1CBF71
:10B270006FEA00506FEA10500EBD00BF13B541F0E9
:10B280000103144601A96A468DF80030FFF7C2FE9B
:10B290009DF805109DF806309DF807202170A270DA
:10B2A00063709DF804001CBD07B5410141F0160113
:10B2B00001F0F601002001AAFFF7E0FF9DF805303C
:10B2C000D80913F0200F18BF40F002000EBD00BFD8
:10B2D00007B5410141F0160101F0F601002001AA75
:10B2E000FFF7CCFF9DF80530C3F3801013F0100F6B
:10B2F00018BF40F002000EBD37B50C4641EA4011C0
:10B3000001AA0546C9B20020FFF7B8FFB4235D4388
:10B310006408032305F5807503FB04549DF80410AD
:10B320002046FCF7BBFF601C9DF80510FCF7B6FF3C
:10B33000A01C9DF80610FCF7B1FF3EBD5F292DE96A
:10B34000F3410D460646144662D8C1F3411811F088
:10B350001E0102D002295BD11EE0032202FB0088FD
:10B36000344A4FEA081083185B688450E01A0028BA
:10B37000B8BF4042B0F5000F0ADB9C42CCBF2E4C58
:10B380002E4C2C4A1C1902EB0812012313733FE0C8
:10B3900002EB081211733BE0032707FB0087254BE4
:10B3A0003801C1587A00C4EB010C0132BCF1000F26
:10B3B000B8BFCCF1000C00EB030EBCF5000F24F07D
:10B3C0007F40CEF8044043F832001DDBA142CCBFE1
:10B3D000194B1A4B4FEA4818E3184FEA234E4FEA2D
:10B3E000232C3046694601AA8DF807308DF8048079
:10B3F0008DF805E08DF806C0FFF70CFE0D4B03EB52
:10B40000071701233B7303E003EBC20300221A7109
:10B410004FEA244C23123046694601AA8DF80450A5
:10B420008DF805C08DF806308DF80740FFF7F2FD66
:10B43000BDE8FC81680D0020FFFF7F00010080FF58
:10B4400038B50D4668210446FFF7C6FE15B140F039
:10B45000010201E020F0010220466821FFF76EFFA3
:10B4600038BD00BF07B513464FEA222C8DF80410F3
:10B470004FF0000E694601AA8DF805E08DF806C070
:10B480008DF80730FFF7C6FD0EBD00BF07B50B46B0
:10B4900011F01E01024601D0022905D110461946BD
:10B4A0000022FFF74BFF0DE04FF0000C694601AAA8
:10B4B0008DF804308DF807C08DF805C08DF806C0F2
:10B4C000FFF7A8FD0EBD00BF10B5C4B22146640150
:10B4D00000200222E4B2FFF759FE002044F00801E8
:10B4E000FFF7D4FF44F00A010020FFF7CFFF10BDA3
:10B4F00007B59DF810C08DF804108DF80520694639
:10B5000001AA8DF806308DF807C0FFF783FD0EBD48
:10B5100030B5430185B0044643F00303002003A97E
:10B5200002AA8DF80830FFF775FD9DF80E109DF802
:10B530000D209DF80F30090241EA024119432046CF
:10B54000FFF732FD174B03EB041108310A7932B3D0
:10B55000154A0C2000FB0422107A00BB2201D518EA
:10B56000D2586B68C3EB020CBCF1000FB8BFCCF132
:10B57000000CBCF5000F05DB9A42CCBF0B4A0C4A0D
:10B580009A1800E008716101C2F30723D4B201F0F8
:10B59000E0010020C2F307420094FFF7A9FF05B0C5
:10B5A00030BD00BF680D00209C0B0020FFFF7F0016
:10B5B000010080FF07B5937892F800E092F801C08F
:10B5C0008DF8041001AA69468DF805E08DF806C0D3
:10B5D0008DF80730FFF71EFD0EBD00BF37B54401E3
:10B5E00044F01604E4B20D4601AA21460020FFF7FC
:10B5F00045FE9DF8053015F0010F1ABF6FEA436351
:10B600006FEA536303F07F038DF805309DF8053032
:10B6100015F0020F14BF43F0200323F020038DF830
:10B62000053000231846214601AA8DF80630FFF7A1
:10B63000C1FF3EBD37B5440144F01604E4B20D46E7
:10B6400001AA21460020FFF719FE9DF8053015F0EC
:10B65000010F14BF43F0400323F040038DF8053081
:10B660009DF8053015F0020F14BF43F0100323F0CE
:10B6700010038DF8053000231846214601AA8DF8E5
:10B680000630FFF797FF3EBD73B5B42545434B0821
:10B69000032205F5807502FB0355044628460E4635
:10B6A000FCF766FD8DF80400681CFCF761FD8DF861
:10B6B0000500A81CFCF75CFD46EA44148DF8060062
:10B6C000E1B2002001AAFFF775FF7CBD2DE9F74F1D
:10B6D0004001C7B24C05002047F0180101AAFFF74E
:10B6E000CDFD9DF80560640D06F00F053609B542E5
:10B6F0000EDB204604F078FEAD1B80460120A840FA
:10B70000894604F081FE0022334B04F0E3FE0FE093
:10B71000204604F069FE751B80460120A84089463A
:10B7200004F072FE02460B4600202B4904F0FCFF99
:10B7300002460B464046494604F0F6FF05F08CF9F8
:10B7400004F074FE22A3D3E9002304F0C3FE05F045
:10B7500083F904F06BFE0022204B04F0BBFE4FF097
:10B76000FF36B046002582468B460120A84004F0F3
:10B770004BFE02460B465046594604F0ABFE05F020
:10B7800043F9A0F180027F2A98BF2E46034605F1B7
:10B79000010588BF43460E2D01D09846E5E70025F8
:10B7A00047F0120101AA28468DF805308DF8066091
:10B7B0008DF80450FFF7FEFE284647F00C012246A4
:10B7C000FFF750FE2846BDE8FE8F00BFAFF30080B4
:10B7D00004560E2DB29DEF3F000060400000204057
:10B7E00013B5154B587E10F0010003D000206821DE
:10B7F000212201E0682120220024FFF79FFD20463E
:10B800007E21202223460094FFF772FEE1B2002041
:10B810000134FFF739FF1D2CF8D10C210020FFF770
:10B82000DBFC01460020FFF751FF0020162143F208
:10B83000FF12FFF717FE1CBD08000020AFF30080C9
:10B84000084B1868034605E02C2A02D100221A7022
:10B8500003E001331A78002AF6D1024A013313605B
:10B86000704700BF3005002010B50E4B02461B7814
:10B87000ABB10D4B1C7994B19C68601CE4180D2A87
:10B880002273986002D03F2800D851B9064C014677
:10B8900004F10C00FDF74EFC0023A36001E0FCF76F
:10B8A00041FF10BD6C0B00203005002030B5012198
:10B8B000044687B02020FFF7D7FF002C04DA2D20A4
:10B8C0000121FFF7D1FF644200230A2194FBF1F22A
:10B8D00001FB124101AD3031E954591C141E01DD48
:10B8E0000B46F2E7ED181C460121013C15F8010951
:10B8F000FFF7BAFFB4F1FF3FF6D107B030BD00BF8C
:10B9000038B50C4D0446A87801214030C0B2FFF78D
:10B91000ABFF687801214030C0B2FFF7A5FF207867
:10B92000FFF7C4FF6068FFF7C1FF0D200121FFF79B
:10B930009BFF38BD0800002070B5124B06461B78EF
:10B94000EBB1FCF76DFE104C054618B100232371D6
:10B95000012016E0E36C226D934208D21A1992F886
:10B960005420013301203270E364207109E004F1B6
:10B970005400FDF7ADFBE5642065284601E0FCF7C7
:10B980004FFE70BD6C0B0020300500202DE9F34107
:10B9900004460DF10700FFF7CFFF002800F0CB8031
:10B9A0008B4B8C4A93F8941019BB51789DF8070083
:10B9B000403188420DD1D3F89810002940F0BB8067
:10B9C0001179012231F0010183F8942040F0B38015
:10B9D000AFE00D2801D01B2802D100227C4B05E0EE
:10B9E000D3F898207E2A00F2A6800132C3F898206E
:10B9F000A1E0117931F0010103D19DF80700FFF7B3
:10BA000033FF9DF807301F2B0BD9714AD2F89810DD
:10BA10007E297FD8481C891881F89C30C2F898008C
:10BA200078E0082B08D16A4BD3F89820002A71D00F
:10BA3000013AC3F898206DE00D2B6BD1644BD3F81D
:10BA40009830002B66D0634B1A79112A15D158789B
:10BA500001214030C0B2FFF707FF002503E0585D29
:10BA6000FFF702FF01355A4B0121D3F898209C3390
:10BA70009542F4D30D20FFF7F7FE554A00231568D1
:10BA8000D2F8987019461A4633E001290FD002D334
:10BA900002292DD122E04E4E06F19C00805C202828
:10BAA00026D09E1986F81C010133012120E0484868
:10BAB00000F19C0C1CF802C0BCF1200F0AD1012B34
:10BAC00004D91818002180F81C110133424D0221BD
:10BAD000ED180DE0181880F81CC108E03C4E06F186
:10BAE0009C00805C202803D09E1986F81C0101333D
:10BAF0000132BA42C9D3364A0021981880F81C1185
:10BB00000120C2F89810156082F8A001C2F89C319B
:10BB100082F894109DF807301B2B0CD12D4A2C4B2A
:10BB200012790021012A83F89410C3F8981002D1E9
:10BB30000D20FFF799FE264B93F8A001002878D03E
:10BB40000022164683F8A0211546DFF8A8800727B3
:10BB500007FB058720483946013503F023FE30B93D
:10BB6000BE797B7916F0010F237049D007E018F8F1
:10BB700006300736002B5ED0FF2DE6D15BE0FFF7E5
:10BB80005FFE23780546042B0CD1144903F00AFE0E
:10BB90000346D8B12846124903F004FE70B1284686
:10BBA00010490FE00D2B28D10F4903F0FBFD034690
:10BBB00060B128460D4903F0F5FD08B9012305E001
:10BBC0000B49284603F0EEFDB0B90223637017E07D
:10BBD00030050020080000204C060020D91A01087A
:10BBE000DD1A0108E11A0108E71A0108ED1A010837
:10BBF000F21A0108D8180108284603F0CDFD60703C
:10BC000016F0020F04D0FFF71BFE03F0C5FDA07075
:10BC100016F0040F0CD0FFF713FE03F0BDFD010E6C
:10BC2000C0F30722C0F30743A17122716371E07072
:10BC30000120BDE8FC8100232370F9E7704700BFB5
:10BC4000FEE700BFFEE700BFFEE700BFFEE700BF64
:10BC5000704700BF704700BF704700BF704700BF0C
:10BC6000704700BF704700BF704700BF704700BFFC
:10BC7000704700BF704700BF704700BF704700BFEC
:10BC8000704700BF704700BF704700BF704700BFDC
:10BC9000704700BF704700BF704700BF704700BFCC
:10BCA000704700BF704700BF08B5024B1B6898473C
:10BCB00008BD00BF8C0B002008B5024B1B689847DD
:10BCC00008BD00BF5C0C002008B5024B1B689847FC
:10BCD00008BD00BFEC0B002008B5024B1B6898475D
:10BCE00008BD00BF100C0020704700BF704700BFA8
:10BCF000704700BF704700BF704700BF704700BF6C
:10BD0000704700BF704700BF704700BF704700BF5B
:10BD1000704700BF704700BF704700BF704700BF4B
:10BD2000704700BF704700BF704700BF704700BF3B
:10BD3000704700BF704700BF704700BF704700BF2B
:10BD4000704700BF704700BF704700BF704700BF1B
:10BD5000704700BF704700BF704700BF704700BF0B
:10BD6000704700BF704700BF704700BF704700BFFB
:10BD7000704700BF704700BF704700BF436830B5D1
:10BD800023F470230C680A7923F48073234343EA75
:10BD90000223436082688D68CC680A4B45EA040C34
:10BDA00002EA03034A794CEA030343EA420383604D
:10BDB0000B7CC26A013B22F47002DBB242EA0353FD
:10BDC000C36230BDFDF7F1FF002301220274C3609E
:10BDD0000360037143718360704700BF19B18368CA
:10BDE00043F0010302E0836823F00103836070479E
:10BDF00019B1836843F4807302E0836823F480738D
:10BE000083607047C9B212B14368194302E04368C6
:10BE100023EA010141607047836843F008038360AF
:10BE2000704700BF8068C0F3C0007047836843F06C
:10BE300004038360704700BF8068C0F380007047D0
:10BE400019B1836843F4A00302E0836823F4A003DC
:10BE5000836070478068C0F3805070474368013941
:10BE600023F4604343EA41334360704719B14368A8
:10BE700043F4006302E0436823F4006343607047C7
:10BE8000092930B511D94FF0030C0CFB01FC072533
:10BE9000ACF11E0C05FA0CF503FA0CFCC46824EA9C
:10BEA000050343EA0C03C3600EE04FF0030C0CFBE8
:10BEB00001FC072505FA0CF503FA0CFC046924EAD9
:10BEC000050343EA0C030361062A0DD80523013A52
:10BED0005A434FF01F0C0CFA02FC9140436B23EACB
:10BEE0000C020A4342631CE00C2A0DD805235A4376
:10BEF0004FF01F0C233A0CFA02FC9140036B23EA2B
:10BF00000C020A4302630CE005235A434FF01F0C56
:10BF1000413A0CFA02FC9140C36A23EA0C020A433C
:10BF2000C26230BD19B1836843F4801302E08368B4
:10BF300023F4801383607047C06C80B2704700BFE9
:10BF4000014B1868704700BF4C24014019B1436889
:10BF500043F4806302E0436823F4806343607047E6
:10BF600019B1436843F4805302E0436823F48053DB
:10BF700043607047836823F4E04341EA030383602E
:10BF8000704700BF19B1836843F4004302E083683F
:10BF900023F400438360704719B1836843F40213AC
:10BFA00002E0836823F40213836070478068C0F363
:10BFB00040507047092930B511D94FF0030C0CFBE4
:10BFC00001FC0725ACF11E0C05FA0CF503FA0CFC7C
:10BFD000C46824EA050343EA0C03C3600EE04FF093
:10BFE000030C0CFB01FC072505FA0CF503FA0CFC0D
:10BFF000046924EA050343EA0C030361836BC3F37A
:10C00000015CCCEB020202324FF0050CD2B20CFB09
:10C0100002F20CF11A0C0CFA02FC914023EA0C0318
:10C020000B43836330BD00BF836B013923F440139E
:10C0300043EA0153836370470A50704728304058E1
:10C0400080B27047436823F4400323F4007341EA4D
:10C0500003034360704700BF41628262704700BFC4
:10C06000436823F01F0341EA03034360704700BFA6
:10C0700020B1054B9A6842F4000203E0024B9A6833
:10C0800022F400029A6070470024014003681942BC
:10C090000CBF002001207047C9430160704700BFFA
:10C0A0004368006810EA112004D0C9B219420CBFDD
:10C0B00000200120704700BF6FEA11210160704726
:10C0C00008B5134B98420FD003F5A053984213D0F4
:10C0D000A3F5C053984219D14FF40070012100F02C
:10C0E000F3FF4FF400700EE04FF48060012100F088
:10C0F000EBFF4FF4806006E04FF40040012100F0B8
:10C10000E3FF4FF40040002100F0DEFF08BD00BF58
:10C11000002801400268002322F00102026003604F
:10C1200043608360C3602D4B984233D011D83C3BB1
:10C13000984229D006D8283B984221D014339842FF
:10C140004BD11FE0264B984220D01433984244D163
:10C150001EE0244B98422CD008D8A3F56773984270
:10C160001DD003F56273984237D11DE01E4B9842F3
:10C1700029D0143398422BD0283B98422DD11DE072
:10C180001A4B12E0194B15E0184B18E0174B1BE047
:10C19000164B1EE0154B5A6842F470021CE0134B1C
:10C1A0005A6842F0706217E0114B5A6842F00F0271
:10C1B00012E00F4B5A6842F0F0020DE00C4B5A6847
:10C1C00042F4706208E00A4B5A6842F4704203E09D
:10C1D000074B5A6842F470225A6070476C00024064
:10C1E000440002401C04024044040240000002409B
:10C1F000000402408A6870B50C6A0B6944EA0202C6
:10C200004C691A438B692243CC6905684E6A42EA3D
:10C21000030323438C6A334325F4FE4C23432CF061
:10C22000F00C43EA0C030360CB6843600B68836047
:10C230004B68C36070BD00BF00238362036043602E
:10C240008360C360036143618361C36103624362CE
:10C25000704700BF19B1036843F0010302E00368AF
:10C2600023F001030360704712B10368194302E031
:10C27000036823EA01010160704700BF406880B293
:10C28000704700BF10F0805F14BF044B044B1B6865
:10C2900003420CBF00200120704700BF0004024091
:10C2A0000000024010F0805F14BF024B024B586048
:10C2B000704700BF000402400000024010F0805FA1
:10C2C00014BF044B044B1B6803420CBF0020012029
:10C2D000704700BF000402400000024010F0805F81
:10C2E00014BF024B024B5860704700BF000402406D
:10C2F00000000240044B00221A605A609A60DA6023
:10C30000024A5A61704700BF00040140FFFF070066
:10C31000837930B5016802794BB3184BCC431D6863
:10C3200090F805C004EA05051D605D682C405C605E
:10C33000D45844EA0101D15002689868D14301EA17
:10C3400000009860D8680140BCF1100FD96007D197
:10C35000996811439960D96841EA0202DA600BE0FA
:10C360005CF8031041EA02024CF8032004E0034B9E
:10C37000D05820EA0101D15030BD00BF0004014077
:10C3800000230C228371427103600371704700BF68
:10C39000024B1A6940EA02021A6170470004014028
:10C3A000034B5B6918420CBF00200120704700BF9F
:10C3B00000040140014B5861704700BF0004014078
:10C3C000054B1A685B69034001D1184603E010422F
:10C3D0000CBF00200120704700040140014B586150
:10C3E000704700BF00040140044B1A6802F0380295
:10C3F0001A601A6840EA02021A6070470020024080
:10C40000044B1A6822F008021A601A6840EA020215
:10C410001A60704700200240044B1A6822F0100294
:10C420001A601A6840EA02021A607047002002404F
:10C43000034B044A5A6002F188325A60704700BFC9
:10C440000020024023016745024B1A6942F0800236
:10C450001A61704700200240014BD869800870477C
:10C4600000200240014B186A704700BF00200240C4
:10C47000024BD869C0F34000704700BF0020024063
:10C48000024B1868C0F34010704700BF0020024004
:10C4900019B1054B1A69104303E0034B1A6922EAEC
:10C4A00000001861704700BF00200240012804D13D
:10C4B000054BD86900F0010005E0034BDB6818422A
:10C4C0000CBF00200120704700200240014BD860C3
:10C4D000704700BF00200240094BDA6812F0010FDC
:10C4E00001D001200BE0DA6812F0040F01D0022025
:10C4F00005E0DB6813F0100F14BF03200420704721
:10C500000020024013B504460AE000230193FF33E4
:10C5100001E0019B013B0193019B002BF9D1013C00
:10C52000FFF7DAFF012802D1002CEED100E004B9B8
:10C5300005201CBDF8B5124C124B0546A36003F153
:10C5400088330F20A3600E461746FFF7DBFF042851
:10C5500014D1236945F0F80543F0100323612E43FD
:10C56000094B37430B305F80FFF7CCFF012805D024
:10C57000226941F6EF7302EA03032361F8BD00BFAD
:10C58000002002402301674500F8FF1F38B505462B
:10C5900040F6FF70FFF7B6FF04283CD11E4C1F4B3E
:10C5A00040F6FF70A36003F18833A360236943F072
:10C5B00020032361236943F040032361FFF7A2FFB7
:10C5C000042820D1226941F6DF7302EA03032361C4
:10C5D000236943F0100323611DB1114B4FF000029A
:10C5E00002E00F4B4FF0A5021A8040F6FF70FFF7F4
:10C5F00089FF01280FD0084A41F6EF73116901EA5B
:10C600000303136107E0012805D0226941F6DF73B7
:10C6100002EA0303236138BD00200240230167457D
:10C6200000F8FF1F10B504460F20FFF76BFF04282A
:10C630003DD11F4A1F4BE443936003F1883393605D
:10C640001169E3B241F01001FF2B116106D01A4AC3
:10C650000B301381FFF756FF04281FD1C4F30723C3
:10C66000FF2B06D0144A0F205381FFF74BFF0428FD
:10C6700014D1C4F30743FF2B06D00F4A0F20938138
:10C68000FFF740FF042809D1240EFF2C01D104201C
:10C6900006E0094B0F20DC81FFF734FF012806D0AC
:10C6A000034A41F6EF73116901EA0303136110BDF8
:10C6B000002002402301674500F8FF1F70B50446C3
:10C6C0000F200E46FFF71EFF042815D10B4D0C4B13
:10C6D0000B30AB6003F18833AB602B6943F0100380
:10C6E0002B612680FFF70EFF012805D02A6941F64D
:10C6F000EF7302EA03032B6170BD00BF002002400C
:10C700002301674570B504460F200E46FFF7FAFE79
:10C71000042810D1084D0B302B6943F001032B6125
:10C720002680FFF7EFFE012805D02A6941F6FE7347
:10C7300002EA03032B6170BD0020024070B504467D
:10C740000F200E46FFF7DEFE042818D10C4DB3B2C1
:10C750002A690B3042F001022A612380FFF7D2FEE2
:10C76000042804D1360C66800B30FFF7CBFE01287D
:10C7700005D02A6941F6FE7302EA03032B6170BDFE
:10C780000020024010B540F6FF70FFF7BBFE042802
:10C790002CD1174C174B40F6FF70A36003F1883380
:10C7A000A360236943F020032361236943F040031E
:10C7B0002361FFF7A7FE042810D1226941F6DF7339
:10C7C00002EA0303236123694FF0A50243F010033B
:10C7D0002361094B0B301A80FFF794FE012805D026
:10C7E000226941F6EF7302EA0303236110BD00BF23
:10C7F000002002402301674500F8FF1F10B540F6F6
:10C80000FF70FFF77FFE042814D10B4C40F6FF7039
:10C81000236943F004032361236943F04003236148
:10C82000FFF770FE012805D0226941F6FB7302EA8A
:10C830000303236110BD00BF0020024038B5054648
:10C8400040F6FF70FFF75EFE042815D10B4C40F652
:10C85000FF70236943F0020323616561236943F09C
:10C8600040032361FFF74EFE012805D0226941F6FF
:10C87000FD7302EA0303236138BD00BF00200240BC
:10C88000CB78F0B513F0100F18BF8A78098803F041
:10C890000F0C18BF4CEA020C11F0FF0F1AD00468FD
:10C8A00000220126964006EA0105B5420ED1960007
:10C8B0000F27B7400CFA06F624EA07043443282B66
:10C8C00001D1456102E0482B08BF05610132082A09
:10C8D000E7D10460FF291CD94468002202F1080551
:10C8E0000126AE4006EA0105B5420ED196000F279B
:10C8F000B7400CFA06F624EA07043443282B01D18A
:10C90000456102E0482B08BF05610132082AE5D1E4
:10C910004460F0BD0423C370022383704FF0FF33E3
:10C9200003807047836819420CBF002001207047C4
:10C93000806880B2704700BFC36819420CBF0020F6
:10C9400001207047C06880B2704700BF0161704726
:10C95000416170470AB1016100E04161704700BF69
:10C96000C160704741F48033836181618361836971
:10C9700083697047064A10B514684FF6807341EA20
:10C98000001104EA030341EA0303136010BD00BF72
:10C9900000000140014B1860704700BF1C0020429E
:10C9A0000304154A00F4401C1B0CBCF5401F30B5B5
:10C9B000546806D1556824F0706425F070655560A0
:10C9C00011E010F4801F06D0C0F303424FF0030CB7
:10C9D0000CFA02F203E0420D120113FA02F224EA09
:10C9E000020444F0706419B1400D000183401C43FF
:10C9F000014B5C6030BD00BF0000014001F003034B
:10CA00009B000F229A4010FA03F310B58908074CD7
:10CA1000023154F8210020EA020244F8212054F89F
:10CA20002120134344F8213010BD00BF0000014015
:10CA30000120014608B500F047FB0120002100F06D
:10CA400043FB08BD08B5264B98422BD00CD8A3F564
:10CA5000006398421AD003F5806398421CD0A3F576
:10CA6000006398423AD10BE01E4B984226D003F562
:10CA70008063984228D0A3F5006398422ED117E036
:10CA80000420012100F020FB042024E008200121E3
:10CA900000F01AFB08201EE01020012100F014FB1A
:10CAA000102018E02020012100F00EFB202012E0D1
:10CAB0004020012100F008FB40200CE080200121F3
:10CAC00000F002FB802006E04FF48070012100F0AE
:10CAD000FBFA4FF48070002100F0F6FA08BD00BFA9
:10CAE00000140140001C01400B4B4FF0FF316FF070
:10CAF0007042C3F88010C3F88420C3F88011C3F8D3
:10CB00008421002303F1C001034A013300200F2BCD
:10CB100042F82100F6D1704700E100E0094B4FF0E8
:10CB200020605860084800224FF0FF319A60D860BA
:10CB30001A615A619A61DA611A625A629962D9621B
:10CB40001963704700ED00E00000FA0540F0BE6098
:10CB5000024B40F42020D860704700BF00ED00E099
:10CB600030B5C27803787AB31C4A4178D2684FF066
:10CB70000F0CD243C2F302222CFA02FCC2F10402CF
:10CB80009140807803F003020CEA000C4CEA010C9F
:10CB9000D2004FEA0C1CFF2090400CFA02FC01244A
:10CBA00003F01F02944099080D4AC03152F82150F9
:10CBB0000CEA000C25EA00004CEA00005B0942F890
:10CBC000210042F8234008E003F01F0201219140B8
:10CBD0005B09034A203342F8231030BD00ED00E02A
:10CBE00000E100E00023C37003704370837070475E
:10CBF000024B5868C0F30930704700BF00ED00E0F9
:10CC0000012200F01F0312FA03F34009044A4030E6
:10CC100052F820001840984214BF002001207047AD
:10CC200000E100E0014B1860704700BF00EF00E03A
:10CC300000F01F0301229A404009024B603043F884
:10CC40002020704700E100E0024B58688005800D0D
:10CC5000704700BF00ED00E0012200F01F0312FA50
:10CC600003F34009044A803052F8200018409842EB
:10CC700014BF00200120704700E100E0014B18685C
:10CC8000704700BF00ED00E021F0604121F07F011E
:10CC9000014B01439960704700ED00E0014A024BEF
:10CCA000DA6070470400FA0500ED00E0014A024B2B
:10CCB000DA6070470100FA0500ED00E019B1054B9C
:10CCC0001A69104303E0034B1A6922EA0000186155
:10CCD000704700BF00ED00E000F01F00012313FAD1
:10CCE00000F019B1044B5A6A104303E0024B5A6A30
:10CCF00022EA00005862704700ED00E0144B70B566
:10CD0000DC684FF0FF0CE443C4F302242CFA04F572
:10CD1000C4F1040411FA04F4C0F30126F6000CFA7D
:10CD200006FC02EA050545EA0404240114FA06F6A5
:10CD3000C0F38110063053F8202022EA0C0243F899
:10CD4000202053F82020164343F8206070BD00BF18
:10CD500000ED00E0C0F3832001238340044A506AC1
:10CD600003EA0000984214BF00200120704700BF72
:10CD700000ED00E000F01F0001228240024B5968E4
:10CD80000A435A60704700BF00ED00E000F01F0248
:10CD90000123013A13FA02F2024B59680A435A601E
:10CDA000704700BF00ED00E0C0F3833001238340F3
:10CDB000044A506A03EA0000984214BF0020012090
:10CDC000704700BF00ED00E0C0F3814313B90A4B88
:10CDD000D86A10E0012B0CD1074AC0F30153906AC6
:10CDE000DA00D040022B14BF00F00F0000F0FF006B
:10CDF00001E0014B186B704700ED00E010F4800F6C
:10CE00000BBF024B014B586B986B704700ED00E075
:10CE100008B5F7F7ADF908BD08B50001F7F7A5F9B2
:10CE200008BD00BF08B5F7F79EF908BD08B5F7F7CC
:10CE300098F908BD08B5F7F792F908BD08B5F7F7F6
:10CE40008CF908BD0D4B0E4A196841F001011960BB
:10CE5000596801EA02025A601A6822F0847222F4C8
:10CE600080321A601A6822F480221A605A6822F40A
:10CE7000FE025A6000229A60704700BF0010024014
:10CE80000000FFF80C4BB0F5803F1A6822F48032A6
:10CE90001A601A6822F480221A6003D0B0F5802F3D
:10CEA00008D103E01A6842F4803202E01A6842F4C2
:10CEB000A0221A60704700BF00100240034B1A689E
:10CEC00022F0F80242EAC0021A60704700100240E5
:10CED000014B1860704700BF00004242044B5A6883
:10CEE00022F47C1240EA02020A435A60704700BFF3
:10CEF00000100240014B1860704700BF60004242C2
:10CF0000034B5A6822F0030240EA02025A6070475B
:10CF100000100240024B586800F00C00704700BF40
:10CF200000100240034B5A6822F0F00240EA02026D
:10CF30005A60704700100240034B5A6822F4E062C6
:10CF400040EA02025A60704700100240034B5A68E0
:10CF500022F4605242EAC0025A6070470010024058
:10CF600019B1054B1A78104303E0034B1A7822EAF3
:10CF700000001870704700BF09100240014B186094
:10CF8000704700BFD8004242034B5A6822F4404227
:10CF900040EA02025A60704700100240064B00222D
:10CFA00001281A701A7002D0042804D101E0187008
:10CFB00001E005221A70704720100240014B1860F2
:10CFC000704700BF80044242024B1A6A40EA0202E4
:10CFD0001A62704700100240014B1860704700BF92
:10CFE0003C0442421F4B10B55A6802F00C02042A5E
:10CFF00013D0082A11D15A685968C2F38342023209
:10D0000011F4803F03D05B6813F4003F01D0164B4E
:10D0100000E0164B5A43026001E0144B0360114AD2
:10D02000134B51680468C1F30311595C34FA01F1E0
:10D0300041605468C4F3022C13F80C4031FA04F434
:10D0400084605468C4F3C22C13F80CC021FA0CF1AC
:10D05000C1605268C2F381329B181B7CB1FBF3F1B3
:10D06000016110BD0010024000093D0000127A006D
:10D07000B819010819B1054B5A69104303E0034B75
:10D080005A6922EA00005861704700BF0010024050
:10D0900019B1054B9A69104303E0034B9A6922EAE0
:10D0A00000009861704700BF0010024019B1054BA5
:10D0B000DA69104303E0034BDA6922EA0000D86121
:10D0C000704700BF0010024019B1054BDA681043E9
:10D0D00003E0034BDA6822EA0000D860704700BF23
:10D0E0000010024019B1054B1A69104303E0034BCD
:10D0F0001A6922EA00001861704700BF0010024060
:10D10000014B1860704700BF40044242014B186059
:10D11000704700BF4C004242014B1870704700BF7F
:10D12000071002404309012B02D1084B1B6805E0A0
:10D13000022B0BBF054B054B1B6A5B6A00F01F00FF
:10D1400033FA00F000F00100704700BF0010024009
:10D1500008B53120FFF7E6FF094B18705A68013215
:10D160005A601A7822B95A6840F2FF139A42F0D1F5
:10D170003120FFF7D7FF003818BF012008BD00BFDE
:10D18000D4060020024B5A6A42F080725A627047FD
:10D1900000100240034B9B6818420CBF0020012086
:10D1A000704700BF00100240014B1870704700BF6D
:10D1B0000A1002400B884A88B1F804C01A43CB8891
:10D1C00042EA0C02B1F808C01A434B8930B542EA72
:10D1D0000C028D89B0F800C0CC891A432A4322433F
:10D1E0000CF4415313439BB20380838B23F40063FD
:10D1F0001B041B0C83830B8A038230BD00234FF07A
:10D200000702C3810282038043808380C38003813D
:10D2100043818381704700BF0023438103804380A3
:10D220008380C3804FF002030381704721B10388DC
:10D230009BB243F0400304E0038823F040031B0447
:10D240001B0C0380704700BF21B1838B9BB243F45A
:10D25000806304E0838B23F480631B041B0C8383B3
:10D26000704700BF0909012313FA01F189B21AB10D
:10D2700083889BB2194303E083889BB223EA0101B0
:10D28000818070471AB183889BB2194303E0838879
:10D290009BB223EA01018180704700BF8181704702
:10D2A000808980B2704700BF4FF6FF63994205D076
:10D2B00003889BB243F48073038002E00388194023
:10D2C0000180704721B183889BB243F0040304E0DE
:10D2D000838823F004031B041B0C8380704700BF6A
:10D2E000038823F400631B041B0C038003889BB298
:10D2F00041EA03030380704703889BB243F48053E1
:10D300000380704721B103889BB243F4005304E0CB
:10D31000038823F400531B041B0C0380704700BFD9
:10D32000012914BF008B808A80B27047008A80B2C6
:10D33000704700BFB1F5804F04D103889BB243F41E
:10D34000804304E0038823F480431B041B0C038008
:10D35000704700BF038919420CBF002001207047AD
:10D36000202906D1038903889BB243F04003038040
:10D3700008E0402901D0082901D1038902E0C9430E
:10D3800089B20181704700BF012301F00F0213FA37
:10D3900002F2B0F804C000891FFA8CFC80B2104081
:10D3A00006D009098B401CEA030F0CBF00200120A6
:10D3B000704700BF552906D1038903889BB243F00B
:10D3C000400303800DE0562901D0532901D1038980
:10D3D00007E001F00F01012313FA01F1C94389B2FB
:10D3E00001817047838BF0B523F47A6323F01F0328
:10D3F0001B041B0C83834FF0020303840B89868B71
:10D40000022B87B004460D46B6B201D1002225E0BA
:10D4100001A88F88FFF7E6FDEB88002F0CBF0127DE
:10D420000227B3F5007F2989019A06D1A3F5FB7382
:10D4300053430902B3FBF1F305E00A2349015A43C0
:10D440004F43B2FBF7F305330A229BB2B3FBF2F36F
:10D4500003F001021202C3F34F0392B2991E89B284
:10D46000FE2928BF002228BF0223E98842EA0303DD
:10D470000B439BB223842B886A8846EA0303A9885E
:10D4800043F4006313436A890B4313439BB2A383A2
:10D4900007B0F0BD08B5154B98421BD003F5744397
:10D4A000984204D0A3F5784398421DD10AE00121A7
:10D4B0004FF48050FFF708FE4FF480500021FFF733
:10D4C00003FE11E04FF480400121FFF70BFE4FF403
:10D4D000804006E04FF400400121FFF703FE4FF4C7
:10D4E00000400021FFF7FEFD08BD00BF003C0040EA
:10D4F000042804D1054B1A6842F0040203E0034BF0
:10D500001A6822F004021A60704700BF10E000E0C1
:10D51000014B5860704700BF10E000E0012804D1C3
:10D52000084B1A6842F0010206E010F1020F05D123
:10D53000044B1A6822F001021A6002E0014B00223B
:10D540009A60704710E000E020B1054B1A6842F085
:10D55000020203E0024B1A6822F002021A607047CE
:10D5600010E000E0014B9868704700BF10E000E059
:10D57000C308022B0BBF044B034B1B68DB6833FA59
:10D5800000F000F00100704710E000E0038803F0B5
:10D590008F0303800388B1F806C04A889BB243EA30
:10D5A0000C0313439BB203808B8883850B88038510
:10D5B000064B984203D003F50063984201D10B7AE1
:10D5C00003864FF001038382704700BF002C0140A7
:10D5D000038C2DE9F04123F001031B041B0C038491
:10D5E000038C0A894C8823F002031C4E14431B044D
:10D5F0008288B1F806C0058B1B0CA4B2B04244EA85
:10D60000030392B20C88ADB2A0F834C003D006F583
:10D610000066B04218D18E894F89B1F80E804FF65E
:10D62000F77C03EA0C0C4CEA070748EA06064FF6BB
:10D63000FB73898847F6FF4C02EA0C0C07EA0303E8
:10D64000B2B20B4342EA0C024FF68F7105EA0101B8
:10D650002143828001830384BDE8F081002C0140D6
:10D66000038C2DE9F04123F010031B041B0C0384F1
:10D67000028CB1F808C022F0200212048488120C37
:10D680004B8842EA0C1242EA0313A2B21B4C068BEF
:10D69000B1F806C0A0420D88B6B29BB2A0F838C05F
:10D6A00003D004F50064A0421BD1B1F80A804FF604
:10D6B0007F748F8903EA040447F2FF3C02EA0C0CF2
:10D6C00044EA0814CA894FF6BF73898804EA030341
:10D6D0004CEA870C43EA01134CEA82023C469BB2B7
:10D6E00092B248F6FF7106EA010141EA052189B2CA
:10D6F000828001830384BDE8F08100BF002C0140DB
:10D70000038C2DE9F04123F480731B041B0C03846C
:10D71000028CB1F808C022F4007212048488120C42
:10D720004B8842EA0C2242EA0323A2B21A4C868BAF
:10D73000B1F806C0A0420D88B6B29BB2A0F83CC0BA
:10D7400003D004F50064A0421BD1B1F80A804FF267
:10D75000FF748F8903EA040444F6FF7C02EA0C0C90
:10D7600044EA0824CA894FF6FF33898804EA030390
:10D770004CEA071C43EA01234CEA02123C469BB2E6
:10D7800092B24FF68F7106EA0101294382808183AC
:10D790000384BDE8F08100BF002C0140038CF0B58C
:10D7A00023F480531B041B0C0384B1F806C0078CC0
:10D7B0000C8882880D89868B4B88A0F840C0DFF8E2
:10D7C00048C0BFB2604592B2B6B203D00CF5006C4F
:10D7D000604505D192048989920C42EA811292B285
:10D7E0004DF6FF7C07EA0C0C48F6FF7106EA0101D2
:10D7F0004CEA053C41EA04214CEA033389B29BB26E
:10D80000828081830384F0BD002C0140B1F802C006
:10D810000B888A884CEA0303B1F806C013430A89CF
:10D8200043EA0C03B1F80AC013438A8943EA0C03A4
:10D8300013439BB2A0F84430704700BF00234FF061
:10D84000FF320372438082800380C380704700BF31
:10D850000023C381038043808380C380038143818D
:10D860008381704700234FF00102038103804380CE
:10D870008280C380704700BF002383810380438080
:10D880008380C38003814381704700BF21B1038837
:10D890009BB243F0010304E0038823F001039B05DE
:10D8A0009B0D0380704700BF39B1B0F844306FEA78
:10D8B00043436FEA53439BB203E0B0F844305B0448
:10D8C0005B0CA0F8443070471AB183899BB21943AE
:10D8D00003E083899BB223EA01018181704700BF85
:10D8E000818270470A43A0F8482070471AB18389A3
:10D8F0009BB2194303E083899BB223EA0101818132
:10D90000704700BF038923F007031B041B0C03812E
:10D91000704700BFB0F808C05FFA8CFC41EA0C0CFD
:10D9200042EA0C0C4CEA032C1FFA8CFCA0F808C04D
:10D93000704700BF10B50446FFF7ECFF23899BB288
:10D9400043F48043238110BD10B50446FFF7E2FF86
:10D95000238923F077031B041B0C43F077032381F7
:10D9600010BD00BF01858282704700BF038823F08D
:10D9700070039B059B0D41EA03030380704700BFC2
:10D98000038923F070031B041B0C41EA030303818A
:10D99000704700BF10B50446FFF7F2FF23899BB222
:10D9A00043F00703238110BD30B50489B0F818C0D7
:10D9B000058C2CF4407CADB22CF0030C24F0070451
:10D9C0004FEA0C4C25F0220542EA050524044FEAF3
:10D9D0001C4C45EA0315240C4CF4807C21434CF08C
:10D9E000010CADB20181A0F818C0058430BD00BFA4
:10D9F000038B23F070031B041B0C41EA0303038316
:10DA0000704700BF038B23F4E0431B041B0C43EA65
:10DA100001239BB203837047838B23F070031B04A5
:10DA20001B0C41EA03038383704700BF838B23F4FD
:10DA3000E0431B041B0C43EA01239BB28383704722
:10DA400021B103889BB243F0800304E0038823F0F4
:10DA500080039B059B0D0380704700BF21B1838825
:10DA60009BB243F0040304E0838823F004031B0407
:10DA70001B0C8380704700BF21B183889BB243F0A9
:10DA8000080304E0838823F008031B041B0C838035
:10DA9000704700BF21B183889BB243F0010304E0CB
:10DAA000838823F001031B041B0C8380704700BF95
:10DAB000038B23F008031B041B0C41EA03030383BD
:10DAC000704700BF038B23F400631B041B0C43EA65
:10DAD00001239BB203837047838B23F008031B044D
:10DAE0001B0C41EA03038383704700BF838B23F43D
:10DAF00000631B041B0C43EA01239BB28383704722
:10DB0000038B23F004031B041B0C41EA0303038370
:10DB1000704700BF038B23F480631B041B0C43EA94
:10DB200001239BB203837047838B23F004031B0400
:10DB30001B0C41EA03038383704700BF838B23F4EC
:10DB400080631B041B0C43EA01239BB28383704751
:10DB5000038B23F080031B041B0C41EA03030383A4
:10DB6000704700BF038B5B045B0C43EA01239BB24D
:10DB700003837047838B23F080031B041B0C41EA53
:10DB800003038383704700BF838B5B045B0C43EA12
:10DB900001239BB283837047038C23F002031B0491
:10DBA0001B0C41EA03030384704700BF038C23F07E
:10DBB00008031B041B0C41EA03030384704700BFE6
:10DBC000038C23F020031B041B0C43EA01139BB2BC
:10DBD00003847047038C23F080031B041B0C43EA6F
:10DBE00001139BB203847047038C23F400731B045E
:10DBF0001B0C43EA01239BB203847047038C23F47C
:10DC000000631B041B0C43EA01239BB2038470478F
:10DC1000038C23F400531B041B0C43EA01339BB217
:10DC20000384704701238B408A40018C89B221EA2A
:10DC300003030384018C0A4392B20284704700BF3D
:10DC400004238B408A40018C89B221EA03030384B8
:10DC5000018C0A4392B20284704700BF01238B40BB
:10DC6000B0F820C010B51FFA8CFC2CEA0303038423
:10DC700009B1082909D11830490844584FF68F7363
:10DC800004EA0303435043580CE004391830C1F34D
:10DC90004E01445848F6FF7304EA0303435012024E
:10DCA000435892B243EA0202425010BD21B10388A8
:10DCB0009BB243F0020304E0038823F002039B05B8
:10DCC0009B0D0380704700BF21B103889BB243F0D6
:10DCD000040304E0038823F004039B059B0D0380E9
:10DCE000704700BF21B183889BB243F0800304E0FA
:10DCF000838823F080031B041B0C8380704700BFC4
:10DD0000038823F008039B059B0D038003889BB2C7
:10DD100041EA030303807047838823F070031B04E8
:10DD20001B0C838083889BB241EA03038380704786
:10DD3000038923F007031B041B0C038103899BB297
:10DD400041EA030303817047038923F080031B0426
:10DD50001B0C038103899BB241EA030303817047D3
:10DD6000818470478185704781867047018770473D
:10DD700081877047A0F84010704700BF038B23F0E5
:10DD80000C031B041B0C0383038B9BB241EA0303AC
:10DD900003837047038B23F440631B041B0C038332
:10DDA000038B9BB243EA01239BB20383704700BFFE
:10DDB000838B23F00C031B041B0C8383838B9BB28C
:10DDC00041EA030383837047838B23F440631B047E
:10DDD0001B0C8383838B9BB243EA01239BB2838317
:10DDE000704700BF0388DBB2038003889BB241EA1F
:10DDF00003030380704700BF808E80B2704700BF6E
:10DE0000008F80B2704700BF808F80B2704700BF24
:10DE1000B0F8400080B27047808C80B2704700BF7D
:10DE2000008D80B2704700BF038A19420CBF0020EA
:10DE300001207047C94389B201827047038A8289F1
:10DE400011EA030092B203D011420CBF002001205E
:10DE5000704700BFC94389B201827047B0F820C043
:10DE600010B52CF0010C4FEA0C4C4FEA1C4CA0F8FA
:10DE700020C0048BB0F820C0A4B21FFA8CFC24F0A0
:10DE8000F30442EA04042CF0020C44EA03144CF0BC
:10DE9000010C4CEA010CA4B20483A0F820C010BD10
:10DEA000B0F820C010B52CF0100C4FEA0C4C4FEA23
:10DEB0001C4CA0F820C0B0F818C0048C2CF4407C96
:10DEC000A4B24FEA0C5C4FEA1C5C24F020044CEA3C
:10DED000022C44F010044CEA033C44EA01141FFAFB
:10DEE0008CFCA4B2A0F818C0048410BD38B50D464F
:10DEF000602D1146044603D10122FFF7D1FF02E055
:10DF00000122FFF7ABFF29462046FFF739FD2389A1
:10DF10009BB243F00703238138BD00BFF8B50C4620
:10DF2000A2884988B4F800C0054600290CBF022722
:10DF30000027012A0CBF022601262389BCF1000F0D
:10DF400010D1FFF78BFF2846E188FFF717FF28461F
:10DF5000394632462389FFF7A3FF2846E188FFF7B9
:10DF600019FF0FE0FFF79CFF2846E188FFF712FF3B
:10DF70002846394632462389FFF770FF2846E18854
:10DF8000FFF7FCFEF8BD00BF38B50B880C46054610
:10DF90004BB94988A2882389FFF760FF2846E188AA
:10DFA000FFF7ECFE53E0042B09D14988A2882389AE
:10DFB000FFF776FF2846E188FFF7ECFE47E0082BE5
:10DFC000B1F802C0B1F804E0098920D1028C22F432
:10DFD00080721204120C0284838B028C9BB292B268
:10DFE00023F0F30322F4007243EA011142EA0C2CFD
:10DFF00089B21FFA8CFC41EA0E0E4CF4807CA0F82A
:10E000001CE0A0F820C0E188FFF7D2FE1FE0028CE0
:10E0100022F480521204120C0284838B028C23F4AB
:10E02000407392B21B051B0D22F4005243EA0E23EB
:10E0300042EA0C3C43EA01331FFA8CFC9BB24CF4DD
:10E04000805C8383A0F820C0E188FFF7BDFE38BD67
:10E0500008B52D4B984237D00BD8A3F500639842F2
:10E0600026D003F58063984228D0B0F1804F4AD182
:10E0700018E0264B984233D004D8A3F58063984229
:10E0800041D127E0224B984204D003F50063984227
:10E0900039D12EE04FF400600121FFF715F84FF45D
:10E0A00000602DE001200146FFF71CF801201CE074
:10E0B00002200121FFF716F8022016E004200121BA
:10E0C000FFF710F8042010E008200121FFF70AF8FC
:10E0D00008200AE010200121FFF704F8102004E0D6
:10E0E00020200121FEF7FEFF20200021FEF7FAFF8D
:10E0F00009E04FF400500121FEF7E6FF4FF4005015
:10E100000021FEF7E1FF08BD000C004000140040B4
:10E11000002C0140002383814FF416528380C3807A
:10E1200003814FF00C030260438170470A8810B5E9
:10E130004C88B1F804C0038AC98844EA020242EA62
:10E140000C0223F470630A431B041B0C92B242EAD4
:10E150000303038210BD00BF0023C38003804380FC
:10E160008380704721B183899BB243F4005304E05C
:10E17000838923F400531B041B0C8381704700BF69
:10E1800001F01F034FF0010CC1F3421161450CFA7D
:10E1900003F301D10C3004E0022901D1103000E07A
:10E1A00014301AB1026842EA030302E0026822EA6C
:10E1B00003030360704700BF1AB1838A9BB21943FF
:10E1C00003E0838A9BB223EA01018182704700BF8A
:10E1D000038A23F00F031B041B0C0382038A9BB2E8
:10E1E00041EA030303827047838923F400631B041D
:10E1F0001B0C838183899BB241EA030383817047AF
:10E2000021B183899BB243F0020304E0838923F0A8
:10E2100002031B041B0C8381704700BF038A23F099
:10E2200020031B041B0C0382038A9BB241EA0303F5
:10E230000382704721B1038A9BB243F4804304E018
:10E24000038A23F480431B041B0C0382704700BF26
:10E25000C905C90D818070478088C005C00D704711
:10E2600083899BB243F0010383817047038BDBB248
:10E270000383038B9BB243EA01230383704700BFF0
:10E28000038B03F47F430383038B9BB241EA0303B5
:10E290000383704721B1838A9BB243F0200304E0DB
:10E2A000838A23F020031B041B0C8382704700BF6A
:10E2B00021B1838A9BB243F0100304E0838A23F0E8
:10E2C00010031B041B0C8382704700BF21B1838A9B
:10E2D0009BB243F0080304E0838A23F008031B0485
:10E2E0001B0C8382704700BF838A23F004031B0446
:10E2F0001B0C8382838A9BB241EA030383827047AB
:10E3000021B1838A9BB243F0020304E0838A23F0A5
:10E3100002031B041B0C8382704700BF0388194251
:10E320000CBF002001207047C94389B201807047AB
:10E330004FF0010CC1F3421201F01F0362450CFAC9
:10E3400003F301D1828903E0022A0CBF028A828A88
:10E3500092B21340028892B20BB9184607E0090A3C
:10E36000012313FA01F111420CBF00200120704774
:10E37000090A01238B40DB439BB20380704700BF37
:10E38000038ACA8823F440531B041B0C13430382E3
:10E3900083898A8830B5044608890D4623F4B05332
:10E3A000498940EA020223F00C030A431B041B0CB8
:10E3B00092B242EA0303A381A38AAA8923F4407399
:10E3C0001B041B0C134387B0A38201A8FEF70AFEAF
:10E3D0000E4B2A689C420CBF049B039B1921594396
:10E3E00092006423B1FBF2F1B1FBF3F212011009C8
:10E3F00003FB101109013231B1FBF3F303F00F03FA
:10E4000043EA020292B2228107B030BD00380140D7
:10E4100008B5214B98422BD008D8A3F50063984249
:10E4200016D003F58063984234D119E01B4B984213
:10E4300026D003F5684398422CD101214FF4804047
:10E44000FEF742FE4FF480400021FEF73DFE21E042
:10E450004FF400300121FEF745FE4FF4003016E086
:10E460004FF480200121FEF73DFE4FF480200EE0A6
:10E470004FF400200121FEF735FE4FF4002006E0A6
:10E480004FF480100121FEF72DFE4FF48010002183
:10E49000FEF728FE08BD00BF004C004000500040C1
:10E4A000684620F007018D4601B5002303E00B49C3
:10E4B0005958995004330A4A0A4998188842F6D3A1
:10E4C000094B02E0002243F8042B084A9342F9D397
:10E4D000F5F756FEBDE8014085467047101B010860
:10E4E000000000203002002030020020800D0020BB
:10E4F00010B5074C20B922684FF00103138205E0E4
:10E50000044B1B681B68984720680A3010BD00BF89
:10E51000180D0020D40C002010B50A4B0A4A1B68C5
:10E520005178DA7891420AD3997841B99C8834B904
:10E530009A72064B1B685B689847204600E00220F1
:10E5400010BD00BF180D002004010020D40C0020D5
:10E5500010B5074C20B922684FF00103138205E083
:10E56000044B1B689B68984720680C3010BD00BFA7
:10E57000180D0020D40C002038B50E4C0E4B22682C
:10E580001B68D1789B695079984723689A7A7AB149
:10E5900070B91A7962B99D7855B9084B1B68DB6868
:10E5A0009847236828465979DA78D9721A7300E0B7
:10E5B000022038BD180D0020B00C0020D40C002023
:10E5C00008B50246244B20B91B684FF0020119829E
:10E5D00040E0224A4FF000011B681180197811F0C9
:10E5E0007F0113D15B7A13F0200F03D0117841F033
:10E5F0000201117013F0400F184B15BF1A781A78EA
:10E6000022F0010242F001021A701EE0012921D01D
:10E61000022901D000221DE0597911F0800F01F08C
:10E620000F0306D00E4951F8233003F03003102BAE
:10E6300006E00B4951F8233003F44053B3F5805FF3
:10E6400003D1137843F001031370064B1B681B6959
:10E650009847024A104608BD180D0020780D00208A
:10E66000005C0040D40C002010B51E4B19684A799C
:10E6700012F0800F22F0800305D01B4850F82300D1
:10E6800000F0300004E0184850F8230000F4405037
:10E69000164C94F800C0634522D24C8804BBF8B1F4
:10E6A000897AE9B112F0800F09D00F4948F6BF729C
:10E6B00051F8230000EA020282F0100208E00A4941
:10E6C0004BF68F7251F8230000EA020282F4805266
:10E6D00041F82320064B1B689B699847002000E007
:10E6E000022010BD180D0020005C00400401002035
:10E6F000D40C002008B5064B1B685A7A42F0200261
:10E700005A72044B1B68DB699847002008BD00BFA4
:10E71000180D0020D40C0020054B1A68538A18B934
:10E720008988CB1A138201E008681818704700BF67
:10E73000180D002030B50E4B1C78002310E05FFA56
:10E7400083FC4FEA8C0202F1804202F5B842156860
:10E7500048F68F7105EA010141EA0C0111600133AD
:10E76000A342ECD3034B40F08000186030BD00BFE3
:10E77000040100204C5C0040704700BF08B50C4B02
:10E78000002093F82C1000F04FFE0A4B1B68187AFB
:10E79000082807D1084B4FF480521A80074B4FF0DE
:10E7A00010021A80092814BF0020012008BD00BFF4
:10E7B00080000020180D00207A0D00207C0D002024
:10E7C00070B52D4B1C68237A032B01D0052B46D145
:10E7D000A369228AABB1A2B1A58A954228BF15468A
:10E7E00028469847228A638A521BEB1806462282E3
:10E7F0006382002000F0E8FD2A460146304600F022
:10E80000FBFB238A5BB11D4B4FF4405200201A8062
:10E81000014600F0E7FD1A4B4FF030021A80A28A41
:10E82000238A9A4203D8144B03221B6803E0124A3E
:10E830001BB1136805221A720DE0126806211172CD
:10E84000104A1168104A89B28A18520013600C4BA2
:10E850004FF030021A80084B1B681B7A06E0072B2A
:10E8600003D10A4B1B68DB6898470823024A1268E9
:10E870001372FFF783FF70BD180D00207A0D002082
:10E880007C0D0020505C004002300020B00C0020C5
:10E89000F8B5244B1C68238A267ABBB9042E15D1FF
:10E8A000214822490278012A0BD1214C214A2468AF
:10E8B0000370A0B28218520013604FF030020A8039
:10E8C0002BE04FF010030B80072626E0A68AA269F2
:10E8D0009E4234BF35461D462846B34294BF0426A7
:10E8E000022690470746002000F060FD2A460146B8
:10E8F000384600F069FB2946002000F073FD638A6A
:10E90000228AEB186382094B551B4FF03002258297
:10E910001A80094B4FF440521A80024B1B681E723A
:10E92000F8BD00BF180D0020DC0600207C0D002083
:10E93000505C0040023000207A0D002008B5144BD6
:10E940001B681A7A022A01D0042A05D1FFF7A0FF1A
:10E950000F4B1B681B7A14E0062A11D15A78052A3E
:10E960000AD11A7812F07F0F06D1D878FFF7E2FEAD
:10E97000084B1B681B6A9847074B1B689B689847A6
:10E980000823034A12681372FFF7F8FE08BD00BFA0
:10E99000180D0020D40C0020B00C002038B5324BEC
:10E9A0001B68187810F07F0004D15A7A22F02002F8
:10E9B0005A7258E0022855D15A88002A52D11A7941
:10E9C000002A4FD15A7912F0800F22F0800405D02E
:10E9D000264951F8241001F0300104E0234951F890
:10E9E000241001F440512248007884423AD2002990
:10E9F00038D09B7A002B35D012F0800F0FD01B4BF4
:10EA000053F8243003F03003102B25D1E4B2204614
:10EA100000F082FC2046302100F05EFB1CE0134D2C
:10EA200055F8243003F44053B3F5805F14D134B962
:10EA3000104B204693F82C1000F0F6FC02E0204624
:10EA400000F056FC55F824204BF68F7302EA0303BE
:10EA500083F4405345F82430074B1B685B699847A3
:10EA6000002000E0022038BD180D0020005C0040AE
:10EA70000401002080000020D40C0020F7B58D4B4D
:10EA80008D4E1A6835688D4B92B2D3182A7A5B0086
:10EA9000092A1B681BD09BB203F1005303F54053B6
:10EAA0005B001C4614F8012B03F10A072A705B78FF
:10EAB0006B70B4F8030000F063FE6880B4F80700E0
:10EAC000346800F05DFEA08033687F88DF807A4C78
:10EAD00001212368DA8819725D78002A62D11A78D8
:10EAE00012F07F022ED1092D02D1FFF715FD3BE078
:10EAF000052D0DD193F90320002A4EDB9A78002AC8
:10EB00004BD19A88002A48D19B7A002B37D044E019
:10EB1000032D0BD1DA78012A27D19A882ABB5B7A98
:10EB200013F0200F21D0FFF7E5FD1DE0012D1CD1D2
:10EB3000DA78012A19D19A88BAB95B7A13F0200FD2
:10EB400013D00AE0012A04D10B2D0ED1FFF714FDDA
:10EB50000AE0022A09D1012D02D1FFF71FFF03E0CD
:10EB6000032D02D1FFF780FD48B1554B28461B68A5
:10EB70005B699847032801D109230FE068B94D4A22
:10EB8000504B12684FF0300192B2D3185B00002254
:10EB90001A604D4B1980062300E00823464A12688C
:10EBA0001372E3E0062D18D11A7812F07F0F40F0AF
:10EBB00097809B78012B03D1414B1B68DB696EE08A
:10EBC000022B03D13E4B1B681B6A68E0032B40F00D
:10EBD00087803B4B1B685B6A61E0002D3CD1598804
:10EBE00000297DD15A6822F47F42B2F5003F77D1E7
:10EBF0001A7812F07F0203D19B88002B70D129E094
:10EC0000012A0BD158792E4B1B689B699847002825
:10EC100066D123689B7A002B62D01BE0022A5FD169
:10EC20005B7913F0800F03F00F0205D0274951F8EC
:10EC3000221001F0300104E0244951F8221001F4BF
:10EC400040512348007882424AD213F0700F47D1D6
:10EC5000002945D01F4B23E0082D05D11B7813F068
:10EC60007F0F3DD11C4B1BE00A2D39D11A7802F0E1
:10EC70007F02012A34D19A7A002A31D0598800299A
:10EC80002ED15A6822F47F42B2F5803F28D15879BC
:10EC90000B4B1B689B69984710BB104B00E0FBB106
:10ECA000054A4FF000011268002093615182984795
:10ECB000002020E0505C0040180D002004300020AF
:10ECC000B00C0020023000207C0D0020005C0040D1
:10ECD00004010020C1E50008F1E4000851E5000846
:10ECE000244C254B22681B6850781B6998470328E1
:10ECF00001D1236806E01F4B4FF6FF711B681A8A8B
:10ED00008A4201D1092203E0022800D012B9082268
:10ED10001A722BE093F90010002921DAD9880191A9
:10ED20000198824202D9019A1A8211E08A420FD2D6
:10ED30001149096891F82C108A4201D2002105E09E
:10ED400092FBF1F001FB102212B901210B4A117064
:10ED5000094A126892F82C209A82FFF799FD05E083
:10ED600003221A72064B4FF440521A80FFF706FD39
:10ED7000FEBD00BF180D0020B00C0020DC060020F6
:10ED80007A0D0020074A022108B507481172074989
:10ED9000074B086007490A60074A13601B689847D9
:10EDA00008BD00BFB80C002008010020D40C0020D2
:10EDB00080000020180D0020B00C002008B529E0CC
:10EDC00047F6FF700860198801F00F018B0003F10E
:10EDD0008043117003F5B843196889B211F4004FEC
:10EDE00009D0186840F68F7100EA010119601278A5
:10EDF0000E4B013A0BE011F0800F0BD0186848F66B
:10EE00000F7100EA010119601278094B013A53F8B9
:10EE1000223098470749084B0868084A80B2188092
:10EE2000188800B20028CBDB08BD00BFE800002036
:10EE3000CC000020445C0040AE0C0020B40C00204C
:10EE4000F8B59AE047F6FF761E601688564F06F032
:10EE50000F06B30003F1804303F5B8433E70002E64
:10EE600064D127682668236807F4405C03EA000041
:10EE700080F400502060236806F0300003EA0101AE
:10EE800081F0200121601388484A13F0100F108090
:10EE9000A5F800C004D023689BB213F0800F08D0FF
:10EEA000226848F60F7302EA03032360FFF746FD6A
:10EEB00016E013F4006F08D0226840F68F7302EA60
:10EEC00003032360FFF7DAFD0AE013F4004F54D088
:10EED000226840F68F7302EA03032360FFF770FC99
:10EEE00021682A884BF68F7301EA030312F4805FCE
:10EEF00018BF83F4805312F4005F2D4A18BF83F4C7
:10EF000000531360294B11681A8848F6BF7301EA51
:10EF1000030312F0100F18BF83F0100312F0200F3C
:10EF2000234A18BF83F0200313603BE01C68A4B29F
:10EF300014F4004F0BD0196840F68F7201EA0202F8
:10EF40001A603A781B4B013A53F82230984714F074
:10EF5000800F12D0144948F60F720B789B0003F112
:10EF6000804303F5B843186800EA02021A600A7881
:10EF7000114B013A53F822309847104B104A1D6844
:10EF80000B4C1FFA85FCA2F800C0B2F800C04BF68B
:10EF90008F700FFA8CFCBCF1000F48F6BF71094D61
:10EFA000FFF650AFF8BD00BFB40C00207C0D002070
:10EFB000005C0040E8000020CC000020445C0040E1
:10EFC000AE0C00207A0D002001F10051013201F554
:10EFD000405110B549005208002308E010F803C062
:10EFE0006478013A4CEA042C21F813C00233C418A7
:10EFF000002AF3D110BD00BF01F10051013201F52B
:10F00000405110B549005208002304E031F8134084
:10F01000013AC4520233002AF8D110BD014B1860E6
:10F02000704700BF405C0040014B186880B27047D9
:10F03000405C0040014B1860704700BF445C0040DA
:10F04000014B186880B27047445C0040014B18685F
:10F0500080B27047485C0040014B1860704700BFA9
:10F060004C5C0040014B186880B270474C5C00401B
:10F070004FF6F873024A00EA03031360704700BFBB
:10F08000505C0040014B186880B27047505C0040F3
:10F09000014B43F820107047005C0040024B53F8CE
:10F0A000200080B2704700BF005C0040054B10B5E7
:10F0B00053F8204048F68F1204EA02020A4343F84C
:10F0C000202010BD005C0040024B53F8200000F4EB
:10F0D000C0607047005C00400A4B10B553F8202018
:10F0E00048F6BF7402EA040411F0100F18BF84F050
:10F0F000100411F0200F18BF84F0200443F82040C2
:10F1000010BD00BF005C00400A4B10B553F8202032
:10F110004BF68F7402EA040411F4805F18BF84F484
:10F12000805411F4005F18BF84F4005443F8204069
:10F1300010BD00BF005C004038B50D460446FFF727
:10F14000ADFF012D02D120F4805003E0022D04D147
:10F1500020F01000014B43F8240038BD005C004053
:10F16000024B53F8200000F030007047005C004074
:10F17000024B53F8200000F440507047005C004000
:10F18000054B48F6BF7253F8201001EA020282F0E4
:10F19000300243F820207047005C0040054B4BF6DE
:10F1A0008F7253F8201001EA020282F4405243F8B1
:10F1B00020207047005C0040054B48F68F6253F8F2
:10F1C000201001EA020242F4807243F820207047C6
:10F1D000005C0040044B48F68F6253F8201001EAAF
:10F1E000020243F820207047005C0040044B48F6C0
:10F1F0008F6253F8201001EA020243F82020704782
:10F20000005C0040054B48F68F6253F8201001EA7D
:10F21000020242F4807243F820207047005C0040F4
:10F22000054B48F68F6253F8201001EA020242F4BF
:10F23000807243F820207047005C0040044B48F681
:10F240008F6253F8201001EA020243F82020704731
:10F25000005C0040044B53F8200000F03000102800
:10F2600014BF002001207047005C0040054B53F89C
:10F27000200000F44050B0F5805F14BF0020012052
:10F28000704700BF005C0040044B40F68F7253F89B
:10F29000201001EA020243F820207047005C004081
:10F2A000044B48F60F7253F8201001EA020243F8AB
:10F2B00020207047005C0040054B48F68F7253F8E1
:10F2C000201001EA020242F4804243F820207047F5
:10F2D000005C0040054B48F68F7253F8201001EA9D
:10F2E000020242F0400243F820207047005C0040D8
:10F2F000084B53F8202012F4804F09D053F8201007
:10F3000048F68F7201EA020242F4804243F820205C
:10F31000704700BF005C0040084B53F8202012F0FB
:10F32000400F09D053F8201048F68F7201EA02020C
:10F3300042F0400243F82020704700BF005C0040CC
:10F34000054B10B553F8204048F68F7204EA0202CC
:10F350000A4343F8202010BD005C0040024B53F8E4
:10F36000200000F00F007047005C0040064B490889
:10F370001B6849009BB203EBC00303F1005303F584
:10F3800040535B0019607047505C0040054A064BD3
:10F390001268490892B202EBC002D3185B00490020
:10F3A00019607047505C004004300020054B1B681A
:10F3B0009BB203EBC00303F1005303F540535B0022
:10F3C00018887047505C0040044A054B126892B29E
:10F3D00002EBC002D3185B0018887047505C0040F5
:10F3E00004300020044A054B126892B202EBC002BE
:10F3F000D3185B0019607047505C00400230002059
:10F400003E2909D94B0911F01F0F01D1013B9BB2D5
:10F410009B0243F4004305E04B0811F0010F18BFB5
:10F4200001339B02036070470D4A0E4B126892B283
:10F43000D31803EBC0035B003E2909D94A0911F038
:10F440001F0F01D1013A92B2920242F4004205E04C
:10F450004A0811F0010F18BF013292021A6070477A
:10F46000505C004006300020054A064B126892B2FC
:10F4700002EBC002D3185B0018688005800D70474E
:10F48000505C004002300020054A064B126892B2E0
:10F4900002EBC002D3185B0018688005800D70472E
:10F4A000505C0040063000200C4B30B51D681C68D5
:10F4B000C0001FFA85FC8444A4B2094B00190CF16A
:10F4C000005CC3180CF5405C490852084FEA4C0038
:10F4D00049005B00520001601A6030BD505C004082
:10F4E00004300020064B49081B6849009BB203EB1F
:10F4F000C00303F1005303F540535B0019607047EC
:10F50000505C0040054A064B1268490892B202EB73
:10F51000C002D3185B00490019607047505C00407E
:10F5200004300020054B1B689BB203EBC00303F1C2
:10F53000005303F540535B0018887047505C00404F
:10F54000044A054B126892B202EBC002D3185B006A
:10F5500018887047505C004004300020012910B525
:10F5600024D1254B25491B68C0009BB259180918A6
:10F570004B003E2A09D9510912F01F0F01D1013960
:10F5800089B2890241F4004105E0510812F0010FEF
:10F5900018BF0131890219601749194B096889B2EE
:10F5A000CB18181840003E2A1ED913E0022922D198
:10F5B000114BC0001C681B68A4B21FFA83FC0F49E2
:10F5C0000F4B844400194118634449005B000A60F2
:10F5D0001A6010E0530912F01F0F01D1013B9BB2DA
:10F5E0009B0243F4004305E0530812F0010F18BFDB
:10F5F00001339B02036010BD505C004002300020CC
:10F600000630002001291BD11349144B096889B227
:10F61000CB1803EBC00040003E2A09D9530912F071
:10F620001F0F01D1013B9BB29B0243F4004305E055
:10F63000530812F0010F18BF01339B0203600AE068
:10F64000022908D10449054B096889B201EBC000C1
:10F65000C3185B001A607047505C00400230002005
:10F6600001291BD11349144B096889B2CB1803EB4C
:10F67000C00040003E2A09D9530912F01F0F01D1E2
:10F68000013B9BB29B0243F4004305E0530812F098
:10F69000010F18BF01339B0203600AE0022908D161
:10F6A0000449054B096889B201EBC000C3185B002F
:10F6B0001A607047505C004006300020054A064B37
:10F6C000126892B202EBC002D3185B001868800582
:10F6D000800D7047505C004002300020054A064B08
:10F6E000126892B202EBC002D3185B001868800562
:10F6F000800D7047505C0040063000200D4BC0006C
:10F7000019680D4A89B241188A185200128812F4F9
:10F710007C4F01D001200CE01A68084B92B280188F
:10F72000C3185B0018888005800D002814BF0220D4
:10F7300000207047505C004006300020023000205E
:10F74000012909D10B4A48F68F7352F8201001EABB
:10F75000030343F040030AE002290AD1054A48F6B0
:10F760008F7352F8201001EA030343F4804342F8F8
:10F7700020307047005C004041EA0020704700BF25
:10F78000030AC0B243EA0020704700BF08B5002258
:10F790000A2300F045F808BD08B500210A2200F050
:10F7A000DFF808BDF0B40378002B2DD040F23412FE
:10F7B000C2F20002156802E010F8013FEBB15A19DD
:10F7C00003F12004527812F001070A7808BF1C46A2
:10F7D00001F10101561C9446AE5D16F0010F18BFF1
:10F7E00002F1200C6445E7D007B1203316F0010F79
:10F7F00018BF2032981AF0BC70470A786F78561CF0
:10F8000007F00107AE5DEFE740F234100A78C2F26C
:10F810000000561C05686F78AE5D07F00107E3E74E
:10F820002DE9F04F40F23415C2F2000583B00C46CA
:10F830001F46D5F800800E460190009216F8015B35
:10F8400008EB050393F801B01BF0080BF6D12D2D42
:10F8500065D02B2D08BF16F8015BD7F1010338BF27
:10F860000023102F14BF1A4643F0010232B1302D8D
:10F8700066D01BB1302D0CBF08270A27BBF1000F43
:10F88000394614BF4FF000496FF00049484600F078
:10F8900059FC48468A46394600F026FB00218C4632
:10F8A00008EB0502A5F13003527812F0040F08D1DD
:10F8B00012F0030F20D012F0010F14BF372357238B
:10F8C000EB1A9F4218DD844594BF0022012252EAC0
:10F8D000D1714FF0FF310CD1844514BF00220122B9
:10F8E0005345D4BF002202F0010212B907FB0C3CC1
:10F8F000012116F8015BD3E7B1F1FF3F14D0BBF152
:10F90000000F09D16046009B1BB101B1741E009A23
:10F91000146003B0BDE8F08FCCF10000F3E716F8F7
:10F92000015B4FF0010B98E7019ABBF1000F4FF01C
:10F93000220314BF4FF000406FF000401360E2E775
:10F940003278782A14BF00210121582A14BF0A46B0
:10F9500041F00102002A8CD07578102702368DE71D
:10F9600010B540F23814C2F200048C46134601462A
:10F9700062462068FFF754FF10BD00BF2DE9F04339
:10F980008BB006460F4600F07BF840F22C24C2F202
:10F99000000494F90030B3F1FF3F8046894638D027
:10F9A0003046394600F084FA0546002831D1304609
:10F9B00039460022002301F01DF8002829D12478BF
:10F9C00041F60033C0F6010308950193CDE90267C3
:10F9D000CDE90467002C21D040F200030022CFF6CD
:10F9E000F0733046CDE9062339460022002300F0AB
:10F9F000D9FF002822D0022300939C4234D06846CD
:10FA000000F064FA00282FD0089B002B27D1DDE9F5
:10FA10000689404649460BB0BDE8F0834FF6FF73B8
:10FA20004FF06042CCF2EF733046CDE90623394601
:10FA30000022002300F0B6FF0028DCD10123022CB5
:10FA4000009316D0684600F041FA90B141F60430B8
:10FA5000C0F6010000F03CFACDE90601D4E700F061
:10FA60003DFA089B0360D2E700F038FA22230360D6
:10FA7000CAE700F033FA21230360E7E70000000043
:10FA8000B1F5801F0B462DE9F04F804687B08946BF
:10FA900004460D463EDB4FF6FF720026C7F6EF72B6
:10FAA000934251DC23F07F4445F6647C24F47004D7
:10FAB000C0F2090CA44440F20002A6F57E760CF4D4
:10FAC000801C073EC3F6F0728CEA020206EB235656
:10FAD00040F20003404642EA0401C3F6F0730022FC
:10FAE00006EB1C5600F042FBA31C23F07F4323F4DB
:10FAF0007003022B804689462FDC0022002300F091
:10FB000051FF002800F0CA80002E40F07C810020C8
:10FB100000211FE021F00043034300F0B5800029DD
:10FB2000C0F2468140F200030022C4F250336FF06D
:10FB3000350600F0CFFC4FF6FF72C7F6EF720B46AA
:10FB4000804693428946ADDD4046494642464B4693
:10FB500000F00EFB07B0BDE8F08F00224FF08043AD
:10FB600000F006FB4EF68635CFF6F97565190246AC
:10FB70000B464046494600F0D7FDCDE9020130462C
:10FB800000F042FCCDE90401DDE9020102460B462A
:10FB900000F0A0FC02460B46CDE9000100F09AFC03
:10FBA000A7A3D3E9002382468B4600F093FCA6A3CB
:10FBB000D3E9002300F0DCFA52465B4600F08AFCF1
:10FBC000A3A3D3E9002300F0D3FA52465B4600F02A
:10FBD00081FCA1A3D3E9002300F0CAFADDE90023E8
:10FBE00000F078FC9EA3D3E90023CDE90001504644
:10FBF000594600F06FFC9CA3D3E9002300F0B8FA4B
:10FC000052465B4600F066FC99A3D3E9002300F05E
:10FC1000AFFA52465B4600F05DFC0B460246DDE95A
:10FC2000000100F0A5FA4BF65103C0F206031B1BBE
:10FC300043EA0505002D82468B4656DD40F200035F
:10FC40000022C3F6E0734046494600F043FC4246BA
:10FC50004B4600F03FFC04460D46002E75D152463F
:10FC60005B4600F085FADDE9022300F033FC024632
:10FC70000B462046294600F079FA02460B464046DC
:10FC8000494600F073FA65E740F2000100200022C7
:10FC90000023CCF2503100F047FD5BE742464B4673
:10FCA0004046494600F016FC73A3D3E900230446FE
:10FCB0000D464046494600F00DFC40F2000300228C
:10FCC000C3F6E07300F054FA02460B46204629467C
:10FCD00000F000FC04460D46002E72D14046494615
:10FCE00022462B4600F042FA34E7002E00F0D48082
:10FCF00063A3D3E90023DDE9040100F0EBFB5246E6
:10FD00005B4606460F464046494600F02FFADDE9BD
:10FD1000022300F0DFFB5CA3D3E9002304460D4679
:10FD2000DDE9040100F0D6FB02460B4620462946D9
:10FD300000F01EFA42464B4600F018FA02460B4607
:10FD40003046394600F012FA04E74DA3D3E9002308
:10FD5000DDE9040100F0BEFB52465B46CDE900013F
:10FD60002046294600F004FADDE9022300F0B2FB48
:10FD700047A3D3E9002306460F46DDE9040100F05E
:10FD8000A9FB02460B463046394600F0F1F902461F
:10FD90000B462046294600F0E9F942464B4600F062
:10FDA000E5F902460B46DDE9000100F0DFF9D1E696
:10FDB00002460B4600F0DAF90022002300F0B4FC02
:10FDC000C8E6304600F020FB2DA3D3E90023064609
:10FDD0000F4600F07FFB2CA3D3E9002382468B461D
:10FDE0003046394600F076FB22462B4600F0C0F93B
:10FDF00042464B4600F0BAF902460B465046594679
:10FE000000F0B4F9A6E6304600F0FEFA1CA3D3E9F0
:10FE1000002306460F4600F05DFB1DA3D3E9002337
:10FE200004460D463046394600F054FB02460B4668
:10FE30002046294600F09CF98CE600BFAFF3008015
:10FE400044523EDF12F1C23FDE03CB966446C73F09
:10FE5000599322942449D23F935555555555E53F22
:10FE60009FC678D0099AC33FAF788E1DC571CC3F2D
:10FE700004FA97999999D93F555555555555D5BF78
:10FE80000000E0FE422EE63F763C7935EF39EABDD0
:10FE9000763C7935EF39EA3D02460B464046494605
:10FEA00000F064F9DDE9022300F014FBE5E600BF91
:10FEB00002464042104321F0004141EAD070C0F1B7
:10FEC000FE4000F57000C00F704700BF0020704773
:10FED00040F200010020C7F6F871704740F2381375
:10FEE000C2F20003186870474A1E08BF7047C0F08E
:10FEF0002481884240F21681114200F01781B0FA45
:10FF000080F3B1FA81F2A2EB0303C3F11F0304A251
:10FF100002EB03134FF000029F4600BFAFF30080D7
:10FF2000B0EBC17F00BF42EB020228BFA0EBC17063
:10FF3000B0EB817F00BF42EB020228BFA0EB8170D3
:10FF4000B0EB417F00BF42EB020228BFA0EB417043
:10FF5000B0EB017F00BF42EB020228BFA0EB0170B3
:10FF6000B0EBC16F00BF42EB020228BFA0EBC16043
:10FF7000B0EB816F00BF42EB020228BFA0EB8160B3
:10FF8000B0EB416F00BF42EB020228BFA0EB416023
:10FF9000B0EB016F00BF42EB020228BFA0EB016093
:10FFA000B0EBC15F00BF42EB020228BFA0EBC15023
:10FFB000B0EB815F00BF42EB020228BFA0EB815093
:10FFC000B0EB415F00BF42EB020228BFA0EB415003
:10FFD000B0EB015F00BF42EB020228BFA0EB015073
:10FFE000B0EBC14F00BF42EB020228BFA0EBC14003
:10FFF000B0EB814F00BF42EB020228BFA0EB814073
:020000040801F1
:10000000B0EB414F00BF42EB020228BFA0EB4140E2
:10001000B0EB014F00BF42EB020228BFA0EB014052
:10002000B0EBC13F00BF42EB020228BFA0EBC130E2
:10003000B0EB813F00BF42EB020228BFA0EB813052
:10004000B0EB413F00BF42EB020228BFA0EB4130C2
:10005000B0EB013F00BF42EB020228BFA0EB013032
:10006000B0EBC12F00BF42EB020228BFA0EBC120C2
:10007000B0EB812F00BF42EB020228BFA0EB812032
:10008000B0EB412F00BF42EB020228BFA0EB4120A2
:10009000B0EB012F00BF42EB020228BFA0EB012012
:1000A000B0EBC11F00BF42EB020228BFA0EBC110A2
:1000B000B0EB811F00BF42EB020228BFA0EB811012
:1000C000B0EB411F00BF42EB020228BFA0EB411082
:1000D000B0EB011F00BF42EB020228BFA0EB0110F2
:1000E000B0EBC10F00BF42EB020228BFA0EBC10082
:1000F000B0EB810F00BF42EB020228BFA0EB8100F2
:10010000B0EB410F00BF42EB020228BFA0EB410061
:10011000B0EB010F00BF42EB020228BFA0EB0100D1
:10012000104670470CBF012000207047B1FA81F2E1
:10013000C2F11F0220FA02F0704708B14FF0FF3001
:1001400000F00EB80029F8D02DE90340FFF7CCFEEF
:10015000BDE8064002FB00F3A1EB0301704700BFBE
:10016000704700BF81F0004102E000BF83F0004310
:1001700030B54FEA41044FEA430594EA050F08BF42
:1001800090EA020F1FBF54EA000C55EA020C7FEA06
:10019000645C7FEA655C00F0E2804FEA5454D4EB83
:1001A0005555B8BF6D420CDD2C4480EA020281EA4D
:1001B000030382EA000083EA010180EA020281EA85
:1001C0000303362D88BF30BD11F0004F4FEA0131D7
:1001D0004FF4801C4CEA113102D0404261EB4101E6
:1001E00013F0004F4FEA03334CEA133302D052426C
:1001F00063EB430394EA050F00F0A780A4F1010428
:10020000D5F1200E0DDB02FA0EFC22FA05F2801861
:1002100041F1000103FA0EF2801843FA05F3594147
:100220000EE0A5F120050EF1200E012A03FA0EFCC6
:1002300028BF4CF0020C43FA05F3C01851EBE371F0
:1002400001F0004507D54FF0000EDCF1000C7EEB0D
:1002500000006EEB0101B1F5801F1BD3B1F5001F4B
:100260000CD349085FEA30004FEA3C0C04F101046A
:100270004FEA445212F5800F80F09A80BCF1004F93
:1002800008BF5FEA500C50F1000041EB045141EA15
:10029000050130BD5FEA4C0C404141EB010111F416
:1002A000801FA4F10104E9D191F0000F04BF0146C1
:1002B0000020B1FA81F308BF2033A3F10B03B3F19F
:1002C00020020CDA0C3208DD02F1140CC2F10C022F
:1002D00001FA0CF021FA02F10CE002F11402D8BF8D
:1002E000C2F1200C01FA02F120FA0CFCDCBF41EA59
:1002F0000C019040E41AA2BF01EB0451294330BD28
:100300006FEA04041F3C1CDA0C340EDC04F1140404
:10031000C4F1200220FA04F001FA02F340EA0300DB
:1003200021FA04F345EA030130BDC4F10C04C4F121
:10033000200220FA02F001FA04F340EA0300294601
:1003400030BD21FA04F0294630BD94F0000F83F44B
:10035000801306BF81F480110134013D4EE77FEA2E
:10036000645C18BF7FEA655C29D094EA050F08BF7A
:1003700090EA020F05D054EA000C04BF194610465B
:1003800030BD91EA030F1EBF0021002030BD5FEA9F
:10039000545C05D14000494128BF41F0004130BDC7
:1003A00014F580043CBF01F5801130BD01F000451B
:1003B00045F0FE4141F470014FF0000030BD7FEA8E
:1003C000645C1ABF194610467FEA655C1CBF0B4689
:1003D000024650EA013406BF52EA033591EA030FA0
:1003E00041F4002130BD00BF90F0000F04BF002198
:1003F000704730B54FF4806404F132044FF00005CB
:100400004FF0000150E700BF90F0000F04BF002143
:10041000704730B54FF4806404F1320410F00045A9
:1004200048BF40424FF000013EE700BF42004FEAA4
:10043000E2014FEA31014FEA02701FBF12F07F4321
:1004400093F07F4F81F06051704792F0000F14BF1E
:1004500093F07F4F704730B54FF4607401F0004562
:1004600021F0004120E700BF50EA010208BF7047B9
:1004700030B54FF000050AE050EA010208BF7047AE
:1004800030B511F0004502D5404261EB41014FF417
:10049000806404F132045FEA915C3FF4DCAE4FF01B
:1004A00003025FEADC0C18BF03325FEADC0C18BF02
:1004B000033202EBDC02C2F1200300FA03FC20FA53
:1004C00002F001FA03FE40EA0E0021FA02F11444A0
:1004D000C1E600BF70B54FF0FF0C4CF4E06C1CEAB5
:1004E00011541DBF1CEA135594EA0C0F95EA0C0F2A
:1004F00000F0DEF82C4481EA030621EA4C5123EA9D
:100500004C5350EA013518BF52EA033541F48011CB
:1005100043F4801338D0A0FB02CE4FF00005E1FB7E
:1005200002E506F00042E0FB03E54FF00006E1FBC8
:1005300003569CF0000F18BF4EF0010EA4F1FF040B
:10054000B6F5007F64F5407404D25FEA4E0E6D414B
:1005500046EB060642EAC62141EA55514FEAC5205C
:1005600040EA5E504FEACE2EB4F1FD0C88BFBCF5D8
:10057000E06F1ED8BEF1004F08BF5FEA500E50F189
:10058000000041EB045170BD06F0004646EA01014F
:1005900040EA020081EA0301B4EB5C04C2BFD4EB81
:1005A0000C0541EA045170BD41F480114FF0000E7A
:1005B000013C00F3AB8014F1360FDEBF002001F0E8
:1005C000004170BDC4F10004203C35DA0C341BDC62
:1005D00004F11404C4F1200500FA05F320FA04F034
:1005E00001FA05F240EA020001F0004221F0004168
:1005F00010EBD37021FA04F642EB06015EEA430EDB
:1006000008BF20EAD37070BDC4F10C04C4F120050A
:1006100000FA04F320FA05F001FA04F240EA0200BD
:1006200001F0004110EBD37041F100015EEA430E8E
:1006300008BF20EAD37070BDC4F1200500FA05F2AE
:100640004EEA020E20FA04F301FA05F243EA02032D
:1006500021FA04F001F0004121FA04F220EA02003C
:1006600000EBD3705EEA430E08BF20EAD37070BD82
:1006700094F0000F0FD101F00046400041EB010162
:1006800011F4801F08BF013CF7D041EA060195F044
:10069000000F18BF704703F00046520043EB0303FE
:1006A00013F4801F08BF013DF7D043EA06037047EB
:1006B00094EA0C0F0CEA135518BF95EA0C0F0CD0F6
:1006C00050EA410618BF52EA4306D1D181EA03013C
:1006D00001F000414FF0000070BD50EA410606BF36
:1006E0001046194652EA430619D094EA0C0F02D17B
:1006F00050EA013613D195EA0C0F05D152EA0336C0
:100700001CBF104619460AD181EA030101F00041DD
:1007100041F0FE4141F470014FF0000070BD41F026
:10072000FE4141F4780170BD70B54FF0FF0C4CF400
:10073000E06C1CEA11541DBF1CEA135594EA0C0F1F
:1007400095EA0C0F00F0A7F8A4EB050481EA030E6C
:1007500052EA03354FEA013100F088804FEA033353
:100760004FF0805545EA131343EA12634FEA022221
:1007700045EA111545EA10654FEA00260EF00041E2
:100780009D4208BF964244F1FD0404F5407402D234
:100790005B084FEA3202B61A65EB03055B084FEAC5
:1007A00032024FF480104FF4002CB6EB020E75EBC2
:1007B000030E22BFB61A754640EA0C005B084FEAEA
:1007C0003202B6EB020E75EB030E22BFB61A754667
:1007D00040EA5C005B084FEA3202B6EB020E75EBB2
:1007E000030E22BFB61A754640EA9C005B084FEA2A
:1007F0003202B6EB020E75EB030E22BFB61A754637
:1008000040EADC0055EA060E18D04FEA051545EA25
:1008100016754FEA06164FEAC30343EA52734FEACE
:10082000C2025FEA1C1CC0D111F4801F0BD141EA47
:1008300000014FF000004FF0004CB6E711F4801FAC
:1008400004BF01430020B4F1FD0C88BFBCF5E06F8C
:100850003FF6AFAEB5EB030C04BFB6EB020C5FEA9C
:10086000500C50F1000041EB045170BD0EF0004EF1
:100870004EEA113114EB5C04C2BFD4EB0C0541EA23
:10088000045170BD41F480114FF0000E013C90E620
:1008900045EA060E8DE60CEA135594EA0C0F08BFE4
:1008A00095EA0C0F3FF43BAF94EA0C0F0AD150EAE3
:1008B00001347FF434AF95EA0C0F7FF425AF104676
:1008C00019462CE795EA0C0F06D152EA03353FF49E
:1008D000FDAE1046194622E750EA410618BF52EA1B
:1008E00043067FF4C5AE50EA41047FF40DAF52EAEF
:1008F00043057FF4EBAE12E74FF0FF3C06E000BF8C
:100900004FF0010C02E000BF4FF0010C4DF804CD98
:100910004FEA410C7FEA6C5C4FEA430C18BF7FEA58
:100920006C5C1BD001B050EA410C0CBF52EA430C86
:1009300091EA030F02BF90EA020F0020704710F106
:10094000000F91EA030F58BF994208BF90422CBF95
:10095000D8176FEAE37040F0010070474FEA410C8E
:100960007FEA6C5C02D150EA013C07D14FEA430CAC
:100970007FEA6C5CD6D152EA033CD3D05DF8040B1D
:10098000704700BF8446104662468C46194663464F
:1009900000E000BF01B5FFF7B7FF002848BF10F126
:1009A000000F01BD4DF808EDFFF7F4FF0CBF01206B
:1009B00000205DF808FB00BF4DF808EDFFF7EAFFE7
:1009C00034BF012000205DF808FB00BF4DF808EDA2
:1009D000FFF7E0FF94BF012000205DF808FB00BF97
:1009E0004DF808EDFFF7CEFF94BF012000205DF821
:1009F00008FB00BF4DF808EDFFF7C4FF34BF01202E
:100A000000205DF808FB00BF4FEA410212F500121A
:100A100015D211D56FF47873B3EB625212D94FEA45
:100A2000C12343F0004343EA505311F0004F23FA2F
:100A300002F018BF404270474FF00000704750EA84
:100A4000013005D111F0004008BF6FF00040704741
:100A50004FF00000704700BF4FEA4102B2F1E0439F
:100A600024BFB3F5001CDCF1FE5C0DD901F0004C95
:100A70004FEAC0024CEA5070B2F1004F40EB8300E5
:100A800008BF20F00100704711F0804F21D113F111
:100A90003872BCBF01F00040704741F480114FEA4A
:100AA0005252C2F11802C2F1200C10FA0CF320FAD3
:100AB00002F018BF40F001004FEAC1234FEAD323F0
:100AC00003FA0CFC40EA0C0023FA02F34FEA43035A
:100AD000CCE77FEA625307D150EA01331EBF4FF0E3
:100AE000FE4040F44000704701F0004040F0FE40FE
:100AF00040F40000704700BF80F0004002E000BFFB
:100B000081F0004142001FBF5FEA410392EA030FF8
:100B10007FEA226C7FEA236C6AD04FEA1262D2EB42
:100B20001363C1BFD218414048404140B8BF5B4247
:100B3000192B88BF704710F0004F40F4000020F0E0
:100B40007F4018BF404211F0004F41F4000121F0F6
:100B50007F4118BF494292EA030F3FD0A2F1010240
:100B600041FA03FC10EB0C00C3F1200301FA03F17E
:100B700000F0004302D5494260EB4000B0F5000FA1
:100B800013D3B0F1807F06D340084FEA310102F160
:100B90000102FE2A51D2B1F1004F40EBC25008BF12
:100BA00020F0010040EA03007047490040EB0000DC
:100BB00010F4000FA2F10102EDD1B0FA80FCACF10B
:100BC000080CB2EB0C0200FA0CF0AABF00EBC2500A
:100BD00052421843BCBFD0401843704792F0000FF8
:100BE00081F4000106BF80F400000132013BB5E74B
:100BF0004FEA41037FEA226C18BF7FEA236C21D0C1
:100C000092EA030F04D092F0000F08BF0846704725
:100C100090EA010F1CBF0020704712F07F4F04D1F3
:100C2000400028BF40F00040704712F100723CBF06
:100C300000F50000704700F0004343F0FE4040F430
:100C4000000070477FEA226216BF08467FEA2363EE
:100C50000146420206BF5FEA412390EA010F40F4D9
:100C6000800070474FF0000304E000BF10F0004325
:100C700048BF40425FEA000C08BF704743F096430C
:100C800001464FF000001CE050EA010208BF704727
:100C90004FF000030AE000BF50EA010208BF7047AE
:100CA00011F0004302D5404261EB41015FEA010CC3
:100CB00002BF84460146002043F0B64308BFA3F1BB
:100CC0008053A3F50003BCFA8CF2083AA3EBC2539D
:100CD00010DB01FA02FC634400FA02FCC2F12002BC
:100CE000BCF1004F20FA02F243EB020008BF20F0F3
:100CF0000100704702F1200201FA02FCC2F1200259
:100D000050EA4C0021FA02F243EB020008BF20EA4D
:100D1000DC7070474FF0FF0C1CEAD0521EBF1CEA7B
:100D2000D15392EA0C0F93EA0C0F6FD01A4480EA69
:100D3000010C400218BF5FEA41211ED04FF0006352
:100D400043EA501043EA5111A0FB01310CF000407E
:100D5000B1F5000F3EBF490041EAD3715B0040EAA4
:100D6000010062F17F02FD2A1DD8B3F1004F40EB74
:100D7000C25008BF20F00100704790F0000F0CF047
:100D8000004C08BF49024CEA502040EA51207F3A0B
:100D9000C2BFD2F1FF0340EAC250704740F40000E6
:100DA0004FF00003013A5DDC12F1190FDCBF00F0D7
:100DB00000407047C2F10002410021FA02F1C2F185
:100DC000200200FA02FC5FEA310040F1000053EA21
:100DD0004C0308BF20EADC70704792F0000F00F06F
:100DE000004C02BF400010F4000F013AF9D040EA75
:100DF0000C0093F0000F01F0004C02BF490011F409
:100E0000000F013BF9D041EA0C018FE70CEAD15306
:100E100092EA0C0F18BF93EA0C0F0AD030F0004C86
:100E200018BF31F0004CD8D180EA010000F000403A
:100E3000704790F0000F17BF90F0004F084691F0F8
:100E4000000F91F0004F14D092EA0C0F01D1420232
:100E50000FD193EA0C0F03D14B0218BF084608D1FB
:100E600080EA010000F0004040F0FE4040F4000045
:100E7000704740F0FE4040F4400070474FF0FF0CD8
:100E80001CEAD0521EBF1CEAD15392EA0C0F93EA1F
:100E90000C0F69D0A2EB030280EA010C49024FEA71
:100EA000402037D04FF0805343EA111143EA10132A
:100EB0000CF000408B4238BF5B0042F17D024FF4E2
:100EC000000C8B4224BF5B1A40EA0C00B3EB510FBD
:100ED00024BFA3EB510340EA5C00B3EB910F24BFA6
:100EE000A3EB910340EA9C00B3EBD10F24BFA3EB2B
:100EF000D10340EADC001B0118BF5FEA1C1CE0D1F3
:100F0000FD2A3FF650AF8B4240EBC25008BF20F0A5
:100F1000010070470CF0004C4CEA50207F32C2BFF9
:100F2000D2F1FF0340EAC250704740F400004FF096
:100F30000003013A37E792F0000F00F0004C02BFC7
:100F4000400010F4000F013AF9D040EA0C0093F091
:100F5000000F01F0004C02BF490011F4000F013BEB
:100F6000F9D041EA0C0195E70CEAD15392EA0C0F53
:100F700008D142027FF47DAF93EA0C0F7FF470AF8B
:100F8000084676E793EA0C0F04D14B023FF44CAFCE
:100F900008466EE730F0004C18BF31F0004CCAD163
:100FA00030F000427FF45CAF31F000437FF43CAF9F
:100FB0005FE700BF4FF0FF3C06E000BF4FF0010CC1
:100FC00002E000BF4FF0010C4DF804CD4FEA4002A3
:100FD0004FEA41037FEA226C18BF7FEA236C11D0ED
:100FE00001B052EA530C18BF90EA010F58BFB2EBA0
:100FF000030088BFC81738BF6FEAE17018BF40F020
:10100000010070477FEA226C02D15FEA402C05D1D3
:101010007FEA236CE4D15FEA412CE1D05DF8040B58
:10102000704700BF844608466146FFE70FB5FFF7EB
:10103000C9FF002848BF10F1000F0FBD4DF808EDA3
:10104000FFF7F4FF0CBF012000205DF808FB00BF94
:101050004DF808EDFFF7EAFF34BF012000205DF8EE
:1010600008FB00BF4DF808EDFFF7E0FF94BF01203B
:1010700000205DF808FB00BF4DF808EDFFF7D2FF38
:1010800094BF012000205DF808FB00BF4DF808ED7B
:10109000FFF7C8FF34BF012000205DF808FB00BF48
:1010A00042000ED2B2F1FE4F0BD34FF09E03B3EBD2
:1010B000126209D44FEA002343F0004323FA02F0FE
:1010C00070474FF00000704712F1610F01D14202EA
:1010D00002D14FF0FF3070474FF00000704700BF63
:1010E00073B96AB9002908BF0028BCBF00204FF0BF
:1010F0000041C4BF6FF000414FF0FF30FFF730B840
:1011000082B0EC462DE9005000F01CF8DDF804E058
:1011100002B00CBC704700BFF8B514461D46064629
:101120000F4600F0D3F900FB05F5A0FB042304FBF8
:101130000154E318B61A67EB0307069BC3E900677F
:10114000F8BD00BFF8B514461D4606460F4600F030
:101150000FF800FB05F5A0FB042304FB0154E31882
:10116000B61A67EB0307069BC3E90067F8BD00BF2B
:1011700000292DE9F04F85B0C0F2C9800026002B70
:10118000C0F2C0808946144605469B46002B4BD1D1
:101190008A4258D9B2FA82F353B1C3F1200001FA5E
:1011A00003F925FA00F812FA03F49D4048EA090908
:1011B000270C484639461FFA84FBFEF795FE394650
:1011C00082464846FEF7BEFF4FEA15420BFB0AF384
:1011D00042EA01494B4509D919EB04090AF1FF3AE2
:1011E00004D24B4584BF0AF1FF3AA144C3EB09097D
:1011F00039464846ADB2FEF777FE39468046484646
:10120000FEF7A0FF0BFB08FB45EA0145AB4507D9FC
:101210002D1908F1FF3803D2AB4588BF08F1FF381C
:1012200048EA0A48002703E08B4257D90027B8460E
:1012300042463B4616B1524263EB43031946104601
:1012400005B0BDE8F08F22B911460120FEF74CFE33
:101250000446B4FA84F8B8F1000F5ED1C4EB090873
:10126000270C1FFA84F90121029139464046FEF706
:101270003BFE394682464046FEF764FF4FEA15487A
:1012800009FB0AF348EA014B5B4509D91BEB040B48
:101290000AF1FF3A04D25B4584BF0AF1FF3AA34446
:1012A000C3EB0B0B39465846ADB2FEF71DFE39466F
:1012B00080465846FEF746FF09FB08F945EA014516
:1012C000A94507D92D1908F1FF3803D2A94588BFD0
:1012D00008F1FF3848EA0A48029FA9E7B3FA83F702
:1012E000002F67D18B422CBF4FF000094FF001094E
:1012F00082428CBF4C4649F00104002C96D04FF03E
:10130000010895E7524263EB4303F6433AE7404254
:1013100061EB41014FF0FF3631E704FA08F4C8F100
:10132000200735FA07F329FA07FA270C09FA08FB10
:101330003946504643EA0B020292FEF7D5FD394684
:101340001FFA84F983465046FEF7FCFE029809FB1B
:101350000BF2030C43EA01439A4204D91B190BF127
:10136000FF3BC0F0AD809B1A394618460193FEF74B
:10137000BBFD0199824608463946FEF7E3FE029816
:1013800009FB0AF31FFA80FC4CEA0142934208D998
:1013900012190AF1FF3A04D2934284BF0AF1FF3ACC
:1013A000121905FA08F54AEA0B4EC3EB0208CDF80C
:1013B00008E05AE7C7F1200003FA07FAC24035FAFD
:1013C00000F342EA0A0B21FA00F801FA07F9404655
:1013D0004FEA1B4A43EA0901029151461FFA8BF278
:1013E0000392FEF781FD514681464046FEF7AAFE74
:1013F0000398029B00FB09F2180C14FA07F340EA69
:101400000144A24204D914EB0B0409F1FF3951D372
:10141000A41A514620460193FEF766FD51468046C8
:101420002046FEF78FFE039C019B04FB08F2029C02
:101430001FFA84FC4CEA0140824204D910EB0B00F5
:1014400008F1FF3830D348EA09481FFA83FC1B0C27
:10145000801A1FFA88FE4FEA184A0CFB0EF90CFBA3
:101460000AF203FB0E2103FB0AF301EB19418A4246
:1014700088BF03F5803303EB114E704510D31FFA7C
:1014800089F905FA07F709EB014014BF0022012290
:1014900087422CBF002702F00107002F3FF4C8AE9F
:1014A00008F1FF380027C3E6824284BF584408F1A0
:1014B000FF38C8E7A24284BF09F1FF395C44A7E7BF
:1014C0009A4284BF0BF1FF3B1B194CE72DE9F04F0B
:1014D0000C4683B08046164689461F4615468A4606
:1014E000002B4BD18A425CD9B2FA82F35BB1C3F1D3
:1014F000200001FA03FA28FA00F216FA03F508FAB6
:1015000003F842EA0A0A2E0C50463146AFB2FEF703
:10151000EBFC31464FEA184481465046FEF712FE76
:1015200007FB09F344EA014A534509D91AEB050AB6
:1015300009F1FF3904D2534584BF09F1FF39AA44A8
:10154000C3EB0A0A314650461FFA88F8FEF7CCFC76
:10155000314604465046FEF7F5FD07FB04F748EA1E
:101560000148474506D9013C18EB050802D247451A
:1015700088BF013C44EA094400265CE08B4258D80D
:10158000B3FA83F6002E5BD18B422CBF00220122DE
:1015900085428CBF154642F00105002D49D001243B
:1015A00049E022B911460120FEF79EFC0546B5FA36
:1015B00085F6002E40F0BB80641B2F0C1FFA85FAC5
:1015C000012639462046FEF78FFC39464FEA184B74
:1015D00081462046FEF7B6FD0AFB09F34BEA014BB4
:1015E0005B4509D91BEB050B09F1FF3904D25B45BB
:1015F00084BF09F1FF39AB44C3EB0B0B39465846A6
:101600001FFA88F8FEF770FC394604465846FEF784
:1016100099FD0AFB04FA48EA0148C24506D9013C93
:1016200018EB050802D2C24588BF013C44EA0944D0
:1016300001E0002634463146204603B0BDE8F08F75
:10164000C6F12000B34032FA00F721FA00FB1F4335
:1016500014FA06F228FA00F158464FEA174A1143E5
:1016600000915146BBB20193FEF73EFC5146B54096
:1016700081465846FEF766FD019C009804FB09F37D
:101680004FEA104C4CEA014B5B4505D91BEB070BAD
:1016900009F1FF39C0F08F80C3EB0B0B5146584660
:1016A000FEF722FC514604465846FEF74BFD0198D2
:1016B000009A00FB04F31FFA82FC4CEA01429342B9
:1016C00006D9013CD21903D2934201D9D219013C67
:1016D00044EA0944A8B2D21A2D0C1FFA84FC4FEA3E
:1016E000144300FB0CF700FB03FE05FB0CE105FBBC
:1016F00003F501EB17418E4588BF05F5803505EBF5
:101700001145AA4210D3BFB208FA06F607EB014210
:1017100014BF4FF0000E4FF0010E96422CBF002672
:101720000EF00106002E86D0013C002683E7B5406E
:10173000C6F1200124FA01F928FA01F22F0CB44075
:101740003946484622430092FEF7CEFB39461FFA3F
:1017500085FA83464846FEF7F5FC009B1A0C0AFB07
:101760000BF342EA0144A34203D964190BF1FF3B96
:1017700027D3E41A39462046FEF7B6FB39468146A0
:101780002046FEF7DFFC00980AFB09F31FFA80FCF5
:101790004CEA0144A34208D9641909F1FF3904D283
:1017A000A34284BF09F1FF39641908FA06F8E41A64
:1017B00049EA0B4605E75B4584BF09F1FF39BB44A5
:1017C0006AE7A34284BF0BF1FF3B6419D1E700BF76
:1017D0000000000000000000010003E8000000001D
:1017E00000000003E800000000000200FA06000309
:1017F00000000000003706000000000000000000AC
:10180000F4010000640000000180080800000000EE
:10181000006400000000000000000000C80000009C
:101820001201100102000040D016A10501150102AD
:101830000301000009024300020100C03209040054
:10184000000102020100052400100105240100012D
:10185000042402020524060001070582030800FF94
:1018600009040100020A000000070503024000000D
:101870000705810240000000040309042603540008
:10188000720069006E0061006D00690063004D0028
:101890006F00740069006F006E0020004300740048
:1018A0006C000000320354004D0043004D002D0039
:1018B0003100310036003100200028007600690038
:1018C00072007400750061006C00200043004F003E
:1018D0004D00290020000000524F52000001065226
:1018E0004F4C000002064D5354000003024D565069
:1018F0000000040753415000000507474150000015
:10190000060353544150000703525341500008034B
:101910005347500000090747475000000A0353543B
:101920004750000B0352534750000C0352465300DC
:10193000000D0353494F00000E0747494F00000FA9
:101940000353414300001D0753434F00001E074748
:10195000434F00001F0343434F0000200341434F08
:10196000000027035546300000400755463100006F
:1019700041075546320000420755463300004307F1
:101980005546340000440755463500004507554686
:1019900036000046075546370000470752554E00AF
:1019A00000810553544F5000800042494E00008B87
:1019B000000000000000000000000000010203041D
:1019C000010203040607080902040608002020207B
:1019D00020202020202028282828282020202020DF
:1019E00020202020202020202020202020881010AF
:1019F000101010101010101010101010100404040B
:101A000004040404040404101010101010104141C8
:101A100041414141010101010101010101010101B6
:101A200001010101010101011010101010104242CA
:101A30004242424202020202020202020202020286
:101A40000202020202020202101010102000000026
:101A50000000000000000000000000000000000086
:101A60000000000000000000000000000000000076
:101A70000000000000000000000000000000000066
:101A80000000000000000000000000000000000056
:101A90000000000000000000000000000000000046
:101AA0000000000000000000000000000000000036
:101AB0000000000000000000000000000000000026
:101AC0000000000000000000000000000000000016
:101AD0003131363156313231004142530052454C9A
:101AE00000434F4F52440053544152540053544FFB
:101AF000500053544154555300000000430000006F
:081B00006C6F6700000000009B
:081B080068F6FF7F01000000F8
:101B1000D01A0108000100000001020000080000C6
:101B200001000000020000000000000000000000B2
:101B300000000000000000000000000000000000A5
:101B40000000000000000000000000000000000095
:101B5000000000000000000000C2010000000800BA
:101B600078180108040000007C1801082600000015
:101B7000A418010832000000B00000201A00000084
:101B8000341801084300000020180108120000006A
:101B9000D1930008DD910008ED8F00080190000846
:101BA000059000086590000889900008CD91000814
:101BB000BD9100089991000800000000400000005D
:101BC0001A0354004D00430031003100360031004B
:101BD000000000000000000000000000ED8E000882
:101BE00079E7000879E7000879E7000879E7000855
:101BF00079E7000879E7000879E7000879E7000845
:101C00002D93000879E7000879E7000879E70008D4
:101C100079E700080401000079E70008C98F00088F
:101C200079E7000879E7000879E7000879E7000814
:101C300079E7000879E70008E18F0008010000005B
:101C4000CD190108CC1901083C010020000000005A
:101C50000000000000000000000000000000000084
:101C6000000000000000000000000000FC1A010855
:101C70000000000000000000000000000000000064
:101C80000000000000000000000000000000000054
:101C90000000000000000000000000000000000044
:101CA0000000000000000000000000000000000034
:101CB0000000000000000000000000000000000024
:101CC0000000000000000000000000000000000014
:101CD0000000000000000000000000000000000004
:101CE00000000000000000000000000000000000F4
:101CF00000000000000000000000000000000000E4
:101D000000000000000000000000000000000000D3
:101D100000000000000000000000000000000000C3
:101D200000000000000000000000000000000000B3
:101D300000000000000000000000000001000000A2
:04000005080041109E
:00000001FF
